:020000040800F2
:1000000010B10010A9020008EF020008D5D50008C1
:10001000F3020008F5020008F702000800000000E3
:10002000000000000000000000000000F9020008CD
:10003000FB02000800000000911D01086576000821
:100040000103000803030008050300080530010848
:10005000090300080B0300080D03000891CB0008FA
:100060001103000813030008150300081703000814
:10007000190300081B0300081D0300081F030008E4
:1000800021030008BD5501082503000827030008C7
:10009000919801082B0300082D0300082F03000886
:1000A00091250108B1260108012701087D230108D7
:1000B0001D2601083B030008852401083F030008B2
:1000C00041030008430300084503000847030008F4
:1000D00049030008AD550108ED550108FD5501081B
:1000E000D94C0108530300085503000857030008C2
:1000F000590300085B0300085D0300085F03000864
:1001000061030008D54C01086D75000867030008FD
:10011000455601088D5601086D0300086F0300085D
:10012000591D0008730300087503000877030008D1
:10013000790300087B0300087D0300087F030008A3
:100140008103000883030008850300088703000873
:1001500089030008D55601087D5501080557010897
:100160009103000893030008950300089703000813
:10017000990300089B0300089D0300089F030008E3
:08018000A1030008A30300081D
:100188002C49072291438D462B482C492C4A00F0D4
:100198003EF82C482C492D4A00F039F82C482D49B6
:1001A8002D4A00F034F82D482D492E4A00F02FF83A
:1001B8002D482E492E4A00F02AF82E482E492F4A5B
:1001C80000F025F82E482F49002200F02BF82E4881
:1001D8002E49002200F026F82D482E49091A082930
:1001E80003DB00220260043001601D481D4988427B
:1001F80005D00268043003B4904703BCF7E7002039
:100208008646EC4600200021234A9047FEE78842B4
:1002180007D0521A05D0037801300B700131013A2A
:10022800F9D17047884202D002700130FAE770476E
:100238001A48704710B10010381A02080000002050
:10024800B0070020B0030008B0030008A0F30108BD
:10025800E82102082441012024410120A0F30108DB
:10026800A0F30108A0F30108A0F30108A0F3010816
:10027800A0F30108A0F30108A0F30108381A020846
:10028800B0070020242900200000001010AF001043
:10029800242900202441012025D50008FFFFFFFF65
:1002A8003E48854617F0CEF94EF63470CEF200007F
:1002B800016831F0404101604EF68850CEF20000EE
:1002C800016851F47001016000BF00BF00BFF1EE8A
:1002D800100A50F04070E1EE100A314831490160CF
:1002E800FFF74EBF7047FEE7FEE7FEE7FEE7FEE7D3
:1002F800FEE7FEE7FEE7FEE7FEE7FEE7FEE7FEE7CE
:10030800FEE7FEE7FEE7FEE7FEE7FEE7FEE7FEE7BD
:10031800FEE7FEE7FEE7FEE7FEE7FEE7FEE7FEE7AD
:10032800FEE7FEE7FEE7FEE7FEE7FEE7FEE7FEE79D
:10033800FEE7FEE7FEE7FEE7FEE7FEE7FEE7FEE78D
:10034800FEE7FEE7FEE7FEE7FEE7FEE7FEE7FEE77D
:10035800FEE7FEE7FEE7FEE7FEE7FEE7FEE7FEE76D
:10036800FEE7FEE7FEE7FEE7FEE7FEE7FEE7FEE75D
:10037800FEE7FEE7FEE7FEE7FEE7FEE7FEE7FEE74D
:10038800FEE7FEE7FEE7FEE7FEE7FEE7FEE7FEE73D
:10039800FEE7FEE7FEE7FEE7FEE7FEE700000220D5
:0803A80008ED00E00000000870
:1003B00070B940F20000C1F2000040F2B1310268B1
:1003C0008388C0F6000153833C20012207F080B8E7
:1003D000012800D0704740F2000CC1F2000CDCF89C
:1003E0000010BCF804200A83704700BF70B940F2C7
:1003F0000000C1F2000040F2ED3102688388C0F6CF
:10040000000153830220012207F062B8012800D0C6
:10041000704740F20003C1F2000340F2ED311A6868
:10042000B3F804C0C0F60001A2F818C03C200222B4
:1004300007F04EB810B5441C072C1ADC40F200033C
:10044000C1F2000393F81B1151FA04F010F00100FF
:100450000BD1FFF7ADFF40F23541C0F6000141205E
:100460002246BDE8104007F04DB80020FFF7BEFF60
:10047000F1E710BD10B540F20004C1F20004012202
:100480002068B4F804C004F58871A0F818C084F896
:10049000142119F069FFA06802688388138310BDD6
:1004A00010B540F20004C1F200040022206884F874
:1004B000142104F5887119F057FFA0680268838839
:1004C000538310BD08B503283DD8DFE800F02B1F8B
:1004D0000602BDE80840FFF7CDBF40F20003C1F2BD
:1004E000000340F2C5411A689888126910420CBF97
:1004F0004FF0000C4FF0010CC0F600011920032250
:1005000083F81AC1BDE8084006F0E2BFFFF7C8FF54
:1005100040F2C541C0F600010A200222BDE80840B1
:1005200006F0D6BF40F20000C1F2000040F2C54123
:1005300002688388C0F60001538302200122BDE8CF
:10054000084006F0C5BF08BD40F20003002810B502
:10055000C1F2000304461ADB93F81B0193F81A1149
:1005600011FA04F242EA0001C8B2062C83F81B011A
:1005700000DD10BD0020FFF7A5FF40F24951C0F695
:100580000001621C4120BDE8104006F0BBBF002204
:10059000104683F81B21EEE708B503283ED8DFE8B4
:1005A00000F02B1F0602BDE80840FFF763BF40F2D2
:1005B0000003C1F2000340F299511A689888126949
:1005C000104214BF4FF0000C4FF0010CC0F60001B8
:1005D0003C20032283F819C1BDE8084006F078BF2B
:1005E000FFF75EFF40F29951C0F600013C20022265
:1005F000BDE8084006F06CBF40F20000C1F2000008
:1006000040F2995102688388C0F6000153834FF489
:10061000F5700122BDE8084006F05ABF08BD00BFD2
:1006200010B50346002854D0012848D040F20004F9
:10063000C1F2000494F81C2150B2002820DDD4F847
:100640000C3113F801CB013A4FF0FF3084F81BC195
:10065000C4F80C3184F81C21FFF7ECFE40F2216154
:100660000222C0F600014FF4167006F065FF94F9FF
:100670001C21002A22D104F10C01C4F80C1110BD78
:1006800094F81D21110616D4501EC2B2032B84F813
:100690001D2152D0130648D44FF0FF30FFF754FF0E
:1006A00040F22161C0F600014FF416700322BDE84C
:1006B000104006F041BF032084F8180110BD40F23D
:1006C0000002C1F2000292F81911C1B982F81801B2
:1006D00010BD40F20002C1F2000282F8193102237B
:1006E00082F81831FFF758FF40F22161C0F600018F
:1006F0004FF47A700122BDE8104006F01DBF02F1F0
:100700000C03CC2182F81B11C2F80C314FF0FF30E2
:10071000FFF790FE40F22161C0F600014FF4167021
:100720000222BDE8104006F007BF40F2000CC1F203
:10073000000C03218CF8181110BDD4F80C3194F87A
:100740001B2103F8012B94F81D21C4F80C31A1E7FB
:1007500010B540F20004C1F200040346002084F802
:100760001C3184F81D11FFF75BFF94F81801022873
:10077000FBD094F8180110BDF8B540F20004C1F2A6
:1007800000044FF490720D460646002120461DF0ED
:10079000BBF82946304608F0D9FE014604F58870BA
:1007A0000127A1602660A58019F09AFE022084F836
:1007B0001501C4F8105184F8147184F81771FFF70B
:1007C00059FE384617F0ECFA002384F81831F8BDCA
:1007D000DFED147AC7EE807A08B59FED137A77EED5
:1007E000C77A17EE900A1AF0BBFF41EC100B1CF011
:1007F000F3FA51EC100B1AF0CFFF07EE100A9FED41
:100800000B6ADFED0B7A67EE076A47EE067A26EE93
:10081000877ADFED086A47EE267A9FED070A37EE02
:10082000C00A08BD0022A1480050C347B9FCD5400A
:100830002A89274396210E3D00808843000000004E
:100840002DE9F04F2DED088BE14CE248E24D8FB0E1
:1008500002F07EF8D4F86801016882884B699FED48
:10086000D87B9FEDDE9A1A428DED087B8DED0C7BD7
:100870008DED0A7B4FF000060CBF4FF000084FF0E3
:100880000108DFEDD7AA0496CDF80880F0EE498A7A
:10089000B0EE498A0396002160780BF0C7FAD4F8CD
:1008A0007C61276C0196606CA16CE26C236DD4F8BE
:1008B00054E0D4F85880D4F85CA0266ED4F880C0F8
:1008C0000596666ED4F884B00696A66ED4F8889025
:1008D0000796E66F84449144D4F88C00D4F89420B1
:1008E000C4F880C08B44D4F89010C4F884B0BF1909
:1008F00003EB000C08EB0206D4F89830D4F89C8087
:10090000E7670EEB0107DDF814E0D4F8A0100AEB5E
:1009100003000EEB080A069BDDF81CE0D4F8A48067
:10092000C4F888905A180EEB0803D4F8B490D4F8A1
:10093000ACE0C4F88CC0C4F89070D4F8B0C0E76ED6
:10094000C4F89460216FD4F8A860C4F8A020C4F85B
:10095000A430626FA36FC4F8980062447144206CA5
:10096000C4F89CA04B44BE19C4F8A860C4F8B020D9
:10097000C4F8B430C4F8AC101AF024FE92A3D3E942
:1009800000231BF08BF800230022C3F6D0731BF06A
:1009900085F81AF001FFD4ED577A0AEE100A95EDAA
:1009A000D67A7AEE277A48EE077A95EDD97A48EE2C
:1009B000877A95EDDC7A49EE077AD4F84480D4F84A
:1009C00048A095EDDFAA404687EE8AAA1AF0FAFD04
:1009D0007DA3D3E900231BF061F800230022C3F6B6
:1009E000D0731BF05BF81AF0D7FED4ED587A06EE00
:1009F000900A95EDD77A76EEA77A48EE077A95EDCC
:100A0000DA7A48EE877A95EDDD7A49EE077A95ED48
:100A1000E07AF1EE677A5046C7EE879A1AF0D2FD77
:100A200069A3D3E900231BF039F800230022C3F6A1
:100A3000D0731BF033F81AF0AFFED4ED597A06EEFE
:100A4000900A95EDD87A76EEA77A48EE077A95ED7A
:100A5000DB7A48EE877A95EDDE7A49EE077A95EDF6
:100A6000E17AF1EE677AC7EE877AD4F8203195ED16
:100A7000E27AF0EE4A6A49EE876A95EDE36A95ED0F
:100A8000E47A47EE866AB0EE696A0AEE076AD5ED47
:100A9000E55AD4ED3E4A07EE103A07EEA56A04EE99
:100AA000A67A94ED3D5A05EE467AF6EE005A27EE08
:100AB000257A95EDE64AD5EDE73A84ED487AD4F803
:100AC000243107EE103A06EE247A06EE857A69EEB6
:100AD000A39A27EE257A4AEE049A84ED497AD4F84F
:100AE000283179EEA79A07EE903A77EEA97A67EE69
:100AF000A55AC4ED4A5A0CF009F9049E8EB1E66C71
:100B0000D4F88870216DD4F88C00D4F89020636DEF
:100B1000BF1B411AD21AC4F88870C4F88C10C4F8EC
:100B20009020DDF804A01AF0010640F00684E06F82
:100B30001AF048FD24A3D3E900231AF0AFFF0022E6
:100B40004FF07F531AF0AAFF1AF026FE0346D4F89E
:100B50008000C4F8B8301AF035FD1BA3D3E9002398
:100B60001AF09CFF00224FF07F531AF097FF1AF003
:100B700013FE0346D4F88400C4F8BC301AF022FDFA
:100B800011A3D3E900231AF089FF00224FF07F530D
:100B90001AF084FF1AF000FE0346D4F88800C4F867
:100BA000C0301AF00FFD08A3D3E900231AF076FF36
:100BB00000230022C3F6D0731AF070FF12E000BFCA
:100BC00000000000000000004BD4AE44D99AD43E8F
:100BD00020010010A0F30108B40200100000000082
:100BE000711B7D3F1AF0D8FD0346D4F88C00C4F881
:100BF000C4301AF0E7FC0FF2D053D3E900231AF007
:100C00004DFF00230022C3F6D0731AF047FF1AF0FD
:100C1000C3FD0346D4F89000C4F8C8301AF0D2FCE3
:100C20000FF2A453D3E900231AF038FF0023002267
:100C3000C3F6D0731AF032FF1AF0AEFD0346D4F8B3
:100C40009400C4F8CC301AF0BDFC0FF27C53D3E909
:100C500000231AF023FF00230022C3F6E0731AF0EA
:100C60001DFF1AF099FDC4F8D000D4F898001AF0CE
:100C7000A9FC0FF25453D3E900231AF00FFF00230D
:100C80000022C3F6E0731AF009FF1AF085FD03464F
:100C9000D4F89C00C4F8D4301AF094FC0FF2285316
:100CA000D3E900231AF0FAFE00224FF07F531AF026
:100CB000F5FE1AF071FD0346D4F8A000C4F8D83050
:100CC0001AF080FC0FF20053D3E900231AF0E6FE7D
:100CD00000224FF07F531AF0E1FE1AF05DFD03464B
:100CE000D4F8A400C4F8DC301AF06CFC0FF2D8433E
:100CF000D3E900231AF0D2FE00224FF07F531AF0FE
:100D0000CDFE1AF049FD0346D4F8A800C4F8E0303F
:100D10001AF058FC0FF2B043D3E900231AF0BEFEDC
:100D200000224FF07F531AF0B9FE1AF035FD03464A
:100D3000D4F8AC00C4F8E4301AF044FC0FF2884355
:100D4000D3E900231AF0AAFE00224FF07F531AF0D5
:100D5000A5FE1AF021FD0346D4F8B000C4F8E8302F
:100D60001AF030FC0FF26043D3E900231AF096FE2C
:100D700000230022C3F6E0731AF090FE1AF00CFD77
:100D8000C4F8EC00D4F8B4001AF01CFC0FF238439D
:100D9000D3E900231AF082FE00230022C3F6E07399
:100DA0001AF07CFE1AF0F8FCC4F8F000D4F8D01069
:100DB000D4F8EC20D4F8F030E66707EE101A06EE0F
:100DC000102AF7EE047A37EE677ADFEDF96A36EE2D
:100DD000676AF3EE097AF0EE674A47EE264A46EE76
:100DE000267A9FEDF4AADFEDF49A34EE8A7A77EE54
:100DF0008A7A94ED3F6AD4ED406A27EE297A67EE4D
:100E0000A97A06EE2A7A46EEAA7A00EE103A94ED16
:100E1000418A84ED3F7AC4ED407AC4F88060C4F81A
:100E20008460C4F88860C4F88C60C4F89060C4F82A
:100E30009460C4F89860C4F89C60C4F8A060C4F8DA
:100E4000A460C4F8A860C4F8AC60C4F8B060C4F88A
:100E5000B460FFF7BDFC28EE2A8A30EE0A0AB0EE35
:100E6000485A00EE295AD4F8B820D4F8BC10D4F867
:100E7000C030D4ED587A04EE902A06EE901A94ED24
:100E8000577AB3EE048A35EE488AD5EDD75A95EDF8
:100E9000D66A76EEA76A34EE877A48EE256A08EEBF
:100EA000067A68EE088AD5EDDA4A95EDD96A04EE3D
:100EB000103AD4ED597AD5EDD85A48EEA46A08EE26
:100EC000867A28EE889AD5EDDD4A95EDDC6A74EED7
:100ED000277A48EE257A49EE246AD5EDDB5A09EEE9
:100EE000067A48EEA57AD5EDDF5A95EDE06A87EEF1
:100EF000257AF1EE666AC6EE866AD5EDDE4A49EEDF
:100F0000247A95EDE16AF1EE677AC7EE867AD5ED3F
:100F1000E25AF0EE474A46EEA54A95EDE46AF0EE55
:100F2000645AF0EE664A47EE064A95EDE34AB0EEA3
:100F3000646AD5EDE54A47EE845A07EEA46AD5ED1A
:100F4000E73A95EDE63A94ED3D4A66EEA33AD4EDE4
:100F50003E4A47EE033A64EE066A25EE847A54EE82
:100F6000A56A06EE247A73EEA77AC4ED4B6A84ED87
:100F70004C7AC4ED4D7AD4F8D430DFED907A07EE98
:100F8000103A27EE277AD4ED437A67EE299A47EE96
:100F9000AA9A84ED415A84ED425AC4ED439AD4F89A
:100FA000D810D4F8DC20D4F8E03095ED976A05EE3F
:100FB000101AD5ED9A2A95EDA63AD5EDA36AD5ED8E
:100FC000A77A03EE902AD5ED985A95EDA47A35EEDE
:100FD000065A95ED9B1A08EE225A48EE036A95EDE3
:100FE000A92A95ED996A73EEA55A08EE277A03EEC1
:100FF000903AD5ED9D0AD5EDAA2A48EE015A33EE76
:10100000866A95ED9E1AD5EDA03A48EE826A08EE02
:10101000A05A08EEA27A95EDAC2A69EE233AD5EDF6
:10102000AD2A48EE815AD5ED9C1A95EDA83AD5ED3A
:10103000A57A49EE026A35EE235A09EE227A08EEC5
:10104000216A48EE037A73EEA55A95EDAB3AD5EDD9
:101050009F1AB1EE455AC5EE266A85EE877A48EEAC
:10106000837A08EEA16A95EDAE3A49EE037A33EE43
:10107000866AD5EDAF5AB1EE466AC6EE277AB0EE73
:10108000665A95EDB16A07EE255AF0EE475A46EEDC
:10109000865AD5EDB03AB0EE656AD5EDB25A07EE94
:1010A000A35A07EEA56AD5EDB43AD5EDB35A27EEAB
:1010B000237A06EEA57A64EE066A24EE054A54EE1B
:1010C000856A04EE864A77EE277AC4ED4E6A84ED8F
:1010D0004F4AC4ED507AD4F8E420D4F8E8309FEDBC
:1010E000386A05EE902A05EE103ADFED366A94ED87
:1010F000457AD4ED467A75EE865A35EE066A05EEE7
:10110000A67A46EE267A95EDEA6AF6EE006A27EEB2
:10111000267A67EEA67AB4EE4A6AF1EE10FA84ED0A
:10112000457AC4ED467A40F0B58184ED477AD4F82B
:10113000C430029904EE903A94ED544AD4F8C83081
:10114000D4F8CC20002900F0738194ED563A03EED8
:10115000902A95EDB72A73EEC31A95EDBA1A72EE7E
:10116000612A48EE012AD5EDBD0A48EEA02A95ED88
:10117000C07A49EE072ABFEE005AD5EDB55AD5ED33
:10118000B89A95EDBB0AD5EDBE0A94ED557AD5ED2A
:10119000B66A95EDB91AD5EDBC1A95EDBF2A03EEE6
:1011A000903AB0EE453AF1EE622AFF2312E000BF1A
:1011B000FFFF794300000000A323393CEA4EEB40D7
:1011C0001283A03E098603474BD4AE44D99AD43E3D
:1011D000FB01863534EEC4AA33EEC74A4AEE035A01
:1011E00044EE056AD5EDC43A95EDC53A95EDC16A70
:1011F00095EDC2AA49EE885A08EE236A41EE086AC4
:1012000008EE03AA95EDC71A95EDC87AD5EDC67A12
:10121000D5EDC39A40EE285A08EE816A41EEA86ADD
:1012200008EE87AAD5EDCABA95EDCBBA48EE279A53
:1012300095EDC95A09EE2B6A42EE096A09EE0BAA2E
:1012400040EE895A48EE859AD5EDCC4AC5EE860A1D
:10125000DDF80CC084F890310CF1010BCDF80CB026
:1012600086EE8A1A49EE249A95EDCD4AC2EEA9BAC5
:10127000D5EDCF3AF0EE602AF0EE417A41EE042A45
:1012800040EEA37A95EDCE3A95EDD02A4BEE832A27
:101290004BEE827AD5EDD21AD5EDD16A94ED3D7A36
:1012A00021EE210AD4ED3E5A00EEA60A27EE27BA17
:1012B00022EE87AA15EEA2BA07EEA5AA70EE2B9A27
:1012C00084ED51BA84ED52AAC4ED539AD4F8C40007
:1012D0001AF046FA02460B46DDE90A011AF09AFABC
:1012E000CDE90A01D4F8C8001AF03AFA02460B46D2
:1012F000DDE90C011AF08EFACDE90C01D4F8CC002E
:101300001AF02EFA02460B46DDE908011AF082FABD
:10131000CDE90801D4F88871D4F884617A0006EE2A
:10132000102A5FED554AB8EE465AC4F8806125EEA2
:10133000244A84ED634A0BF0F3FCD4F86831029937
:101340001A689B88566933420CBF002001208142F5
:101350006AD05269134060D003981AF01BF988468E
:10136000814643464A46DDE90A011AF04DFC1AF06F
:1013700013FA09EE900A43464A46DDE90C01C4ED32
:10138000549A1AF041FC1AF007FA0AEE100A434682
:101390004A46DDE9080184ED55AA1AF035FC1AF039
:1013A000FBF9DDF80C80C4F85801B8F1640F0BEEBE
:1013B000100A79DD79EEA92A012712EE900A029728
:1013C0001AF0CEF902460B46DDE90A011AF020FABE
:1013D0007AEE0A5ACDE90A01A8F1020A15EE900A3E
:1013E000CDF80CA01AF0BCF902460B46DDE90C0161
:1013F0001AF00EFA3BEE0B0ACDE90C0110EE100AC2
:1014000004971AF0ADF902460B46DDE908011AF01F
:10141000FFF9CDE90801FFF73EBA4FF00109CDF819
:1014200010900293FFF737BA00270497FFF733BAFB
:1014300005EE102A94ED56BA95EDB72A75EE4B9A43
:10144000D5EDBA1A39EE826A08EE216AD5EDBD6A89
:1014500008EEA66AD5EDC00A09EE206AB7EE005A7A
:1014600003EE903AD5EDB55AD5EDB89A95EDBB0A95
:10147000D5EDBE0A94ED557AD5EDB66A95EDB91A5B
:10148000D5EDBC1A95EDBF2AF1EE462AB0EE453AED
:1014900001239FE6F7EE005AB4EE656AF1EE10FA0A
:1014A00007D1C4ED477A42E6012602960496FFF77B
:1014B000F2B9B0EE000AB4EE406AF1EE10FA7FF431
:1014C00036AE77EE277A67EEA66AC4ED476A2EE657
:1014D00010B540F2B423C1F200032DED028BDFED15
:1014E0000C7A93ED968A28EE278A40F22014B0EE0B
:1014F000480A1BF07DFFC1F2000484ED3D0AB0EE06
:10150000480A1BF0DDFB84ED3E0ABDEC028B10BDEA
:1015100035FA8E3C000000002DE9F04F2DED048BD4
:10152000642083B017F0C4F932200BF061FB9FED0B
:101530008A7B40F22015C1F200055BEC17AB8DED04
:10154000007BD5F88041D046D9463226D5F8803187
:10155000A342FBD0D5F88041D5F8B8001AF000F9C5
:1015600002460B46404649461AF054F98046D5F8E3
:10157000BC0089461AF0F4F802460B46504659461C
:101580001AF048F98246D5F8C0008B461AF0E8F800
:1015900002460B46DDE900011AF03CF9013ECDE9B7
:1015A0000001D3D1D5ED420A40F2B4240023C1F2A8
:1015B00000040022C4F2490340464946B3EE048ABF
:1015C00030EEC88A1AF020FBD4EDD68A28EE280A1D
:1015D000064610EE100A0F461AF0C2F802460B46F5
:1015E000304639461AF016F968EE088A94EDD99A11
:1015F00028EE897A064617EE100A0F461AF0B0F860
:1016000002460B46304639461AF004F928EE289A6D
:10161000D4EDDC7A69EE276A064616EE900A0F468C
:101620001AF09EF802460B46304639461AF0F2F898
:101630001AF0B2F806EE100A0023F1EE465A002224
:10164000C4F2490350465946C5ED575A1AF0DCFA20
:1016500094EDD75A68EE054A064614EE900A0F46F6
:101660001AF07EF802460B46304639461AF0D2F898
:1016700094EDDA4A68EE843A064613EE900A0F4675
:101680001AF06EF802460B46304639461AF0C2F898
:1016900094EDDD3A69EE032A064612EE900A0F46F3
:1016A0001AF05EF802460B46304639461AF0B2F898
:1016B0001AF072F802EE100A0023F1EE421A00222C
:1016C000C4F24903DDE90001C5ED581A1AF09CFA8D
:1016D00094EDD81A28EE018A064618EE100A0F4635
:1016E0001AF03EF802460B46304639461AF092F898
:1016F000D4EDDB0A68EEA08A064618EE900A0F4683
:101700001AF02EF802460B46304639461AF082F897
:1017100094EDDE0A29EE009A064619EE100A0F46ED
:101720001AF01EF80B460246394630461AF072F897
:101730001AF032F807EE100A0023F1EE477AC5EDF1
:10174000597AC5F82C31C5F83031C5F8343103B0B9
:10175000BDEC048BBDE8F08F00000000000000002D
:101760002DE9F04F4FF2B43040F220189DB0C1F295
:101770000008C0F601004FF4805A01F0E9F8C4F205
:10178000020A4FF4CA72002140461CF0BDF8FFF770
:101790009FFE4FF48061504607F0D8FEB0F804C0B9
:1017A0000268C8F868014FF48071A2F818C050466A
:1017B00007F0CCFE0646C820C8F86C6117F078F830
:1017C000D8F86C311C689D881420258317F070F8B8
:1017D000D8F86C01076881881420798317F068F8BD
:1017E00050464FF4805107F0B1FE4FF4006B026891
:1017F0008688C8F87001C4F2020B56834FF400418A
:10180000584607F0A3FE03688488C8F874015C8317
:1018100019A818F065FE002000244FF0030AFD25EA
:10182000C4F2020019A919958DF868A08DF86B40D3
:1018300018F09AFD4FF48060C4F2020019A93F2706
:10184000CDF864A046F2104918F08EFD584619A94B
:10185000C4F20209199718F087FD01214FF4E060E6
:1018600018F014FFA3214846C8F8781142F2083650
:1018700018F08CFA40F2B0726023C4F20106C2F292
:1018800000024FF0040B48466946029201964FF45D
:10189000807204934FF480654FF440334FF4006737
:1018A0004FF400560A9306950797089609920094FC
:1018B00003940594CDF82CB0CDF830A00D940E947F
:1018C00018F066FB01224846182118F01DFC4FF263
:1018D0003D014846C9F2000118F02EFC012148469E
:1018E00018F0B4FB4FF0010938251BA88DF86C5097
:1018F0008DF86D408DF86E408DF86F900BF078FE8E
:1019000015A818F0CBF916274FF4804115A84FF40D
:101910000055C4F2010517911597169418F0A4F913
:101920000FA818F097F910260FA928468DF85060D7
:101930000F948DF840908DF841901194139418F005
:101940005DF90721022328464A4618F0B7F902221A
:1019500007211346284618F0B1F90721022328462B
:10196000524618F0ABF90721022328465A4618F0D0
:10197000A5F90E2105220223284618F09FF90E2111
:1019800006220223284618F099F907220223284646
:101990000E2118F093F90E2128460822022318F090
:1019A0008DF90F2109220223284618F087F90F210B
:1019B0000A220223284618F081F90F210B22022364
:1019C000284618F07BF90F210C220223284618F034
:1019D00075F908210D220223284618F06FF9082115
:1019E0000E220223284618F069F908210F22284602
:1019F000022318F063F9102228460223082118F068
:101A00005DF94FF4045749462846C4F2010718F01F
:101A1000A5F90FA818F01EF9102238460FA98DF865
:101A200050200F948DF840908DF8419011941394AC
:101A300018F0E4F83846092102234A4618F03EF926
:101A4000022238460921134618F038F93846092190
:101A50000223524618F032F93846022309215A4629
:101A600018F02CF9384605220223594618F026F9B9
:101A7000384606220223594618F020F93846072234
:101A80000223594618F01AF938460822594602230B
:101A900018F014F9384605210922022318F00EF92E
:101AA000384605210A22022318F008F93846052194
:101AB0000B22022318F002F9384605210C220223DA
:101AC00018F0FCF8384606210D22022318F0F6F82B
:101AD000384606210E22022318F0F0F83846062177
:101AE0000F22022318F0EAF84FF4085610220223BE
:101AF00006213846C4F2010618F0E0F80FA818F0E5
:101B0000A9F8304610230FA98DF850300F948DF8A6
:101B100040908DF841901194139418F06FF80223BF
:101B2000304651464A4618F0C9F8022330461A4654
:101B3000514618F0C3F8304602235146524618F079
:101B4000BDF83046022351465A4618F0B7F83046E1
:101B50000A210522022318F0B1F830460B21062293
:101B6000022318F0ABF80221304607220B4618F08A
:101B7000A5F80221304608220B4618F09FF80221F2
:101B8000304609220B4618F099F8022130460A2205
:101B90000B4618F093F830460D210B22022318F063
:101BA0008DF80C2230460223114618F087F8304693
:101BB0000D220223214618F081F830460E2202231E
:101BC000214618F07BF8304602230F22214618F0F8
:101BD00075F8102202233046214618F06FF8484667
:101BE00018F0C6F82846494618F05EF838464946C7
:101BF00018F05AF83046494618F056F8214648463B
:101C00000AF08EF84FF2C0310646C0F601015820A6
:101C100088F8016016F0D8FD40F67006C2F20006A2
:101C2000074640F6410007F5AE73214645F60A0225
:101C3000C0F60000376015F08FFF8446284688F80C
:101C400000C018F085F8642016F0AAF8D8F8D01073
:101C5000D8F8EC20D8F8F00003EE901A02EE902AA3
:101C6000B7EE043A33EEC30ADFED376A32EEC36AE9
:101C7000F3EE091AF0EE615A40EE265A46EE261AA5
:101C800000EE100AC8ED3F5AC8ED401AFEF7A0FD5D
:101C9000D8F8D430DFED2D0A01EE103A61EE207A4B
:101CA00088ED410AC8ED437AFFF736FCD8ED437A58
:101CB000B2EE017AF4EEC77AF1EE10FA22D49FED7B
:101CC000244AF4EEC47AF1EE10FA31D4F3EE014A6C
:101CD000F4EEE47AF1EE10FA1FD49FED1E5AF4EE02
:101CE000C57AF1EE10FA0AD54FF200400021C4F295
:101CF000A001C0F60100C8F8101100F029FE1DB0C7
:101D0000BDE8F08F4FF2C4304FF08041C0F60100C3
:101D1000C8F8101100F01CFEF1E74FF2EC304FF064
:101D20008142C0F60100C8F8102100F011FEE6E77C
:101D300000234FF2D830C4F24003C0F60100C8F8C7
:101D4000103100F005FEDAE7FFFF7943EA4EEB4081
:101D5000CDCC4C416666AA4110B54FF4C84CC4F2D4
:101D6000020CDCF800104FF23D02C9F20002CCF880
:101D7000082048F22000C1F2000001EA000323B964
:101D800040F2B073C2F2000300E0864B40F2201232
:101D9000C1F20002B3F848C0B3F84E108C44B3F857
:101DA00054008444B3F85A106144506808185060D5
:101DB000B3F802C019898C44D8898444998A614453
:101DC000906808189060B3F804C059898C44188A48
:101DD0008444D98A6144D0680818D060B3F800C040
:101DE000D9888C4498898444598A614410690818B8
:101DF0001061B3F818C0D98B8C44988C8444598DE9
:101E00006144506908185061B3F830C0D98E8C44D1
:101E1000988F8444B3F84210614490690818906127
:101E2000B3F81CC0D1690CEB0100D061B3F840C01D
:101E3000116A0CEB01001062B3F81AC0198C8C44C3
:101E4000D88C8444998D6144506A08185062B3F864
:101E500032C0198F8C44D88F8444B3F84410614445
:101E6000906A08189062B3F84AC0B3F850108C44D6
:101E7000B3F856008444B3F85C106144D06A081883
:101E8000D062B3F828C0D98D8C44988E8444598F81
:101E90006144106B08181063B3F84CC0B3F85210CB
:101EA0008C44B3F858008444B3F85E106144506B1E
:101EB00008185063B3F822C0916B0CEB01009063DB
:101EC000B3F846C0D36B0CEB0301D163D2F87801B1
:101ED00000F10103C2F87831A42B62D14FF44060C5
:101EE000C4F20000416A96464FF00003C2F8783110
:101EF000D2F87C2102F10104CEF87C4114F0010FEC
:101F00000BD040F2201CC1F2000CDCF868311A68DA
:101F100054699B88234242D0538340F22014C1F27B
:101F20000004636823644FF000036360A06860648A
:101F3000A360E268A264E3602069E06423616269EF
:101F400022656361A0696065A361E269A265E361DE
:101F5000206AE0652362626A22666362A06A606644
:101F6000A362E26AA266E362206BE0662363626BAF
:101F700022676363A06B6067A363E26BA267E3639E
:101F8000D4F884010A1AC4F88821C4F8841107F02F
:101F90002BFA60780AF086F807F02CFA10BD13834C
:101FA000BBE710BD100800202DE9F04101FB02F451
:101FB000A3B28846064604211846174616F0E2FBEF
:101FC0001FFA88F105460346BAB2304605F0C6FB53
:101FD0009FED030A28462146BDE8F04105F072BB9B
:101FE000000000002DE9F04F2DED028B8BB0B2F810
:101FF00000A00692B2F802B044880588069E0990B7
:102000009FED8C8A0BFB0AF30891A542B4BFAA4648
:10201000A2467068CDF810A0B0EE480A194605F047
:1020200051FB5246002A00F06682099B5A680292D0
:10203000DDF80880029E4FEA840B611C08EB0B0A56
:102040004FF000088800043E444505900096079034
:10205000CDF80CA0F0EE485A40F3E3800098D0EDA4
:10206000017AF0EE486A47EEA76A6FEA080C08F1B9
:1020700001030CEB0409021D9C4209F00101F0EE82
:10208000667A15DD41B10432D2ED000A01339C427B
:10209000164640EEA07A0BDD92ED010A40EE007A82
:1020A00092ED027A023308329C4247EE077AF3DC63
:1020B000B1EEE76A0299D1ED000AF4EEC80AF1EE3A
:1020C00010FAC8BFB1EE466AB4EE486AF1EE10FAF3
:1020D000894600F0A980069B5A885E6802FB088A40
:1020E00006EB8A0E8EED006AD1ED001A08F10106AA
:1020F00031EEC61AB542019681ED001A7ADD0398D9
:10210000009FB446C246464654456EDD6FEA06035C
:102110001A19D0ED001A97ED012A731C02F001087C
:10212000F0EE657A3A1D9C42014641EEC27A1EDD10
:10213000B8F1000F0AD0043290ED010A92ED007A56
:102140000133011D9C4240EE477A10DD91ED013ACA
:10215000D2ED013A43EE637A91ED022AD2ED022AE2
:102160000233083108329C4242EE627AEEDCD9ED4D
:10217000006A26EE265A90ED004AC7EE857AF143B2
:10218000721C01EB04080346944208F0010107F1B8
:102190000408D7ED014A07EEE44AA3EC014A24DD26
:1021A00061B108F1040893ED005AD8ED006A07EE1A
:1021B000E65A01329442A3EC015A16DDD3ED000A2F
:1021C00098ED011A47EEC10A9E46EEEC010A98ED21
:1021D000020A93ED017A07EEC07A02327346944206
:1021E000A3EC017A08F10808E8DC0CF1010C654564
:1021F000584489DCDDF808A00598039E009B0799E8
:102200000AEB000C1A18DDF810A0CDF808C0701801
:10221000019E0092564503900ED0B04644453FF7CC
:102220001DAFF0EE487A43E700200BB0BDEC028B07
:10223000BDE8F08F00000000049A02F1FF3B002A85
:1022400048D002FB04B76FEA0403B800DDF824A00D
:10225000069F009411464FEA8309A2008D4201F1C6
:10226000FF3C33DDB7F80280DAF804407B680CFBF2
:1022700008162418013E03EB8606D4F800806FEAA6
:10228000010C4B1C0CEB050EC6F8048004369D4275
:102290000EF0010C144419DDBCF1000F07D0D4F886
:1022A00000C001339D4246F804CF14440EDDD4F83B
:1022B00000C004EB020EC6F804C0DEF80040023392
:1022C000B46008369D420EEB0204F0DC013948444C
:1022D000C4D1009C089B002B00F00B81089D1A883C
:1022E0006988686801FB02F11FED2E0A05F0EAF922
:1022F000049E631E9E4225DC621C686802FB03FC90
:1023000000EB8C0EC2EB82719D1BA31E89004FF067
:102310007E509E42CEF8000005F001050EEB010252
:1023200010DC2DB1049D1060013B9D420A4409DC84
:10233000DDF810A010605518023B9A45286005EBA7
:102340000102F5DDBBF1FF3F00F0D380089E099A42
:1023500075685268631C03FB0BF081006D18C3EBBA
:10236000837301959B00E6431FED4E5A0138049399
:10237000019B5118B50002EB8006F0EE455A009122
:10238000059502960393A200019800994FF07E559F
:10239000056091ED006AB4EE456AF1EE10FA8846E8
:1023A00000F090805C4540F38D800699039D4E8837
:1023B0004B6806FB0BB703EB8709029FDC465E46C2
:1023C000D7ED017A95ED003AF0EE652A43EE672AE3
:1023D0006FEA06031919731C381D9C4201F0010AAB
:1023E000F0EE627A05EB020121DDBAF1000F0AD0AE
:1023F000043091ED004AD0ED004A01339C4244EE96
:10240000647A114413DDD1ED003A90ED014A01EBFD
:10241000020A43EEC47A90ED023ADAED002A023362
:1024200008309C4242EEC37A0AEB0201EBDC99EDE4
:10243000000A26EE007AD7ED016AC7EE877AF043EC
:10244000711C00EB040E8C420EF0010007F1040A2F
:1024500005EB0203D5ED004A47EEE64AC5ED004A1A
:1024600028DD70B10AF1040A93ED006ADAED003A52
:1024700007EEE36A01318C4283ED006AD6461344CD
:1024800018DD9AED012AD3ED001A47EEC21A03EBCC
:10249000020EC3ED001A9AED021ADEED000A47EEB5
:1024A000C10A02318C42CEED000A0AF1080A0EEB95
:1024B0000203E6DC0CF1010C0435644502DD98ED05
:1024C000006A7DE704990098019DDDF80CC046186C
:1024D0006B180096029D059E01930BF1FF3BAD1911
:1024E0000CEB060ABBF1FF3F0295CDF80CA07FF480
:1024F0004BAF012099E64FF0FF3BEBE62DE9F04FA3
:1025000016888BB01E80B2F800A0149CA3F802A01D
:10251000A4F800A01D46DDF854A00B88B2F802E034
:10252000AAF80030B2F800C0A4F802E00E4609880C
:10253000AAF802C005915488079029461046149ABB
:10254000FFF750FD30462946159A05F00BF9059B1B
:10255000002B00F09480621C04F1FF3CA000C2EB51
:102560008271CDF810C00690002004FB04F30390A4
:10257000880004990190013B4FEA8C0A02FB01F2AA
:102580009800CDF808A008920990049A01326CD006
:10259000DDF850B0DDF85490DBF80400099E029F8E
:1025A000D9F80450DDF81C800899D8F804903A1D39
:1025B0006FEA040300EB060C049E00EB8108AD18E3
:1025C0004FEA830B731C9C425CDD09EB070292ED22
:1025D000017A55ED017ADCED016A46EEC77A6FEAC1
:1025E000030E01330EEB040104329C4201F0010A98
:1025F00045ED017A28460CF1040125DDBAF1000F02
:102600000DD004310432D1ED002A92ED003A42EEB1
:10261000C37A01339C428E4645ED017A14DD91ED7B
:10262000011AD2ED011A41EE617A023340ED017ACE
:1026300091ED020AD2ED020A40EE607A08310832CA
:102640009C4240ED017AEADC98ED002AC7EE827ADE
:10265000013EDDF804A009EB0700043D043F731CB4
:10266000D044DC44C0ED007AACD10299069B0398BB
:10267000CA18059B029201308342039085DC0BB09F
:10268000BDE8F08F55ED017ADEE700BF08B510F028
:10269000E3FB04F0BDFE11F0D5FC09F0FDF914F0E8
:1026A00095FF06F0A9F904F057FD0BF0CFFE09F0F5
:1026B0008DFF0AF011FB0FF049F910F087F906F0D1
:1026C00061FD0AF0B5F90DF003FD0AF00DFF10F001
:1026D000A1FE16F027F914F039FF4FF21440C0F6AE
:1026E000010000F035F94FF23840C0F6010000F06B
:1026F0002FF940F27463C2F200034CF6FF12C3F6E6
:102700009A321A60BDE8084015F0CCBA40F678035A
:10271000C2F20003586D12F0DBBE00BF2DE9F04796
:10272000D743154687EA0712D4B240F6B0522609BD
:10273000C2F2000286F0FF0848EA042C96798CEA7F
:10274000C40989EA060484EA04175FFA87FC4FEAA1
:10275000192440F6681E84EA1C17C2F2000E87EAAC
:102760000C2888EACC049EF800709EF801E01FFA5D
:1027700084FC8CEA070989EA09185FFA88F94FEAAC
:102780001C2484EA191444EA092888EAC90989EA58
:102790000E0C8CEA0C14E4B24FEA192888EA141CD7
:1027A0008CEA042989EAC4081FFA88F484EA000C38
:1027B0008CEA0C1982B05FFA89FC240A84EA1C14A2
:1027C00044EA0C288DF802600C460136FE218DF893
:1027D00001508DF800108DF803708DF804E08DF82D
:1027E0000500967188EACC0C002D52D094F800E0D8
:1027F0008EEA0C0888EA0812D1B24FEA1C2C621C3F
:102800006E1E52FA86F6E0438CEA1119301849EA36
:10281000012EB24200F001008EEAC10C39D098B10D
:1028200012F8018B88EA0C0989EA091E5FFA8EF812
:102830004FEA1C2080EA181181EA082080EAC801CA
:10284000B2421FFA81FC24D0104692F8019010F891
:10285000011B81EA0C0282EA0211C9B24FEA1C276D
:1028600087EA111C8CEA012282EAC1011FFA81FC6D
:1028700089EA0C0E8EEA0E185FFA88F14FEA1C22E4
:1028800082EA111242EA0129421CB24289EAC10CD1
:10289000DAD183EA0C0181EA01124FEA1C20D1B29D
:1028A00080EA111383EA012282EAC10083B2FE2189
:1028B00000205FFA83F84FEA1329FFF727FF9DF8FE
:1028C00001100020FFF722FF9DF802100020FFF703
:1028D0001DFF9DF803100020FFF718FF9DF804105E
:1028E0000020FFF713FF9DF805100020FFF70EFFF3
:1028F00015B3002705F1FF330126E15D384603EAF1
:10290000060AFFF703FFB54216D9BAF1000F06D049
:10291000A15D38460226FFF7F9FEB5420CD9A15D4C
:1029200001363846FFF7F2FEA15D38460136FFF763
:10293000EDFEB0B28542F2D800204146FFF7E6FE38
:102940000020494602B0BDE8F047FFF7DFBE00BFF8
:1029500040F67803C2F200030146D8780FF074BF46
:10296000F0B540F6B053C2F2000340F6681793F892
:1029700006C08CF0950686EA0614E6B23209C2F269
:10298000000782F02C0197F800E07F7841EA0625E5
:1029900085EAC60181EA0E0484EA0412D2B20D0A65
:1029A00085EA121686EA022484EAC2018CB284EA1D
:1029B000070585EA0516220AF5B282EA151141EAF1
:1029C000052686EAC5052E2685EA060484EA041251
:1029D000D2B2290A81EA121484EA022585EAC201E8
:1029E00089B281EA000484EA04150246EDB2080ABD
:1029F00080EA151444EA052181EAC50585EA12201A
:102A000080EA0014E4B2290A81EA141080EA04255D
:102A100085EAC4018CB284F00B0085B080EA001511
:102A2000EDB2210A81EA15108DF806C00CF1010CF7
:102A300083F806C040EA0524FE210020ADF80C20F2
:102A400002228DF805208DF807E08DF808708DF8CA
:102A50000960FFF75BFE9DF805100020FFF756FEAA
:102A60009DF806100020FFF751FE9DF8071000208A
:102A7000FFF74CFE9DF808100020FFF747FE9DF879
:102A800009100020FFF742FE9DF80C100020FFF710
:102A90003DFE84EAC5049DF80D100020FFF736FEC8
:102AA000E1B20020FFF732FE210A002005B0BDE8A8
:102AB000F040FFF72BBE00BFF0B540F6B053C2F2B6
:102AC000000340F6681793F806C08CF0950686EA76
:102AD0000614E6B23209C2F2000782F02C0197F820
:102AE00000E07F7841EA062585EAC60181EA0E0406
:102AF00084EA0412D2B20D0A85EA121686EA02248A
:102B000084EAC2018CB284EA070585EA0516220A26
:102B1000F5B282EA151141EA052686EAC5052A269C
:102B200085EA060484EA0412D2B2290A81EA121460
:102B300084EA022585EAC20189B281EA000484EAB6
:102B400004150246EDB2080A80EA151444EA05218C
:102B500081EAC50585EA122080EA0014E4B2290A58
:102B600081EA141080EA042585EAC4018CB284F05D
:102B70001C0085B080EA0015EDB2210A81EA15102B
:102B80008DF806C00CF1010C83F806C040EA05245C
:102B9000FE210020ADF80C2002228DF805208DF8D2
:102BA00007E08DF808708DF80960FFF7AFFD9DF81C
:102BB00005100020FFF7AAFD9DF806100020FFF782
:102BC000A5FD9DF807100020FFF7A0FD9DF8081057
:102BD0000020FFF79BFD9DF809100020FFF796FDF0
:102BE0009DF80C100020FFF791FD84EAC5049DF8C4
:102BF0000D100020FFF78AFDE1B20020FFF786FDEF
:102C0000210A002005B0BDE8F040FFF77FBD00BFFE
:102C10002DE9F04F4FF4406240F61060C4F200021C
:102C2000C2F20000546A03689C42DDB0C0F0E58146
:102C300040F67805C2F2000514F0AAFCA8780CF062
:102C4000D7F841F6942CC1F2000C03269CF8BC3155
:102C500085F8D660402113F0480F85F8D41000F0B5
:102C60008481052385F8D63041F2D81EC1F2000ECA
:102C70009EF838556A1E032A0FD8DFE812F0B30118
:102C8000A80104009D0140F67803C2F2000393F806
:102C9000D40040F0180683F8D46041F6942CC1F2B9
:102CA000000C9CF8BC21930709D540F6780EC2F2BF
:102CB000000E9EF8D41061F07F058EF8D45040F6D7
:102CC0007806C2F20006B36D9C4200F2A381736ED7
:102CD000002B00F0518140F6780EC2F2000EDEF8B3
:102CE0009C108C4200F24484002B00F0498140F695
:102CF000780CC2F2000CDCF8B000844201F20682CB
:102D0000002B00F0468140F67805C2F20005D5F8A8
:102D1000A400844201F23384002B00F0438140F68A
:102D20007805C2F20005D5F8A8108C4200F20A8797
:102D300040F6780EC2F2000E5BA903319EF8030044
:102D40000FF056FD9DF86F310146002B40F0DD80FD
:102D50008DF834300DF135003222002901F0E18781
:102D60001AF0B4FD40F6B05CC2F2000C40F66816F2
:102D70009CF8060080F09F0383EA0315EBB21F095D
:102D8000C2F2000687F00C0141EA03223778767818
:102D90008DF8620182EAC30585EA070E8EEA0E18F5
:102DA0005FFA88F3290A81EA131A8AEA032989EA71
:102DB000C30295B285EA060E8EEA0E185FFA88F312
:102DC000290A81EA131545EA032A8AEAC303FD2585
:102DD00083EA050989EA09125FFA82FE190A81EA83
:102DE0001E1282EA0E28FE2333210DF13409013030
:102DF00088EACE0A8DF860318DF864618DF8611132
:102E00008DF863718DF865518CF806001FFA8AF20F
:102E100009EB01064B469946170A19F8010B93F87E
:102E2000018099F8019080EA020C8CEA0C1E5FFA8E
:102E30008EF187EA111545EA012787EAC10088EA81
:102E4000000A8AEA0A12D2B2050A85EA121747EA8C
:102E5000022181EAC20789EA070080EA0015E8B288
:102E6000390A81EA101C03334CEA0022B34282EA99
:102E7000C002D0D182F0530686EA0610C1B2170A0A
:102E800087EA111585EA012282EAC1030020FE21AA
:102E90009EB2FFF73BFC9DF861110020FFF736FC66
:102EA0009DF862110020FFF731FC9DF863110020AE
:102EB000FFF72CFC9DF864110020FFF727FC9DF81C
:102EC00065110020FFF722FC5FFA86FA4FEA162907
:102ED0000DF133050DF16608002669783046FFF7DD
:102EE00015FCA9783046FFF711FC6F1C15F8031F7D
:102EF0003046FFF70BFC4545EFD100205146FFF768
:102F000005FC00204946FFF701FC40F67803C2F2B9
:102F100000031A6ED3F8CC00824203D2DB6D9C42D0
:102F200001F2228240F67805C2F2000595F8DA1027
:102F300095F8D930994204D2D5F8DC20944201F2B8
:102F40000E86994201F0118014F02AFB40F67801B8
:102F5000C2F2000188780BF0C5FF40F61063C2F2A0
:102F600000031C605DB0BDE8F08F5A077FF57CAEB2
:102F7000042085F8D60077E6B26E002A7FF4ABAE67
:102F800040F6780EC2F2000EDEF87C1000297FF4C5
:102F9000AEAE40F6780EC2F2000EDEF87020002AC7
:102FA0007FF4B1AE40F6780EC2F2000EDEF8740087
:102FB00000283FF4BDAEB2E640F6780EC2F2000E35
:102FC0009EF8D41041F014058EF8D45065E640F612
:102FD000780CC2F2000C9CF8D42042F011008CF85E
:102FE000D4005AE640F67806C2F2000696F8D430CD
:102FF00043F0100186F8D4104FE640F67805C2F28F
:103000000005002105F19800A965E96534221AF050
:103010007BFC0DE640F6B058C2F2000840F6681797
:1030200098F8063096F8D55096F8D410559583F058
:10303000460B8BEA0B1C5FFA8CF2C2F200071009F8
:1030400080F0920E97F8009097F801B0CDF80C90B0
:103050004EEA022080EAC20E8EEA090282EA0219D2
:103060005FFA89F94FEA1E2080EA191282EA0920E4
:1030700080EAC90290B280EA0B09CDF810B089EA63
:10308000091B5FFA8BF24FEA102E8EEA121040EA0B
:10309000022989EAC20E8EEA0E1B5FFA8BF24FEA12
:1030A0001E2080EA121080EA022080EAC2091FFA7C
:1030B00089F0454085EA051B5FFA8BF94FEA102E2F
:1030C0008EEA191242EA092585EAC90080EA001B46
:1030D0005FFA8BFE050A85EA1E1242EA0E2080EA9C
:1030E000CE0585EA05195FFA89FB280A80EA1B12DA
:1030F00042EA0B2E8EEACB0585EA05195FFA89FBB9
:10310000280A80EA1B1297F802C08DF85A1142EA89
:103110000B2585EACB0080EA0C0E8EEA0E195FFAC9
:1031200089FB050A85EA1B1080EA0B2282EACB0E96
:103130001FFA8EF04FF0050E80EA0E0989EA091594
:10314000EDB2020A82EA151040EA052B8BEAC505AA
:1031500085EA010989EA0912D2B2280A80EA121521
:1031600085EA022196F8D6A08DF859E181EAC20BD2
:103170001FFA8BF585EA0A0989EA09105FFA80FBD4
:10318000290A81EA1B1242EA0B2080EACB094FF0A0
:10319000030B89EA0B0585EA0511CDB24FEA192028
:1031A00080EA151282EA052181EAC50085B285F020
:1031B000320282EA02195FFA89F24FEA1521581C9D
:1031C00081EA1211059041EA0229DDF814E08DF838
:1031D0005CB189EAC20909220025DDF810B08DF83A
:1031E0006121039A88F806E02846FE218DF85BA14C
:1031F0006FF0010A8DF858C18DF862318DF86321A6
:103200008DF860A18DF864B18DF86551FFF77EFAF5
:1032100028469DF86111FFF779FA28469DF862115A
:10322000FFF774FA28469DF86311FFF76FFA2846F6
:103230009DF86411FFF76AFA28469DF86511FFF7BB
:1032400065FA28469DF85411FFF760FA28469DF864
:103250005511FFF75BFA28469DF85611FFF756FA0D
:1032600028469DF85711FFF751FA28469DF8581146
:10327000FFF74CFA28469DF85911FFF747FA284600
:103280009DF85A11FFF742FA28469DF85B11FFF7A7
:103290003DFA28469DF85C11FFF738FA5FFA89F18C
:1032A0002846FFF733FA4FEA19212846FFF72EFA8E
:1032B00042F2A03CC2F2000CDFEDA87ADCF800106C
:1032C00098F8062097F801E097F800C0B6F8D0709B
:1032D000D6F8E0B0049700EE101AF8EE406A82F0DB
:1032E000F10326EEA77A83EA031AC7EE275A5FFA9C
:1032F0008AF341F6D0601909C2F2000040F2746707
:10330000C2F2000781F0E7090068D7F800A0C6F80C
:10331000E00049EA032181EAC30140F22013CBEB2C
:103320000009C1F2000393ED432A0AFB09F304EEFE
:10333000903A81EA0C07DFED8C1AF8EE643A87EADE
:10334000071B9FED874A5FFA8BFA0B0A63EEA12AEF
:1033500083EA1A1732EE445A9FED823A87EA0A212D
:1033600082EEA51A81EACA039FB287EA0E0989EAAA
:10337000091B5FFA8BF3390A81EA131747EA032A1C
:103380008AEAC30B01278BEA070989EA09115FFA68
:1033900081FA85EE036A4FEA1B2383EA1A1181EA58
:1033A0000A2383EACA011FFA81F940F61861C2F2C2
:1033B000000189EA0913DBB208604FEA192B8BEA96
:1033C000131949EA0329FCEEC16A62EE210A26EECE
:1033D000210ABCEEE07A16EE90AAFDEEC07A16EE57
:1033E000901ACAF57A7B17EE100AA6F8D210ADF83B
:1033F00098B00499ADF89A004FF6FF7617EE90BAA0
:1034000002EB070AADF89C606FF001001F262395C0
:1034100024952595ADF89E50ADF8A010ADF8A250BA
:10342000ADF8A450ADF8A650ADF8A8508DF86221C3
:10343000CDED036A8DED057ACDED067A8DF8AAB053
:103440008DF860018DF861610DF1AB058DF863C1F8
:103450000DF18D028DF864E18DF8657188F806A094
:1034600089EAC30110460E0A10F8017B92F8018028
:10347000794081EA011C5FFA8CF386EA131E4EEA5A
:10348000032989EAC30288EA020787EA0716110AB4
:10349000F7B281EA1713421C43EA0726AA4286EADA
:1034A000C701DFD181F07C0585EA0517FAB2090A68
:1034B00081EA121686EA022383EAC20085B2FE215F
:1034C0000020FFF723F99DF861110020FFF71EF996
:1034D0009DF862110020FFF719F99DF86311002093
:1034E000FFF714F95FFA85F99DF8641100204FEA9F
:1034F00015285CADFFF70AF900269DF8651100203C
:10350000FFF704F915F8E41D30460DF1AA07FFF79F
:10351000FDF869783046FFF7F9F8A97830460235AA
:10352000FFF7F4F8BD42F4D100204946FFF7EEF86A
:1035300000204146FFF7EAF802EE104ADFED071AD5
:10354000B8EE426A40F6780C36EE211AC2F2000C50
:10355000FCEEC10ACCED160AFFF7EABB0024744961
:10356000CDCC1C419A99494100007A440AD7233CAA
:1035700040F6B052C2F2000240F6681591793994D3
:1035800081F0300787EA0713D8B20609C2F20005B6
:1035900086F07A0E4EEA002B2E786D788DF8621147
:1035A0008BEAC00787EA060A8AEA0A195FFA89F8ED
:1035B000380A80EA181787EA082383EAC80087B226
:1035C00087EA050C40F22013C1F200038CEA0C1EBE
:1035D0005FFA8EF04FEA1727D3F838A1D3F83C9161
:1035E000D3F84081D3F82CC1D3F830E187EA101B1F
:1035F000D3F834710597D3F844710397D3F8487121
:103600000497D3F84C318DF863615FED297A4BEA6A
:10361000002704EE90AADDED036A87EAC0079DED5E
:10362000047A1A269DED050A64EEA73A04EE109A74
:1036300000EE908A05EE10CA05EE90EA87EA060CC5
:1036400003EE103A66EEA76A8CEA0C1E20EE270AFB
:1036500027EE277A5FFA8EF324EE272A25EE271A23
:103660004FEA1720FDEEE32A60EEA71A23EE273A71
:1036700065EEA70ABDEEE65A80EA131BFDEEC75AB7
:10368000FDEEC03A12EE90AA15EE100AFDEEC32A26
:103690008BEA032BBDEEC26AFDEEE17AFDEEC14A74
:1036A000BDEEE04A13EE907A8BEAC30B15EE903A2A
:1036B000ADF8F40016EE109A17EE908A14EE90CA48
:1036C00014EE10EA12EE900A0131ADF8F270ADF886
:1036D000F630FE271623CDED035ACDED042AADF8C2
:1036E000E8A0ADF8EA90ADF8EC80ADF8EEC0ADF82A
:1036F000F0E0ADF8F8008DF860718DF861319171EE
:103700008DF864518DF865611FFA8BF10DF1FA05A2
:1037100039AA10460E0A10F8013B92F801C083EA5C
:10372000010989EA09175FFA87F886EA181343EA5C
:10373000082282EAC8078CEA070686EA0611CEB29A
:103740003B0A83EA161242EA0621421CAA4281EA97
:10375000C601DED1CDB285F0AA0383EA03175FFA72
:1037600087FA0E0A86EA1A1282EA0A2181EACA0058
:1037700085B2FE210020FEF7C9FF9DF861110020EF
:10378000FEF7C4FF9DF862110020FEF7BFFF9DF811
:1037900063110020FEF7BAFF9DF864110020FEF7C8
:1037A000B5FF9DF865110020FEF7B0FF5FFA85F9BF
:1037B0004FEA15280DF1E40B0DF1E3050DF1F907C2
:1037C000002669783046FEF7A1FFA9783046023519
:1037D000FEF79CFFBD42F4D100204946FEF796FF5C
:1037E00000204146FEF792FF40F6B053C2F20003BC
:1037F00040F6681C93F80680519488F0F90585EA34
:103800000512D6B23009C2F2000C80F0E60141EA9E
:10381000062A9CF800009CF801E08DF863018AEA12
:10382000C60585EA000989EA09175FFA87FC290AB3
:1038300081EA1C1686EA0C2282EACC0A1FFA8AF177
:1038400081EA0E0787EA07155FFA85F90E0A86EA0C
:10385000191242EA092787EAC9051D2785EA070CDC
:103860008CEA0C1A5FFA8AF9290A81EA191686EAA3
:10387000092282EAC90C1FFA8CF181EA040A8AEA59
:103880000A155FFA85F90E0A86EA191242EA092535
:1038900085EAC90585EA142181EA0116F6B22A0AE9
:1038A00082EA161141EA062C8CEAC60585EA144A1A
:1038B0008AEA0A195FFA89F12A0A82EA111640F2A5
:1038C0002012C1F20002D2ED477A5FEDD83A46EA03
:1038D000012585EAC10967EEA32A89EA146C8CEAFE
:1038E0000C1ACDED522A5FFA8AF14FEA192686EAC0
:1038F000111545EA012A9DF848919DF849C19DF8A6
:103900004A619DF84B518DF862818AEAC10080EAD4
:10391000090181EA0111C9B2000A80EA111040EAE6
:10392000012080EAC10080EA0C0181EA011C5FFAF3
:103930008CFC000A80EA1C1141EA0C2080EACC00D1
:1039400080EA060181EA011C5FFA8CF1060A86EA28
:10395000111040EA012686EAC10080EA050C8CEAD3
:103960000C15E9B2060A86EA111040EA012585EA3B
:10397000C10686EA061C5FFA8CF1300A80EA11154E
:1039800045EA012686EAC10080EA001C5FFA8CF154
:10399000050A85EA111646EA012080EAC10585EA92
:1039A000051C5FFA8CF12E0A92ED422A9FED636AA4
:1039B00086EA111040EA012C62EE061A8CEAC10672
:1039C00086EA0615BDEEE11AE9B2320A82EA111062
:1039D00040EA012511EE102A85EAC10080EA020CB6
:1039E0008CEA0C16F6B2050A85EA161181EA062061
:1039F00080EAC605A8B280EA122181EA011C5FFABA
:103A00008CF1060A86EA111545EA012080EAC10513
:103A100085F0730686EA061C5FFA8CF6290A81EAAD
:103A200016104FF0FE0C40EA062508F10108614629
:103A300083F80680002085EAC605ADF850210026EF
:103A40000E228DF860C18DF861218DF864E15396E6
:103A50008DF86571FEF75AFE00209DF86111FEF7A2
:103A600055FE00209DF86211FEF750FE9DF863118F
:103A70000020FEF74BFE00209DF86411FEF746FE85
:103A800000209DF86511FEF741FE00209DF84411CD
:103A9000FEF73CFE00209DF84511FEF737FE0020A2
:103AA0009DF84611FEF732FE00209DF84711FEF703
:103AB0002DFE00209DF84811FEF728FE00209DF8FD
:103AC0004911FEF723FE00209DF84A11FEF71EFE65
:103AD00000209DF84B11FEF719FE00209DF84C11B7
:103AE000FEF714FE00209DF84D11FEF70FFE00209A
:103AF0009DF84E11FEF70AFE00209DF84F11FEF7CB
:103B000005FE00209DF85011FEF700FE00209DF8F4
:103B10005111FEF7FBFDE9B20020FEF7F7FD290A7F
:103B20000020FEF7F3FD40F6780CC2F2000CDCF842
:103B300068100819CCF89C00FFF7FAB80000C842DA
:103B400035FA8E3C40F6B05AC2F2000A40F66811CF
:103B50009AF806002B9480F06A0585EA0513DAB21C
:103B60001709C2F2000187F0D50686EAC2080F786D
:103B700049788DF8620188EA022686EA070B8BEA0B
:103B80000B15EDB2320A82EA151E8EEAC50383EAEE
:103B90000526B2B282EA010C41F6287E40F22018D6
:103BA000C1F200088CEA0C19C2F2000E5FFA89F625
:103BB000130AD8F82CB1D8F830C1D8F834218DF8D0
:103BC000637183EA1615DEF83C348DF8641185EADA
:103BD000C60585EA062601EE102A1E2703EE10BA56
:103BE000D3ED096A01EE90CA93ED0A7AD3ED0B4A40
:103BF00086EA07050EF580680EF581695FED302ACB
:103C000085EA0513D8ED030A71EEC73A31EE644A2E
:103C100099ED000A98ED016A73EE667A5FFA83FB0C
:103C2000320A82EA1B1620EEA25A60EE225A26EED3
:103C3000222A67EEE21A23EEA21A64EE220A86EA2C
:103C40000B2585EACB06FE231C2201308DED2C5A74
:103C5000CDED2D5A8DED2E2ACDED2F1A8DED301A8A
:103C6000CDED310A8DF860318DF861218DF86571E7
:103C70008AF80600B2B232AD2BAB1946160A11F81B
:103C8000010B93F8019080EA020B8BEA0B12D7B27A
:103C900086EA171E4EEA072C8CEAC70789EA070056
:103CA00080EA00135FFA83FA3E0A86EA1A124B1C76
:103CB00042EA0A20AB4280EACA02DED182F027053E
:103CC00085EA0510160A5FFA80F886EA181787EA6F
:103CD000082383EAC8018DB20020FE21FEF716FDFD
:103CE0009DF861110020FEF711FD9DF86211002082
:103CF000FEF70CFD9DF863110020FEF707FD9DF80F
:103D000064110020FEF702FD9DF865110020FEF70A
:103D1000FDFC5FFA85F94FEA15280DF1C7070DF193
:103D2000AB05002669783046FEF7F0FCA9783046EE
:103D30000235FEF7EBFCBD42F4D149460020FEF708
:103D4000E5FC41460020FEF7E1FC40F6B052C2F22D
:103D5000000240F6681690794B9480F0AB0585EA36
:103D60000513D9B20F09C2F2000687F0480989EAA3
:103D7000C108377876788DF8620188EA012585EAEE
:103D8000070C8CEA0C1B5FFA8BF9290A81EA191AD5
:103D90008AEAC90383EA09281FFA88F181EA060C36
:103DA0008CEA0C155FFA85FB0B0A83EA1B1585EA82
:103DB000CB0141F22013C1F2000381EA0B29242533
:103DC00089EA050AB3F842E0B3F846C0B3F83CB05C
:103DD000CDF814E08AEA0A11C9B24FEA192888EA34
:103DE000111AB3F83E90B3F84080B3F844E0CDF830
:103DF0000CC0B3F848C0B3F84A30ADF830B18AEA25
:103E0000012B8BEAC10BADF83291FE21DDF8149045
:103E1000DDF80CA0ADF83E31002301308DF84031C3
:103E20008DF86011152350A98DF861318DF8655119
:103E30009071ADF83481ADF83691ADF838E1ADF858
:103E40003AA1ADF83CC18DF863718DF864611FFA39
:103E50008BF24D1C4BAB9A46170A1AF8010B93F8DC
:103E600001909AF801B080EA020686EA06115FFA2C
:103E700081FE87EA1E1242EA0E2080EACE0789EA16
:103E8000070888EA08165FFA86FC390A81EA1C12DC
:103E900042EA0C2080EACC078BEA070A8AEA0A1673
:103EA000F2B2390A81EA121E03334EEA0220AB4213
:103EB00080EAC202CFD15FFA82F888F0DE0C8CEA89
:103EC0000C1B5FFA8BF7100A80EA171686EA0721A7
:103ED00081EAC7020020FE2195B2FEF717FC9DF88B
:103EE00061110020FEF712FC9DF862110020FEF720
:103EF0000DFC9DF863110020FEF708FC9DF864118D
:103F00000020FEF703FC9DF865110020FEF7FEFB84
:103F10004AAB5FFA85FA4FEA15290DF5967BDD1C51
:103F20000DF5A078002669783046FEF7EFFBA978FA
:103F30003046FEF7EBFB6F1C15F8031F3046FEF70B
:103F4000E5FB4545EFD100205146FEF7DFFB0020A1
:103F50004946FEF7DBFB40F67803C2F200035A6FD6
:103F60001519C3F8A850FEF7E3BE40F6B053C2F2ED
:103F7000000340F6681C93F806A08AF01C0686EA47
:103F80000612D7B23809C2F2000C80F03D0141EAB6
:103F900007299CF800009CF801C08DF86B0189EAA4
:103FA000C70686EA000E8EEA0E155FFA85F8310A1A
:103FB00081EA181787EA082282EAC8091FFA89F1FC
:103FC00081EA0C0585EA05165FFA86FE0F0A87EA84
:103FD0001E1242EA0E2585EACE064FF02F0E86EA23
:103FE0000E0888EA08195FFA89F2310A40F6780665
:103FF000C2F2000681EA121787EA022585EAC208A2
:1040000096F8D79096F8D8708DF86AA11FFA88F0C4
:1040100089EA000181EA0115EDB2020A82EA15116E
:1040200041EA052080EAC50181EA070282EA021816
:104030005FFA88F20D0A85EA121080EA022181EA0D
:10404000C2081FFA88F080EA0015EDB2010A81EA81
:10405000151242EA052080EAC505E9B281F099020D
:1040600082EA02185FFA88F24FEA152080EA1211FC
:10407000002541EA02280AF1010A83F806A088EA2D
:10408000C20828460322FE218DF869218DF86CC1F3
:104090008DF86DE18DF861718DF86251FEF736FB98
:1040A0009DF869112846FEF731FB9DF86A112846F4
:1040B000FEF72CFB9DF86B112846FEF727FB9DF8B9
:1040C0006C112846FEF722FB9DF86D112846FEF77D
:1040D0001DFB28464946FEF719FB28463946FEF7E0
:1040E00015FB28462946FEF711FB5FFA88F12846A2
:1040F000FEF70CFB4FEA18212846FEF707FB96F85F
:10410000DA20531C86F8DA30FEF71EBF41F2600554
:10411000C1F2000591A3D3E90023D5E90E0117F000
:10412000BDFC17F0BBFA41F2D816C1F200068BA312
:10413000D3E9002396F83B750646D5E9100117F040
:10414000ADFC17F0ABFA40F6B052C2F2000240F6F6
:10415000681392F806E01D908EF0780181EA011153
:10416000C9B2C2F200034FEA111C8CF0F60C93F8AE
:10417000018093F800901C964CEA012383EAC10168
:1041800081EA090383EA0313DBB2090A81EA131106
:1041900081EA032181EAC30399B281EA080383EA31
:1041A0000313DBB2090A81EA131141EA0321D5EDB9
:1041B000125A4FF0180C81EAC303DFED677A95EDD0
:1041C0001D6A83EA0C01D5ED1E6A95ED187A65EE3D
:1041D000A75A81EA0111D5ED197AC9B21B0ABCEEC2
:1041E000C66A83EA1115FCEEE66ABCEEC77AFCEEFD
:1041F000E77A1AAB85EA01254FF0000B16EE100A9C
:1042000085EAC101CDF86CB01D4616EE906AFE231A
:10421000FDEEE55A17EE10AA17EE90BA8DF862E19E
:10422000ADF87C008DF860310EF1010E1E23FF20E9
:10423000ADF87E608DF861318DED036ACDED046AD5
:104240008DED057ACDED067A1A94CDED1E5AADF8B6
:1042500080A0ADF882B08DF884708DF885000DF1E6
:1042600086068DF863912B4682F806E08DF864810E
:104270008DF865C18AB2194693F8019011F8010BC7
:1042800080EA0203170A83EA0312D0B287EA101CFD
:104290004CEA002E8EEAC00389EA030888EA081770
:1042A000FFB2180A80EA171343EA07224B1CB342F5
:1042B00082EAC702DFD182F0180686EA0610130AE6
:1042C0005FFA80F983EA191282EA092787EAC901AD
:1042D0008EB20020FE21FEF719FA9DF86111002030
:1042E000FEF714FA9DF862110020FEF70FFA9DF810
:1042F00063110020FEF70AFA9DF864110020FEF712
:1043000005FA9DF865110020FEF700FA5FFA86F9BC
:104310004FEA16281D350DF16706002771783846DB
:10432000FEF7F4F9B17838460236FEF7EFF9AE42FF
:10433000F4D100204946FEF7E9F941460020FEF796
:10434000E5F940F6780CC2F2000CDCF87C100D198F
:10435000CCF8B050FEF7ECBC00007A44000000003E
:10436000D012634100409C4640F2B42940F2000E56
:10437000C1F2000909EB820CC2F2000EDCF80080E9
:104380005EF82210ADF8CE200922ADF8CC008DF8F1
:10439000E020CDF8C88034A81022002900F0C584A0
:1043A00019F094FA40F6B053C2F2000340F66816D2
:1043B000987980F0C70E8EEA0E15E9B20A09C2F2AA
:1043C000000682F0820796F800E076788DF86201A8
:1043D00047EA012C8CEAC10585EA0E0888EA08192B
:1043E0005FFA89F22F0A87EA121181EA022585EA2B
:1043F000C20C1FFA8CF787EA060888EA08195FFAE8
:1044000089F2390A81EA121545EA022787EAC201D0
:10441000162581EA050C8CEA0C185FFA88F20F0A5F
:1044200087EA12115CAF81EA022989EAC20C17F807
:10443000A88D8DF863E11FFA8CF288EA020181EA07
:1044400001195FFA89F1120A82EA111C01304CEA63
:1044500001224FF0FE0E4FF019088DF8655198714A
:104460008DF860E18DF861818DF864610DF1E105F1
:104470000DF1C90382EAC102194693F8019011F8BF
:10448000010B80EA0203160A83EA03125FFA82F83C
:1044900086EA181E4EEA082C8CEAC80389EA030053
:1044A00080EA0016F6B21A0A82EA161343EA0620D8
:1044B0004B1CAB4280EAC602DED1D1B281F0DC05F2
:1044C00085EA0510130A5FFA80F983EA191282EA75
:1044D000092686EAC9018DB20020FE21FEF716F9F1
:1044E0009DF861110020FEF711F99DF8621100207E
:1044F000FEF70CF99DF863110020FEF707F95FFA4B
:1045000085F99DF8641100204FEA15285CADFEF78F
:10451000FDF800269DF865110020FEF7F7F815F864
:10452000A81D30461837FEF7F1F869783046FEF7D7
:10453000EDF8A97830460235FEF7E8F8BD42F4D12F
:1045400000204946FEF7E2F800204146FEF7DEF87B
:1045500004EE104A40F6780CF8EE442A1FED7F5A1C
:10456000C2F2000C72EE855ADCF86000BCEEE52A5F
:10457000431CCCF860308CED172AFEF7E5BC40F602
:10458000B053C2F2000340F2B42099793F94C1F2D3
:10459000000081F0300E8EEA0E12D0ED061AD7B26E
:1045A000D0ED080A3D09BDEEE14A85F07A06D0ED6E
:1045B000037A46EA072614EE10CAFDEEE05A86EAB0
:1045C000C70641F63807C1F2000790ED027AD0ED38
:1045D000042A90ED056A90ED071A90ED090AFDEEA8
:1045E000E73A15EE900A0CF1040C043037F81CC0C1
:1045F000039013EE90AAFDEEC06A40F66812C2F274
:104600000002BDEEC73AADF814C0BDEEE22ADDF8F7
:104610000CC0157837F81CC08DF86211FDEEC64A43
:10462000BDEEC15A0AF1040A16EE900A37F81AA034
:10463000ADF80CC013EE10BA043012EE109A14EE5E
:10464000908A15EE10EA049097ED0F7A86EA05003D
:10465000DDF810C00AF5806A0BF1040B09F10409BA
:1046600008F104080EF1040ECDF820A080EA001035
:10467000BDF80CA037F81CC037F81BB037F81990FC
:1046800037F8188037F81EE0ADF818C0C0B2370A06
:10469000BCEEC73A87EA10160AF580670796BDF8A0
:1046A00014C08DED043A0397BDF81860DDF81CA026
:1046B0008DF8635106F58067ADF80E7100270BF594
:1046C000806B8DF8107113EE107AADF800B1DDF843
:1046D0000CB08DF811718AEA002608F58068FE2773
:1046E000DDF820A0ADF80681ADF80CB186EAC0086F
:1046F00092F801B08DF8607116278DF861711FFA7C
:1047000088F70EF5806EADF802A187EA0B0AADF8C6
:104710000AE18AEA0A1E5FFA8EF53E0A86EA151059
:1047200040EA052787EAC505232085EA00020CF543
:10473000806CADF808C182EA021C5FFA8CFA09F5B8
:1047400080692E0AADF8049186EA1A1989EA0A28C6
:10475000013188EACA0799718DF864B18DF8650155
:10476000BAB20DF589753FAB1946100A11F8016B05
:1047700093F8019086EA020E8EEA0E12D7B280EA12
:10478000171B4BEA072A8AEAC70689EA060888EA5D
:10479000081C5FFA8CF7300A80EA171343EA0726F1
:1047A0004B1CAB4286EAC702DED1D5B285F0F401DC
:1047B00081EA0116120AF7B282EA171C8CEA072076
:1047C00080EAC703FE2100209DB2FDF79FFF9DF800
:1047D00061110020FDF79AFF9DF862110020FDF79E
:1047E00095FF9DF863110020FDF790FF9DF864117F
:1047F0000020FDF78BFF9DF865110020FDF786FF77
:104800003FA95FFA85F94FEA152801F115070DF167
:10481000FB05002669783046FDF778FFA978304619
:104820000235FDF773FFBD42F4D149460020FDF784
:104830006DFF41460020FDF769FF40F6B052C2F21D
:10484000000240F2B42190794594C1F2000180F059
:10485000300791ED020A87EA071391ED037AD1ED53
:10486000047AD1ED052A91ED066A91ED072AD1ED82
:10487000081A91ED091A40F66811DDB2C2F2000182
:104880004FEA151991F800B08DF86201FDEEE73A94
:10489000FDEEC15A89F07A09FDEEC06A49EA0529A0
:1048A000BDEEC73ACDF810B013EE90CA89EAC50B39
:1048B00015EE909A16EE906A13EE108AFDEEE24A1B
:1048C000BDEEC64ABDEEC25AFDEEE10ACDF80CB00F
:1048D00041F638030CF1040B09F1040CC1F200039A
:1048E000CDF814C0DDF81090DDF80CC006F1040A14
:1048F00008F1040814EE90EA14EE107A15EE106A2E
:1049000010EE905A33F81AA08CEA090C0EF1040E3E
:1049100033F8189033F81B80DDF814B0CDF818C0C8
:104920000437043605F1040533F81EC033F817E0E8
:1049300033F8167033F8156033F81B50DDF818B0F3
:1049400093ED0F0A0AEB4A030AEB830A039B1B0A47
:10495000029309EB4903039308EB480305930CEB1F
:104960004C0306930EEB4E030793AAF5185A07EB78
:1049700047030893AAF1160A06EB46030993CDF8FC
:1049800004A005EB4503DDF80CA00A938BEA0B1B92
:10499000029B5FFA8BFB09EB8A09DDF818A0ADF8E2
:1049A0001A9183EA1B1302930CEB8A0C059BDDF82A
:1049B00020A0DDF81090ADF81EC108EB830807EBCE
:1049C0008A07079BDDF828A0ADF82271FCEEC06ACB
:1049D0000EEB830E05EB8A05099BDDF808A0ADF808
:1049E000265116EE905A06EB830600278AEA0B231F
:1049F0008DF828718DF82951162783EACB058DF89B
:104A0000639191F80190ADF824618DF86171FE26F3
:104A1000AFB28DF8606187EA090686EA0611CEB268
:104A20003B0A83EA1615ADF820E145EA062E8EEA28
:104A3000C6072225ADF81C8187EA050888EA081C0C
:104A40005FFA8CFE390A81EA1E16DDF804A08DF8A3
:104A5000649186EA0E2383EACE08471CCDED0B6AEB
:104A6000ADF818A145AB8DF8655197710DF59575A9
:104A70001FFA88F2194693F8018011F8010B80EAB9
:104A8000020787EA0713D8B2160A86EA101242EA2A
:104A9000002989EAC00788EA070C8CEA0C1E5FFA35
:104AA0008EF23B0A83EA12164B1C46EA0220AB4206
:104AB00080EAC202DED1D6B286F0ED0585EA0511A4
:104AC0005FFA81FE100A80EA1E1787EA0E2383EA46
:104AD000CE06B2B20020FE215FFA82F94FEA122818
:104AE000FDF714FE9DF861110020FDF70FFE9DF803
:104AF00062110020FDF70AFE9DF863110020FDF70A
:104B000005FE9DF864110020FDF700FE9DF865117B
:104B10000020FDF7FBFD44AD45A9033501F1150764
:104B2000002669783046FDF7F1FDA9783046023558
:104B3000FDF7ECFDBD42F4D100204946FDF7E6FD4E
:104B400000204146FDF7E2FD40F6780CC2F2000C71
:104B5000DCF870301A19CCF8A420FEF7E9B840F65A
:104B6000B053C2F2000340F6681C9A79ADF86811A0
:104B700082F0A30E8EEA0E185FFA88F74FEA17103C
:104B8000C2F2000C80F049069CF800809CF801C03D
:104B900095F8D7A095F8D8908DF86AA146EA072035
:104BA00080EAC70787EA080E8EEA0E16F6B23F0AB9
:104BB00087EA161080EA062787EAC60087B287EAE6
:104BC0000C0E8EEA0E16F6B2380A80EA161747EA7D
:104BD000062E8EEAC6074FF0280E87EA0E0080EAFE
:104BE0000016F6B23F0A87EA161080EA062787EA1F
:104BF000C60080B280EA010787EA0716F6B2010A0A
:104C000081EA161747EA062080EAC60787EA0711F5
:104C1000C9B23E0A86EA111040EA012787EAC100BC
:104C200080EA0A0686EA061A5FFA8AF6070A87EA1F
:104C3000161181EA062080EAC607BEB286EA09019B
:104C400081EA011A5FFA8AF1300A80EA111747EA0D
:104C5000012686EAC106F0B280F0E60787EA071A65
:104C60005FFA8AF7310A81EA171002F1010A40EA75
:104C7000072683F806A00020FE2186EAC70604273F
:104C80008DF862218DF864C18DF865E18DF86B9126
:104C90008DF861718DF86381FDF738FD00209DF876
:104CA0006111FDF733FD00209DF86211FDF72EFD27
:104CB00000209DF86311FDF729FD00209DF8641187
:104CC000FDF724FD00209DF86511FDF71FFD002074
:104CD0009DF86811FDF71AFD00209DF86911FDF798
:104CE00015FD00209DF86A11FDF710FD00209DF8CC
:104CF0006B11FDF70BFDF1B20020FDF707FD310A46
:104D00000020FDF703FD00EE904A9FED0A6AB8EE21
:104D1000600A70EE067AFCEEE73AC5ED373AFEF728
:104D200013B918F0F1FDFEF71DB818F0EDFDFFF70F
:104D300039BB00BF002474492DE9F041858C042D56
:104D400084B000F0F080F52D00F0BF80042440F620
:104D5000B053C2F2000340F6681E9A79ADF80C50C9
:104D600082F01C0888EA081C5FFA8CF00709C2F27E
:104D7000000E87F03D069EF800C09EF801E08DF819
:104D8000062046EA002181EAC00686EA0C0888EA85
:104D90000817FFB2300A80EA171686EA072181EA6F
:104DA000C70087B287EA0E0686EA0611CEB2380A35
:104DB00080EA161848EA062787EAC6004D2780EAE7
:104DC000070181EA0116F6B2000A80EA161888EA9D
:104DD000062181EAC60086B286EA050181EA011849
:104DE0005FFA88F1300A80EA111646EA012080EA6B
:104DF000C10080EA152888EA0816F6B2010A81EA9D
:104E0000161545EA062080EAC60585EA040181EA0E
:104E100001185FFA88F1280A80EA111646EA01258E
:104E200085EAC105E8B280F08F0686EA06185FFAC7
:104E300088F6290A81EA161002F1010840EA0625DF
:104E400083F8068085EAC6050020FE2103268DF83A
:104E500007C08DF808E08DF80E408DF805608DF8DC
:104E60000970FDF753FC9DF805100020FDF74EFC7E
:104E70009DF806100020FDF749FC9DF80710002062
:104E8000FDF744FC9DF808100020FDF73FFC9DF85D
:104E900009100020FDF73AFC9DF80C100020FDF7EA
:104EA00035FC9DF80D100020FDF730FC0020214658
:104EB000FDF72CFCE9B20020FDF728FC290A0020B0
:104EC00004B0BDE8F041FDF721BC41F69421C1F2E8
:104ED000000191F8BC3113F0040330D1D0ED027A17
:104EE000F5EE407AF1EE10FA2BD0B7EE007AF4EE40
:104EF000477AF1EE10FA30D0B0EE000AF4EE407AC4
:104F0000F1EE10FA21D0F0EE080AF4EE607AF1EE3C
:104F100010FA7FF41BAF184603F0D2FD0028ACBF97
:104F20000124042413E740F6E054C2F200042046B2
:104F300013F0DEFC2046FDF70BFD012407E70224F9
:104F400005E703F087FC012401E7184603F09EFC07
:104F50000028ACBF01240424F9E603F089FC0124F5
:104F6000F5E600BF2DE9F04F2DED048B40F67803F8
:104F7000F1B0C2F200034FF24C50C0F6010060AF36
:104F80000DF5CC789FEDBE9ADFEDBE8A5D6DFDF725
:104F9000DFFC0397CDF80880052012F001FF41F6F1
:104FA0009424C1F20004284610F0AAFA0028F3D095
:104FB000284610F0B3FA40F6B052C2F200020026C2
:104FC000D1781670C3B209292CD8DFE811F0180186
:104FD0001801F6003001B800D7000A008F005D000C
:104FE0003E0040F67018C2F20008B8F8000088F8D9
:104FF000073083EA000B8BEA0B12D3B2070A87EA69
:10500000131141EA032A98F803608AEAC30940F6BB
:10501000B053A8F80090C2F20003002E40F02681A1
:105020000826DE7040F6B058C2F20008002298F858
:10503000026088F8022040F67803C2F20003B3F859
:10504000D070F619A3F8D060ADE740F67016C2F242
:1050500000063188B3EB112F00F0168140F6B052F4
:10506000C2F20002012092F80280D07008EB000723
:10507000FE2B9770D6D1022100234FF6FF79D17015
:10508000F370A6F80090CDE740F67012C2F200026D
:105090004FF24C4BD1791088C0F6010B1BF801A0E0
:1050A0008AEA000989EA0916F7B2000A80EA1718A5
:1050B00048EA072E8EEAC701CEB21180B34240F60D
:1050C000B051C2F2000100F0D48091F802C001207A
:1050D0000CEB0007FE2BC8708F70A3D102270026AF
:1050E0004FF6FF73CF70D67013809BE740F6B05138
:1050F000C2F2000140F6701E0F79C2F2000E0EEBF4
:10510000070C01378CF80830BEF800009EF803C089
:1051100083EA000B8BEA0B1A5FFA8AF9060A86EA21
:105120001912F8B242EA092383EAC90884450871D2
:10513000AEF800807FF476AF0823CB7072E740F6BC
:10514000701CC2F2000C40F6B05BBCF800208CF87A
:10515000043083EA020989EA09185FFA88F6100A1E
:1051600080EA161E4EEA0627C2F2000B87EAC60145
:105170000323ACF800108BF8033053E740F6701AA5
:10518000C2F2000A40F6B059BAF800208AF8063098
:1051900083EA020E8EEA0E1C5FFA8CF6100A80EA91
:1051A000161B4BEA0627C2F2000987EAC60106234E
:1051B000AAF8001089F8033034E740F6701CC2F2F8
:1051C000000C40F6B05BBCF800208CF8033083EA9A
:1051D000020A8AEA0A195FFA89F7100A80EA1718A0
:1051E000C2F2000B48EA072E8EEAC701002604230C
:1051F0008BF80460ACF800108BF8033012E7FE2B3C
:105200007FF410AF40F6B05A40F67019C2F20009B0
:10521000C2F2000A022200274FF6FF708AF803202C
:1052200089F8037089F80230A9F80000FAE640F620
:10523000701BC2F2000B40F6B05ABBF800208BF88E
:10524000053083EA020888EA081E5FFA8EF6100A23
:1052500080EA161C4CEA0627C2F2000A87EAC60159
:105260000523ABF800108AF80330DBE60721D9707C
:10527000D8E691F804E072440920C8701372D1E6B0
:105280000024744900007A4440F6B057C2F2000787
:105290004FF0010B3A7987F800B006EB020A0AA832
:1052A0008AF8093031464FF4887287F803B018F055
:1052B0000DFB3B78012B41F0968536793A897E715A
:1052C00002B97A8140F6B05CC2F2000C501C002793
:1052D0009CF80260ACF808008CF8027040F6780E7A
:1052E000C2F2000E9EF8020009F082FD9DF82F2008
:1052F000531F472B74D8DFE813F0AC08730073001A
:105300007300730073005204730073007300730022
:105310007300730073007300E80635037300F80729
:1053200073007300730073007300730073007300E5
:1053300073007300730073007300730073005303F2
:105340007F05180373001F0292007701730073003A
:1053500073007300730073007300730073007300B5
:1053600073007300730073007300730073007300A5
:1053700073007300480073007300730073007300C0
:1053800073007300730073007C0040F66818C2F26B
:1053900000089DF8321098F800708F4220D1BDF8B7
:1053A00030309DF834205F1EB8B2C62801F26B8100
:1053B0000C2A01F268819DF83510002901F0638103
:1053C00004EE903AB8EEE44A40F67809C9EE043AA1
:1053D000C2F2000909EB820ABCEEE33A8AED193AFF
:1053E00040F6780BC2F2000B9BF8020009F07AFD40
:1053F00021E640F66818C2F200089DF84E0098F8C1
:1054000000708742ECD140F6780BC2F2000B0AA87C
:10541000FFF792FC9BF8020009F064FD0BE640F6F2
:105420006819C2F200099DF8320099F80070B8427C
:10543000D6D19DF830A0BAF1190F41F238814FF062
:10544000010840F6B053C2F2000340F668199A7999
:105450008DF8BC7182F01C0C8CEA0C1A5FFA8AFB86
:105460004FEA1B1080F03D0141EA0B2080EACB009F
:1054700080EA070E8EEA0E1C5FFA8CF14FEA1020CC
:10548000C2F2000980EA111A99F801908DF8AE2154
:105490004AEA012B8BEAC10080EA090E8EEA0E1C53
:1054A0005FFA8CF1000A80EA111A4AEA012B8BEAB2
:1054B000C1004FF02F0B80EA0B0E8EEA0E1C5FFA34
:1054C0008CF1000A80EA111A8AEA012080EAC10EF2
:1054D0001FFA8EF087EA000C8CEA0C1A5FFA8AF148
:1054E000000A80EA111040EA012E8EEAC10080EA2B
:1054F000090C8CEA0C1A5FFA8AFC000A80EA1C1E6E
:105500008EEA0C2181EACC0080B280EA080A8AEA9D
:105510000A115FFA81FA000A80EA1A1E4EEA0A2C82
:105520008CEACA00C1B281F0990181EA01115FFAE7
:1055300081FE010A81EA1E11501C4FF0FE0A0590FF
:1055400041EA0E2C8CEACE0E51468DF8ACA1059A9C
:105550008DF8BE814FF0030A0020CDF810E08DF8E1
:10556000BD918DF8ADA18DF8AF718DF8B0918DF82A
:10557000B1B19A71FDF7CAF89DF8AD110020FDF7A1
:10558000C5F89DF8AE110020FDF7C0F89DF8AF11E9
:105590000020FDF7BBF89DF8B0110020FDF7B6F82C
:1055A0009DF8B1110020FDF7B1F839460020FDF754
:1055B000ADF849460020FDF7A9F841460020FDF767
:1055C000A5F8049F0020F9B2FDF7A0F840F6780B8B
:1055D000049BC2F2000B0020190AFDF797F89BF814
:1055E000020009F07FFC26E540F66819C2F20009C6
:1055F0009DF8307099F800309F427FF4F1AE0AF0C8
:1056000053FE40F6B053C2F2000380469A7999F8EF
:1056100001C099F800B0CDF814C082F01C0181EAF5
:10562000011A5FFA8AF1080980F03D0989EAC10090
:1056300080EA012080EA0B0A8AEA0A195FFA89FAED
:10564000000A80EA1A1181EACA0080EA0A2188B2B7
:1056500080EA0C0A8AEA0A1C5FFA8CF1000A80EAE6
:10566000111080EAC10989EA012080F02F0A8AEA34
:105670000A1C5FFA8CF9000A80EA191181EA0920F4
:1056800080EAC90188B287EA000A8AEA0A1C5FFA3E
:105690008CF1000A80EA111989EAC10080EA012030
:1056A0004FF0BE0980EA090A8AEA0A1C5FFA8CFAFE
:1056B000000A80EA1A1181EACA0080EA0A2188B247
:1056C00080EA080C8CEA0C1A5FFA8AFA010A81EA6D
:1056D0001A1040EA0A2C8CEACA00C1B281F0990182
:1056E00081EA01115FFA81FE010A81EA1E11501C54
:1056F0008DF8AE21059A06904FF0FE0A41EA0E2C75
:105700008CEACE0C51468DF8ACA18DF8B0214FF04B
:10571000030A4FF02F028DF8B1218DF8BC710020E3
:10572000CDF810C08DF8BD918DF8BE818DF8ADA17A
:105730008DF8AFB1069A1CE740F66818C2F200086F
:105740009DF8302098F800B093457FF449AE9DF85D
:105750002D709DF82EB00AF08DFD40F6B053C2F2C8
:10576000000398F800C09A7998F801A0ADF8AC0150
:1057700082F0A30181EA01195FFA89F14FEA111859
:1057800088F0490E4EEA012989EAC10E8EEA0C081A
:1057900088EA0811C9B24FEA1E2989EA111888EA75
:1057A000012E8EEAC1091FFA89FE8EEA0A0888EAEC
:1057B0000811C9B24FEA1E2989EA111848EA012ED8
:1057C0008EEAC10E8EF02C0989EA09185FFA88F971
:1057D0004FEA1E2181EA191181EA092181EAC901F2
:1057E0001FFA81F989EA000888EA081E5FFA8EF834
:1057F0004FEA192181EA181141EA082E8EEAC809F8
:1058000089EA102080EA0011C9B24FEA192888EA13
:10581000111E8EEA012080EAC1091FFA89F080EA90
:10582000070888EA081E5FFA8EF1000A80EA111064
:1058300040EA012989EAC10080EA0B0888EA081ECB
:105840005FFA8EF8000A80EA181989EA082181EACD
:10585000C80080B2C1B281F0DD0181EA01115FFAB6
:1058600081FE010A501C04908DF8AE7104278DF85A
:10587000B571049F8DF8B62181EA1E114FF0FE0824
:1058800041EA0E292C229F714146002089EACE0967
:105890008DF8B7C18DF8B9218DF8AFB18DF8B4810D
:1058A0008DF8B8A1FCF732FF9DF8B5110020FCF788
:1058B0002DFF9DF8B6110020FCF728FF9DF8B711C9
:1058C0000020FCF723FF9DF8B8110020FCF71EFF15
:1058D0009DF8B9110020FCF719FF9DF8AC110020CC
:1058E000FCF714FF9DF8AD110020FCF70FFF9DF8A9
:1058F000AE110020FCF70AFF40F6780B9DF8AF11BF
:105900000020FCF703FFC2F2000B5FFA89F10020D0
:10591000FCF7FCFE00204FEA1921FCF7F7FE9BF88C
:10592000020009F0DFFAFFF786BB40F6681BC2F2FF
:10593000000B9DF832209BF8008090457FF450AD1D
:10594000BDF83030182B3FF64BAD40F6780BC2F265
:10595000000BD8B209F018FC9BF8020009F0C2FA5B
:10596000FFF769BB40F66818C2F200089DF83020C6
:1059700098F8009091457FF433AD40F6780BC2F271
:10598000000B0027CBF86070CBF85C7040F6780B0A
:10599000C2F2000B9BF8020009F0A4FAFFF74BBB20
:1059A00040F66818C2F200089DF8502098F8007080
:1059B000BA427FF415ADBDF84CB09DF85280BBF1F2
:1059C000180F07D8B8F1000F00F01E86B8F1030FCA
:1059D00000F01A864FF0010840F6B05AC2F2000AF1
:1059E000CDF814A09AF806A08AF01C0E8EEA0E10CC
:1059F000C2B2130983F03D0141EA022080EAC203EA
:105A000083EA070C8CEA0C1E40F668195FFA8EF2E6
:105A1000190AC2F2000981EA121099F8019040EACD
:105A2000022383EAC20181EA090C8CEA0C1E5FFAA8
:105A30008EF2080A80EA121343EA022181EAC200C8
:105A400080F02F0C8CEA0C1E5FFA8EF2030A83EAB8
:105A5000121181EA022080EAC20C1FFA8CF187EA57
:105A6000010E8EEA0E135FFA83FC080A80EA1C120C
:105A700042EA0C2383EACC0383EA090181EA01109C
:105A8000C0B21A0A82EA101181EA002E8EEAC0031F
:105A900099B281EA080282EA021C5FFA8CF3080AD2
:105AA00080EA131E4EEA032181EAC301CAB240F61E
:105AB000780CC2F2000C82F099004FF4406280EA48
:105AC0000013C4F200020BF101005FFA83FE8CF8B0
:105AD000DA00080A536A8DF8BC7180EA1E1141EAA7
:105AE0000E22CCF8DC3082EACE0CDDF814E0CDF8E2
:105AF00010C00AF101034FF0FE0B03228EF80630AE
:105B0000594600208DF8AD214FF02F028DF8B121BC
:105B10008DF8ACB18DF8AF718DF8BD918DF8BE8167
:105B20008DF8AEA18DF8B091FCF7F0FD9DF8AD11A8
:105B30000020FCF7EBFD9DF8AE110020FCF7E6FD20
:105B40009DF8AF110020FCF7E1FD9DF8B011002099
:105B5000FCF7DCFD9DF8B1110020FCF7D7FD3946BC
:105B60000020FCF7D3FD49460020FCF7CFFD41465D
:105B70000020FCF7CBFD049F0020F9B2FCF7C6FD26
:105B800040F6780B049BC2F2000B0020190AFCF7C8
:105B9000BDFD9BF8020009F0A5F9FFF74CBA40F6ED
:105BA0006813C2F200039DF83420187882427FF413
:105BB00017AC40F6B051C2F2000193F801C08F79E2
:105BC0009DF835908DF8B67187F0F10E8EEA0E1AB9
:105BD0005FFA8AF34FEA131888F0E70B4BEA032EBB
:105BE0008EEAC30B40F220108BEA020AC1F20000D9
:105BF000D0ED431A8AEA0A18DFED7D2A5FFA88F3AE
:105C00004FEA1B2080EA131E71EEE26A9FED792AAB
:105C10004EEA032A8AEAC30086EE821A80EA0C085A
:105C200088EA081B5FFA8BFE030A83EA1E1080EAEB
:105C30000E2383EACE0A1FFA8AF04FF0010E80EAA3
:105C40000E0888EA081B5FFA8BFA000A80EA1A132A
:105C500043EA0A2080EACA0840F67803C2F2000349
:105C600088EA0810C0B24FEA182B21EE280AB3F8D0
:105C7000D2A0B3F8D08083F8D49061EEA80A8BEA62
:105C8000101383EA002BBDEEC07A8BEAC00BFCEE4A
:105C9000E07A4FF6FF700023ADF8700117EE100A9E
:105CA00017EE909A589359935A93ADF87231ADF814
:105CB0007631ADF87831ADF87A31ADF87C31FE232C
:105CC0007744CAF57A7A8DF87E018DF8B4311F20B9
:105CD0005FAB8DF8B7218DED047A58AA8F71ADF8BE
:105CE0006CA1DF1CADF86E91ADF874818DF8B50133
:105CF0008DF8B8C18DF8B9E101321FFA8BF3114666
:105D000092F801B011F8019B89EA030C8CEA0C129D
:105D10004FEA13205FFA82FA80EA1A1E4EEA0A2836
:105D200088EACA028BEA020080EA00135FFA83FC69
:105D3000100A80EA1C1242EA0C294A1CBA4289EA7B
:105D4000CC03DCD183F07C0080EA0011C8B21B0ACE
:105D500083EA101787EA002282EAC0018BB2002092
:105D6000FE215FFA83FB4FEA132AFCF7CFFC9DF874
:105D7000B5110020FCF7CAFC9DF8B6110020FCF715
:105D8000C5FC9DF8B7110020FCF7C0FC9DF8B811C8
:105D90000020FCF7BBFC4FF000089DF8B911002073
:105DA000FCF7B4FC9DF86011404658AF0DF5BF7983
:105DB000FCF7ACFC79784046FCF7A8FCB978404683
:105DC0000237FCF7A3FC4F45F4D1594640F6780B57
:105DD0000020C2F2000BFCF799FC00205146FCF7B2
:105DE00095FC9BF8020009F07DF8FFF724B900BF8D
:105DF000CDCC1C419A99494140F66818C2F200087E
:105E00009DF8323098F800709F427FF4E9AABDF8FF
:105E1000307038460AF064FA90F82C2090F82D90F3
:105E2000012A0CBF4FF0030B4FF0000BB9F1010F2B
:105E3000824600F07385B9F1030F01F06D80B9F16E
:105E4000020F01F02480B9F1040F00F0D487B9F1FA
:105E5000050F00F08F869DF82D308169049341F283
:105E6000D812C1F2000244F6D35392F83A25C1F297
:105E70006203A3FB01E39B09C7EB020EDEF1000204
:105E800007EE103AD0E9000142EB0E020892B8EE9C
:105E9000478A15F081FC0690DAE9020115F07CFCD6
:105EA00040F6B053C2F2000398F80090997998F840
:105EB00001C08DF8AE1181F0280282EA0212D2B23E
:105EC0004FEA121E8EF0790E4EEA022E8EEAC20EB4
:105ED0008EEA090282EA0212D2B24FEA1E2E8EEA3E
:105EE000121E8EEA022E8EEAC20E1FFA8EFE8EEA75
:105EF0000C0282EA0212D2B24FEA1E2E8EEA121869
:105F000048EA02284FF0270E88EAC20888EA0E0203
:105F10004FEA1828CDF82480DAF82480CDF81480D0
:105F2000DAF81080DAF814A0CDF81C80CDF838A18A
:105F300082EA0212DDF824A05390D2B28AEA121843
:105F400001F1010A88EA02214FF000080798CDF814
:105F50004081DDF814805490CDF84481ADF854713F
:105F6000DDF81880049FCDF848811020ADF8560167
:105F7000BE208DF8590181EAC2028DED4F8A8DF85D
:105F800058718DF85AB183F806A09DF83831DDF8C4
:105F900020808DF8AF9192B25340012083EA031321
:105FA000DBB2120A8DF85C01FE2082EA13118DF833
:105FB000AC0125208DF8AD0141EA032157A84EAA76
:105FC0008DF85B818DF8B0C18DF8B1E101300132FF
:105FD00081EAC303114692F801B011F801CB8CEAB3
:105FE000030E8EEA0E125FFA82F94FEA132787EA50
:105FF000191343EA092787EAC9028BEA020888EAEB
:10600000081A5FFA8AFC170A87EA1C1242EA0C2374
:106010004A1C824283EACC03DCD15FFA83FA8AF01D
:10602000FE0787EA0711CFB21B0A83EA171080EA3E
:10603000072282EAC7018BB20020FE215FFA83FAB1
:106040004FEA1329FCF762FB9DF8AD110020FCF725
:106050005DFB9DF8AE110020FCF758FB9DF8AF11D9
:106060000020FCF753FB9DF8B0110020FCF74EFB1D
:106070009DF8B1110020FCF749FB4FF000084EA835
:1060800007469DF8381140460DF5AE7BFCF73EFB08
:1060900079784046FCF73AFBB97840460237FCF77E
:1060A00035FB5F45F4D100205146FCF72FFB002063
:1060B0004946FCF72BFB40F6780BC2F2000B9BF82D
:1060C000020008F00FFFFEF7B6BF40F66818C2F2F4
:1060D00000089DF8322098F8007097427FF480A95C
:1060E00040F6780BC2F2000BBDF83030DBF8CC0084
:1060F0008342BFF675A940F2B42E40F2000CC1F203
:10610000000E0EEB8301C2F2000CD1F800905CF897
:106110002310ADF886310923CDF88091ADF88401C4
:106120008DF89831002900F02D8762A8102217F011
:10613000CDFB40F6B05BC2F2000B40F668119BF855
:10614000060080F0C70888EA0817FAB21309C2F2FD
:10615000000183F0820991F8008049788DF8AE0142
:1061600049EA022A8AEAC20787EA080E8EEA0E1C6A
:106170005FFA8CFA3A0A82EA1A1989EA0A2383EA50
:10618000CA07BFB287EA010282EA02135FFA83FC00
:106190003A0A82EA1C1747EA0C2E8EEACC0316272D
:1061A00083EA070989EA091A5FFA8AFE1B0A83EA69
:1061B0001E1260AB82EA0E2C8CEACE0213F8019B11
:1061C0008DF8AF811FFA82FC89EA0C0A8AEA0A1E5E
:1061D0005FFA8EFA4FEA1C22013082EA1A1242EA72
:1061E0000A224FF0FE094FF019088BF8060066A846
:1061F0008DF8AC918DF8AD818DF8B0118DF8B1713D
:10620000013082EACA02194693F801A011F8017B15
:1062100087EA02034FEA122B83EA0312D7B28BEA12
:10622000171848EA072989EAC7038AEA030E8EEAA3
:106230000E1C5FFA8CFB1F0A87EA1B1343EA0B2232
:106240004B1C834282EACB02DDD15FFA82FA8AF0EC
:10625000DC0E8EEA0E115FFA81FC100A80EA1C1730
:1062600087EA0C2383EACC018AB20020FE215FFA80
:1062700082FA4FEA1229FCF749FA9DF8AD11002085
:10628000FCF744FA9DF8AE110020FCF73FFA9DF8A8
:10629000AF110020FCF73AFA9DF8B0110020FCF78E
:1062A00035FA9DF8B1110020FCF730FA4FF00008E4
:1062B00060A807469DF8801140460DF5CC7BFCF7A1
:1062C00025FA79784046FCF721FAB978404602373A
:1062D000FCF71CFA5F45F4D100205146FCF716FA92
:1062E00000204946FCF712FAE5E640F66813C2F2D0
:1062F00000039DF834C0187860457FF471A80DF153
:106300003601102267A817F0E1FA40F67801C2F2D0
:106310000001D1F8CCE0BEF1000F7FF761A840F298
:106320000000C2F20000002750F8042B9DF89C31B9
:10633000117899427CD1002900F0C4819DF89D31EB
:106340005178994274D1002900F0BC819DF89E31AA
:10635000917899426CD1002900F0B4819DF89F3169
:10636000D178994264D1002900F0AC819DF8A03128
:10637000117999425CD1002900F0A4819DF8A131E6
:106380005179994254D1002900F09C819DF8A231A5
:10639000917999424CD1002900F094819DF8A33164
:1063A000D179994244D1002900F08C819DF8A43123
:1063B000117A99423CD1002900F084819DF8A531E1
:1063C000517A994234D1002900F07C819DF8A631A0
:1063D000917A99422CD1002900F074819DF8A7315F
:1063E000D17A994224D1002900F06C819DF8A8311E
:1063F000117B99421CD1002900F064819DF8A931DC
:10640000517B994214D1002900F05C819DF8AA319A
:10641000917B99420CD1002900F054819DF8AB3159
:10642000D17B994204D1002B00F04C819DF8AC3116
:10643000002B00F04781013777457FF475AF40F6B8
:10644000780BC2F2000B9BF8020008F04BFDFEF740
:10645000F2BD40F66811C2F200019DF8303091F8AB
:1064600000904B457EF4BCAF40F6B052C2F2000241
:10647000497892F806E004918EF01C0989EA091720
:10648000F9B2080980F03D0B4BEA012787EAC10009
:1064900080EA030181EA011C5FFA8CF7000A80EAB6
:1064A000171949EA072B04999DF82D809DF831A012
:1064B0008DF8AF318BEAC70080EA010C8CEA0C172B
:1064C0005FFA87FB010A81EA1B1080EA0B2989EA3F
:1064D000CB07B8B280F0060181EA011C5FFA8CF7A5
:1064E000000A80EA171949EA072B8BEAC70788EAEE
:1064F000070181EA011C5FFA8CFB380A80EA1B194C
:1065000049EA0B2787EACB0080EA0A0181EA011CED
:106510005FFA8CF7000A80EA171989EA072B8BEAE1
:10652000C70188B280EA001C5FFA8CF7000A80EA93
:10653000171949EA072B8BEAC70787F06801049B04
:106540008DF8AEE181EA01105FFA80FC0EF10100E6
:1065500005908DF8B0314FF00603390A8DF8B1314E
:10656000059B8DF8B481002781EA1C114FF0FE0BCA
:1065700041EA0C299371384659468DF8ACB14FF079
:10658000030B89EACC098DF8ADB18DF8B5A18DF872
:10659000B671FCF7BBF89DF8AD113846FCF7B6F8BC
:1065A0009DF8AE113846FCF7B1F89DF8AF113846AA
:1065B000FCF7ACF89DF8B0113846FCF7A7F89DF849
:1065C000B1113846FCF7A2F838464146FCF79EF870
:1065D00038465146FCF79AF840F6780B384639466B
:1065E000FCF794F8C2F2000B5FFA89F13846FCF729
:1065F0008DF838464FEA1921FCF788F89BF802001D
:1066000008F070FCFEF717BD9DF84E30142B00F01B
:106610002E85102B00F01D85B32B00F06E81162BFC
:1066200000F0B684012B00F0E484152B7FF4D2A98E
:10663000584609F055FE0746A8F10300D0F10008BE
:1066400048EB00080523109887F82C8087F82D3038
:1066500015F086F802460B461198C7E9002315F09D
:106660007FF8129BDDF834E03B610F9B0E9ABB6212
:10667000A94BC7F820E0C7E90201FA614FF0000812
:106680001F78FFF7A9B940F6780EC2F2000E183253
:1066900040F6780B0EEB820CC2F2000B0020CCF817
:1066A00004009BF8020008F01DFCFEF7C4BC09F0D2
:1066B000FBFD012800F0798399F800704FF0010884
:1066C000FEF7BFBEBE457EF78BAE9DED0C8AB0EEE9
:1066D000480A15F023FC002800F0F98440F67808F9
:1066E000C2F2000840F2B42CB8F8CC90ADF8867134
:1066F000C1F2000C0CEB8700ADF8849140F6B05964
:106700000368C2F2000967A91022092762A86093F2
:106710008DF8987117F0DAF899F8060080F0C70A3A
:106720008AEA0A11CAB240F6681B1309C2F2000BCA
:1067300083F082079BF800A09BF801B08DF8AFA111
:1067400047EA022E8EEAC20181EA0A0C8CEA0C1892
:106750005FFA88FE0A0A82EA1E1787EA0E2383EA96
:10676000CE0C1FFA8CF787EA0B0181EA01125FFA5F
:1067700082F83B0A83EA181141EA082282EAC80734
:10678000162187EA010E8EEA0E1C5FFA8CF83B0A8E
:1067900083EA181260AB82EA082787EAC80213F876
:1067A00001EB8DF8AE0197B28EEA070C8CEA0C185B
:1067B0005FFA88FA4FEA172787EA1A124FF0FE07A6
:1067C0008DF8AC714FF01907013042EA0A228DF8BA
:1067D000AD7166AF89F806008DF8B0B18DF8B111D2
:1067E000781C82EACA02194693F8018011F8017BED
:1067F00087EA020383EA031B5FFA8BF74FEA122E44
:106800008EEA171242EA072C8CEAC70388EA0309CA
:1068100089EA091A5FFA8AF21F0A87EA121B4B1CDF
:106820004BEA022E83428EEAC202DCD15FFA82FB7F
:106830008BF0DC0E8EEA0E1C5FFA8CF0120A82EAF4
:10684000101989EA002A8AEAC0018FB20020FE21CD
:10685000FBF75CFF00209DF8AD11FBF757FF002010
:106860009DF8AE11FBF752FF00209DF8AF11FBF72A
:106870004DFF00209DF8B011FBF748FF0DF5BE78E5
:1068800000209DF8B111FBF741FF08F103034FF021
:1068900000086FEA030240469DF8801102F0010BE8
:1068A000FBF734FF02985FFA87F94FEA172A60AFC7
:1068B000874218D0BBF1000F09D060AB40469DF86D
:1068C00081115F1CFBF722FF029887420BD0797879
:1068D0004046FBF71BFFB9784046FBF717FF029BCA
:1068E00002379F42F3D100204946FBF70FFF0020FB
:1068F0005146FBF70BFFFEF773BD9DF85380B8F1CF
:10690000000F00F0FD83044F08F0A2FB4FF00008D9
:106910003F78FFF761B800BF6809002009F0EAFC82
:106920009DF82D308169049341F2D812C1F2000222
:1069300044F6D35392F83A25C1F26203A3FB01E374
:106940009B09C7EB020BDBF1000207EE103A42EBAA
:106950000B028246D0E900010892B8EE478A14F093
:106960001BFF0690DAE9020114F016FF40F6B0535F
:10697000C2F2000398F800B0997998F801C08DF838
:10698000AE1181F0280282EA0212D2B24FEA121E40
:106990008EF0790E4EEA022E8EEAC20E8EEA0B02BD
:1069A00082EA0212D2B24FEA1E2E8EEA121E8EEA3E
:1069B000022E8EEAC20E1FFA8EFE8EEA0C0282EAC8
:1069C0000212D2B24FEA1E2E8EEA121848EA0228AC
:1069D0004FF0270E88EAC20888EA0E024FEA18280C
:1069E000CDF82480DAF82480CDF81480DAF810800D
:1069F000DAF814A0CDF81C80CDF838A182EA021292
:106A0000DDF824A05390D2B28AEA12180798ADF8A4
:106A1000547101F1010A88EA02214FF00008CDF813
:106A20004081DDF8148054901420CDF84481ADF8F5
:106A30005601DDF81880049FCDF84881BE208DF8FE
:106A40005901002081EAC2028DED4F8A8DF85871FC
:106A50008DF85A0183F806A09DF83831DDF82080C2
:106A60008DF85C9192B2534083EA0313DBB2FE20AF
:106A7000120A82EA13118DF8AC0125208DF8AD01C0
:106A800041EA032157A84EAA8DF85B818DF8AFB17A
:106A90008DF8B0C18DF8B1E10130013281EAC30354
:106AA000114692F801A011F801EB8EEA030B8BEA74
:106AB0000B124FEA1327D3B287EA131848EA0327C9
:106AC00087EAC3028AEA020989EA091C5FFA8CF89C
:106AD000170A87EA181E4A1C4EEA082B82428BEAE4
:106AE000C803DDD15FFA83FC8CF0FE0787EA07114B
:106AF000CFB21B0A83EA171080EA072282EAC70195
:106B00008BB20020FE215FFA83FA4FEA1329FBF7CC
:106B1000FDFD9DF8AD110020FBF7F8FD9DF8AE11CD
:106B20000020FBF7F3FD9DF8AF110020FBF7EEFD11
:106B30009DF8B0110020FBF7E9FD9DF8B111002090
:106B4000FBF7E4FD4FF000084EA807469DF838110A
:106B500040460DF5AE7BFBF7D9FD79784046FBF753
:106B6000D5FDB97840460237FBF7D0FD5F45F4D13B
:106B7000FFF799BA41F2D813C1F200039DF82D2016
:106B800093F83A350492C7EB030CDCF1000343EBB6
:106B90000C03D0E90001099314F0FEFD0890DAE936
:106BA000020114F0F9FD40F6B053C2F2000398F868
:106BB0000090997998F801C08DF8AE1181F0280203
:106BC00082EA0212D2B24FEA121E8EF0790E4EEA1B
:106BD000022E8EEAC20E8EEA090282EA0212D2B2B6
:106BE0004FEA1E2E8EEA121E8EEA022E8EEAC20E88
:106BF0001FFA8EFE8EEA0C0282EA0212D2B24FEA2D
:106C00001E2E8EEA121848EA02284FF0270E88EA54
:106C1000C20888EA0E0282EA0212D2B24FEA1828AB
:106C200088EA121888EA022888EAC2081FFA88F857
:106C300088EA08124FEA1828CDF80080DAF8208098
:106C4000CDF81480DAF81C80CDF81880DAF82880A6
:106C5000DAF810A0CDF81C80CDF850A1DDF800A026
:106C6000ADF85471D2B28AEA121801F1010A00217A
:106C70004E910599049F4F91069953905091079911
:106C80005191089952911521ADF85611BE218DF8F8
:106C900058718DF859110121099F8DF85C11FE2161
:106CA00048EA02288DF8AC1183F806A0252157A8E0
:106CB0004EAB8DF85AB18DF85B718DF8AD118DF832
:106CC000AF918DF8B0C18DF8B1E10130013388EAA0
:106CD000C202194693F8019011F8017B87EA02037A
:106CE00083EA03185FFA88F74FEA122A8AEA171232
:106CF00042EA072C8CEAC70389EA030E8EEA0E1BD0
:106D00005FFA8BF91F0A87EA19184B1C48EA092A0F
:106D100083428AEAC902DCD15FFA82F989F0FE0E69
:106D20008EEA0E115FFA81FB100A80EA1B1787EAD0
:106D30000B2383EACB018AB20020FE215FFA82FA9C
:106D40004FEA1229FBF7E2FC9DF8AD110020FBF79A
:106D5000DDFC9DF8AE110020FBF7D8FC9DF8AF11CB
:106D60000020FBF7D3FC9DF8B0110020FBF7CEFC10
:106D70009DF8B1110020FBF7C9FC4FF000084EA8A8
:106D800007469DF8381140460DF5AE7BFBF7BEFC7B
:106D900079784046FBF7BAFCB97840460237FBF7F2
:106DA000B5FC5F45F4D1FFF77EB940F6780EC2F22C
:106DB000000E9DF82D709DF82E308EF8D7704FF490
:106DC000406C4FF00008C4F2000C8EF8D8308EF8FA
:106DD000D9A08EF8DA80DCF8241099F80070CEF88B
:106DE000DC10FEF72EBB0021BE78B970002B7EF4BC
:106DF00075AAFEF720B9BF4BD0F818E093F83A35E2
:106E00009DF82D804FF47A72BEFBF2F2C7EB0309B6
:106E1000D9F1000307EE102AD0E9000143EB090382
:106E2000B8EE478A019314F0B7FC8146DAE9020113
:106E300014F0B2FCDAF81010DAF81CC0DAF824E02A
:106E4000019BDAF814A054910122BE218DED4F8AE6
:106E5000CDF838A1CDF840C1CDF844E1CDF8489146
:106E60005390ADF85471ADF856218DF858818DF8D6
:106E700059118DF85AB18DF85B318DF85C212720BE
:106E80004EA92522FE23FBF749FCFEF7A9BA994B30
:106E9000D0F818E093F83A359DF82D804FF47A72C7
:106EA000BEFBF2F2C7EB030EDEF1000307EE902A01
:106EB000D0E9000143EB0E03B8EE678A019314F0AA
:106EC0006BFC8146DAE9020114F066FCDAF8102066
:106ED000DAF824E0DAF82010DAF814C054928DEDD4
:106EE0004F8ACDF838C1CDF840E15191CDF84891A5
:106EF0005390ADF8547116220198ADF85621BE2377
:106F000001228DF858818DF859318DF85AB18DF8DC
:106F10005B018DF85C21B2E7764BD0F818E093F86E
:106F20003A359DF82D804FF47A72BEFBF2F2C7EB32
:106F3000030CDCF1000307EE102AD0E9000143EB5B
:106F40000C03B8EE478A019314F026FC8146DAE977
:106F5000020114F021FCDAF81020DAF81CE0DAF86B
:106F60002410DAF814C05492CDF838C18DED4F8A50
:106F7000CDF840E15191CDF848915390ADF854715E
:106F80001022B9E762A8102216F0BEFCFFF7D1B8B4
:106F9000584609F0A5F9A8F1030C0746DCF10008F2
:106FA00048EB0C080223109887F82C8087F82D30C6
:106FB00014F0D6FB02460B461198C7E9002314F0E3
:106FC000CFFB129A0C9B3A61DDED0D7A7B610F9B32
:106FD0000E9A3B6267EEA87A474B7A62FCEEE77A3C
:106FE000C7E90201C7ED067A4FF000081F78FEF7E7
:106FF000F3BC584609F074F90746A8F10300414272
:1070000041EB0002109887F82C20042387F82D30DC
:1070100014F0A6FB02460B461198C7E9002314F0B2
:107020009FFBDDED0D7A129A0C9B3A6167EEA87A10
:107030007B610F9B0E9A7B62FCEEE77AC7E9020147
:10704000C7ED067A2C4BFA611F784FF00008FEF767
:10705000C3BC584609F044F9A8F103030746584257
:1070600040EB030187F82C1010980323CEE7584615
:1070700009F036F9012380F82D3009F03BF9074675
:107080000323109887F82D3014F06AFB02460B4654
:107090001198C7E9002314F063FB129A0C9B3A6124
:1070A0007B610F9BDDED0D7A7B62144B67EEA87A56
:1070B000D3F8FC31FCEEE77AFB610F4BC7E9020124
:1070C000C7ED067A4FF000081F78FEF785BCB0EEDA
:1070D000480A14F00FFF00287FF400AB94F8BC219D
:1070E00051073FF5FBAA054800EB870E8EED008A9D
:1070F000FFF7F4BAD811001068090020B40200109C
:1071000009F0F8F807460323109887F82D3014F09B
:1071100027FB02460B461198C7E9002314F020FB19
:10712000129A0C9B3A617B610F9BDDED0D7A7B62BD
:10713000074B67EEA87AD3F8FC31FCEEE77AFB61E7
:10714000044BC7E90201C7ED067A1F78FEF744BC7D
:10715000B4020010680900202DE9F04F40F67804D1
:10716000C2F2000440F2B42B83B00021F022C1F23D
:10717000000B204616F0C8FBDBED7D1AFCEEE17A31
:1071800000264FF4805017EE901A33464FF44072A9
:10719000C4F2010000960EF085F8606507F0FAFD74
:1071A000012203461421201DA3700BF0D1FA0146E1
:1071B0004FF26C50C0F60100E170FBF7C9FB40F2E2
:1071C0006B10C4F8CC00206609F054F84FF27C51E3
:1071D000C5B26A1CC0F601014FF48C7084F8D95016
:1071E00084F8DA2011F0F0FA40F6146AC2F2000ACC
:1071F000074600F58A6341F6280244F66570314679
:10720000C0F20102CAF800700C33C0F6000010F0A2
:10721000A3FC03463046637005F072F844F6D35180
:10722000C1F26201A1FB001540F66819C2F2000923
:107230002A09FA274FF4406807FB12030125C4F21C
:10724000000802220327BE2189F8003089F80220B5
:1072500089F8011084F8D57084F8D46084F8D65089
:10726000D8F8246002EE106A9FED473AF8EE422A01
:10727000DFED463A72EE837A9FED454ADFED454AEF
:107280009FED455ADFED455A9FED456A9FED451A42
:10729000DFED456ADFED450A9FED457A9FED450A32
:1072A000DFED451A37EEA32A77EE842A37EEA43AAB
:1072B00077EE853A37EEA54A77EE864A37EE815A61
:1072C00077EEA65A37EEA06A37EE871A77EE800A75
:1072D00037EEA10ABCEEC22AFCEEE22ABCEEC33AAB
:1072E000BCEEC44AFCEEE44AFCEEE55A44F240230C
:1072F000FCEEE33ABCEEC55ABCEEC66AFCEEC16ACF
:10730000BCEEE07AFCEEC07A48F2A062C0F20F0355
:1073100065F31F4212EE10AA12EE909A13EE108A35
:1073200014EE107A14EE906A15EE90BA84ED2F6A7E
:10733000C4ED306A84ED317AA36684ED272AE366D2
:10734000C4ED282A236784ED293AC4ED2A3AA367BD
:1073500084ED2B4AE367C4ED2C4AC4F8803084EDF9
:107360002D5AC4F88430C4ED2E5AC4F88830C4F8BD
:107370008C30C4F89030C4F89430C4ED327A62672F
:1073800003B0BDE8F08F00BF8096984A00409C454E
:1073900000401C4600606A4600409C460050C346C0
:1073A0000060EA4600B8084700401C4700C82F4765
:1073B0000050434700D8564700606A474FF440608A
:1073C000C4F20000B0F80CC02CF0020211040B0C47
:1073D0000221838114F014B84FF44060C4F200001D
:1073E000B0F80CC02CF0040211040B0C04218381B2
:1073F00014F006B84FF44060C4F20000B0F80CC0BE
:107400002CF0080211040B0C0821838113F0F8BF43
:1074100070B58AB000250126322209A88DF82420F3
:107420008DF825608DF826508DF8276006F0E0F87D
:107430000820314613F01CF942F2A03CC2F2000CC5
:107440004DF68360DCF80830ADF8205013FA06F4EE
:10745000C4F21B30A0FB04214FF44064C4F20004CA
:10746000880C4FF0FF32431E06A920460792ADF864
:107470001830ADF81A5013F0D3FC2946204613F00B
:1074800039FDFFF79BFFFFF7A7FFFFF7B3FF01A849
:1074900013F06AFE2023204601A9ADF80430ADF8B0
:1074A0000660ADF8105013F039FD2046294613F060
:1074B00065FE204601A913F07DFD2046294613F004
:1074C00067FE2046314613F01BFD0AB070BD00BFB9
:1074D00010B44FF4406340F61C64C4F20003C2F2DF
:1074E00000044FF6FD7CE2602160A3F810C0596AE9
:1074F00042185A63998988B240F002029A8110BCFE
:10750000704700BF10B44FF4406340F61C64C4F2EF
:107510000003C2F200044FF6FB7C22616160A3F815
:1075200010C0596A42189A63998988B240F00402DF
:107530009A8110BC704700BF10B44FF4406340F60E
:107540001C64C4F20003C2F200044FF6F77C6261CF
:10755000A160A3F810C0596A4218DA63998988B209
:1075600040F008029A8110BC704700BF70B54FF41C
:107570004064C4F200042046022113F035FF20BB12
:107580002046042113F030FF58B92046082113F09B
:107590002BFF002841D12046102113F025FF38BBD6
:1075A00070BD4FF6FB7CA4F810C0A18940F61C6E9C
:1075B00021F00400C2F2000E0204130CDEF81000E9
:1075C000DEF80410A381884770BD4FF6FD72228259
:1075D000A38940F61C6C23F00200C2F2000C0104E7
:1075E0000A0CDCF80C00DCF80030A281984770BD72
:1075F00041F68005C1F2000520466E6913F0C4FE15
:10760000B11C05EB810C0136CCF80400102120469A
:107610006E61BDE8704013F0F3BE4FF6F772228240
:10762000A38940F61C6E23F00800C2F2000E01048C
:107630000A0CDEF81400DEF80830A281984770BD0D
:10764000034610B442F8043C4FF080746FF001031D
:10765000A2F13C00146042F8083C42F81C1C10BC2B
:10766000704700BFF8B540F6456540F63864C2F291
:107670000005C2F20004D4E9000142F2D8732F7869
:10768000C2F20003012201371E6800238018FFB2F6
:1076900041EB03012F70C4E9000126B1F369012B0E
:1076A0000BD9013BF36140F64661C2F200010122B1
:1076B0000A70BDE8F84001F0BFBE0020F06110F094
:1076C000BBFBF0E730B48D082FD06B1E1C4603F0D7
:1076D000010280ED000A80ED010A80ED020A80EDD2
:1076E000030A00F11003F4B152B183ED000A83EDF7
:1076F000010A83ED020A83ED030A1033013C12D024
:1077000083ED000A83ED010A83ED020A83ED030A8B
:1077100083ED040A83ED050A83ED060A83ED070A6B
:107720002033023CECD100EB051011F0030113D023
:1077300001390B46A0EC010A01F0010163B119B156
:10774000013BA0EC010A07D00246A2EC010A80ED41
:10775000010A101D023BF7D130BC70470180428006
:10776000436070472DE9F00F4B8844884F6852689A
:107770008EB0A1080A93DDF828804368008801973D
:107780004FEAC806059604F003074D1EDDF814C045
:10779000079008F1FF39A8B27E1E1FFA89F5039100
:1077A0004FEA880101300497B6B2AF000CEB4105F7
:1077B0000B92A40003EB001C0022043700FB05F031
:1077C000B600099408920C9706900D960B9F0898A6
:1077D0000C9E0D9C07EB800808EB06029FED776A74
:1077E000019E02924FF0000904F1040B039C002C4F
:1077F00000F0E080D6ED007AD3ED002AB0EE462A04
:1078000002EEA72A7018D0ED001A059F93ED011A19
:10781000F0EE427AF01941EE217AD0ED000A93EDB4
:10782000020A421840EE207AC3EB0C0A92ED007A6D
:10783000D3ED036A03F11002AAF110049445C4F3D6
:10784000001A674646EE877A05EB0604284460D0A6
:10785000BAF1000F20D092ED004AD4ED004A04EBBB
:10786000010A44EE247A92ED013ADAED003A43EE51
:10787000237A92ED022AD0ED002A00EB010A42EEB3
:10788000227A92ED031ADAED001A1032944541EE95
:10789000217A2C4428443CD09A4692ED003AD4ED0B
:1078A000003A631843EE237A92ED012AD3ED002AC1
:1078B00042EE227A92ED021AD0ED001A431841EE00
:1078C000217A92ED030AD3ED000A2C1940EE207ABA
:1078D000D2ED046A94ED007A631846EE877A92ED51
:1078E000055AD3ED005A401945EE257A92ED064A25
:1078F000D0ED004A431844EE247A92ED073AD3EDD6
:10790000003A2032974243EE237A2C442844C4D1D3
:107910005346069AB618049850B33A46B2EC014A58
:10792000D6ED004A5F44ABF10404BA42C4F38000D0
:1079300044EE247A0E441BD040B1B2EC010AD6EDDD
:10794000000ABA420E4440EE207A11D01046F0EC04
:10795000016A96ED007A761846EE877A92ED015A22
:10796000D6ED005A021DBA4245EE257A0E44EDD1FD
:10797000E8EC017A029F019A09F101041FFA84F9E7
:10798000B84502EB89067FF431AF079E0A9F721E4D
:10799000089E90B2F4190790A2B20998079C089229
:1079A0001B188444002C7FF411AF20460EB0BDE8B4
:1079B000F00F7047F0EE467A1F46ACE7000000007B
:1079C0002DE9F00FB0F802A003884568496886B039
:1079D0004FEA9A00421E5C1E009090B29A00DB00B3
:1079E000019303910199A3B24FEA001B01EB4201FD
:1079F00001305C1C01FB00F302900AF0030A0494BE
:107A00004FF000090BF1100B0593039C009B1FFA2C
:107A100089F004EB800C002B4FD02E68019BCCF832
:107A20000060D5F804800CEB0200ABF11006C0F842
:107A30000080AF680CEB030084180760EF6805EB6B
:107A40000B0805F1100398452760C6F3001601EBFB
:107A50000C0408442CD076B11E6826605F68A61816
:107A60000C1937609E680660DF68861810339845E9
:107A7000376008441CD02F461D6825605E68A51835
:107A80000C192E609D680560DE68851840182E6010
:107A90001D6925605E69A5180C192E609E69066037
:107AA000DE698518203398452E600844E4D13D46B0
:107AB000029B059C05EB0315A444BAF1000F28D0E6
:107AC0000AF1FF372B46BEB205EB860453F8047B60
:107AD000601B0434A342CCF80070C0F380009444CF
:107AE00014D030B153F8040BA342CCF800009444F6
:107AF0000CD0184650F8047BCCF800705F689444B2
:107B0000031DA342CCF800709444F2D1013605EB7A
:107B10008605049B09F1010999457FF476AF0020A1
:107B200006B0BDE8F00F704770B48D087AD0D0ED84
:107B3000001A9FED3E2AD0ED016A32EE211AD0EDF7
:107B4000020A31EE260A6B1E70EE207A90ED037A5F
:107B50001C4603F0010677EE877A00F11003B4B3F8
:107B600096B1D3ED006A93ED017A37EEA61AD3ED04
:107B7000020A71EE077A93ED030A37EEA06A10331A
:107B8000013C76EE007A22D0D3ED001AD3ED016AE3
:107B900037EEA11A93ED027A71EE260A93ED030AED
:107BA00070EE877A93ED046A77EE805A93ED055A6A
:107BB00075EE864A93ED064A74EE853A93ED073AE0
:107BC00073EE842A2033023C72EE837ADCD100EB20
:107BD000051011F003041BD0013CB0EC012A234630
:107BE00077EE827A04F0010493B12CB1F0EC015AE3
:107BF000013B77EEA57A0BD00446F4EC013A90ED08
:107C0000013A77EEA32A201D023B72EE837AF3D16C
:107C100005EE101AF8EE454A87EEA44A82ED004AB6
:107C200070BC7047DFED017AD3E700BF00000000B1
:107C3000F0B58D0883B09FED870A00F00881D0ED84
:107C4000001A01EEA10A90ED011A01EE010AD0ED31
:107C5000020A00EEA00A6B1ED0ED037A1C4603F068
:107C6000010607EEA70A00F11003B4B396B1D3EDF5
:107C7000005A05EEA50A93ED011A01EE010AD3EDB3
:107C8000020A00EEA00AD3ED037A1033013C07EE9E
:107C9000A70A22D0D3ED005A05EEA50A93ED015AAA
:107CA00005EE050AD3ED024A04EEA40A93ED034A59
:107CB00004EE040AD3ED043A03EEA30A93ED053A69
:107CC00003EE030AD3ED062A02EEA20A93ED072A79
:107CD0002033023C02EE020ADCD100EB051311F066
:107CE00003071BD07E1EB3EC016A344606EE060A7B
:107CF00006F0010694B12EB1F3EC016A013C06EEE8
:107D0000A60A0BD01E46B6EC017A07EE070AD3EDA1
:107D1000016A331D023C06EEA60AF3D100EE901A6A
:107D2000B8EE606AF7EE007A76EE675A80EE250AC2
:107D3000002D00F0898090ED004ADFED464AD0ED3D
:107D4000013A34EE843AD0ED022A33EE232A6C1E37
:107D500032EE221AD0ED031A214671EE217A04F098
:107D6000010400F11003B1B394B193ED007A93EDE7
:107D7000015A77EE874A93ED024A74EE853A93ED05
:107D8000033A73EE842A1033013972EE837A22D0DB
:107D900093ED007A93ED015A77EE874A93ED024A0C
:107DA00074EE853A93ED033A73EE842A93ED042A38
:107DB00072EE831A93ED051A71EE820AD3ED066A0C
:107DC00070EE817A93ED077A37EEA65A20330239A6
:107DD00075EE077ADCD100EB0510DFB1013FF0EC66
:107DE000016A3B4677EEA67A07F0010793B12FB1FF
:107DF000B0EC012A013B77EE827A0BD00146B1EC60
:107E0000011AD0ED010A77EE817A081D023B77EE68
:107E1000A07AF3D1C7EE861AC6EE255A21EEA16AE2
:107E20009FED0C7A06EE650AB4EEC70AF1EE10FA81
:107E300003DC82ED007A03B0F0BD019215F068FB1F
:107E4000019A82ED000AF6E7DFED027AC5E7034604
:107E500045E700BF00000000DFED0F7AB4EEE70A4F
:107E6000F1EE10FA08D59FED0D7A30EE070AB4EE68
:107E7000E70AF1EE10FAF8D4DFED087AB4EEE70A7B
:107E8000F1EE10FA06DB30EE670AB4EEE70AF1EE27
:107E900010FAF8DA704700BF000000000000B44399
:107EA00030EEC00ADFED107AB4EEE70AF1EE10FA18
:107EB00008DD9FED0E7A30EE470AB4EEE70AF1EEE8
:107EC00010FAF8DCDFED0A7AB4EEE70AF1EE10FA08
:107ED00008D89FED067A30EE070AB4EEE70AF1EE15
:107EE00010FAF8D9704700BF000034430000B443D3
:107EF000000034C340F2B423C1F200032DE9F00FB7
:107F00004FF0000BC4F2CE2BC3F800B04FF0804B03
:107F1000C3F810B04FF0000BC4F2400BC3F814B01C
:107F20004FF0814BC3F818B04FF0000BC4F2A00B18
:107F3000C3F81CB04FF0000BC4F2C00BC3F820B064
:107F40004FF0000BC4F2E00BC3F824B04FF0824BAB
:107F5000C3F828B04FF0000BC4F2101BC3F82CB0CC
:107F60004FF0000BC4F2201BC3F830B04FF0000BF1
:107F7000C4F2301BC3F834B04FF0000BC4F2400B16
:107F8000C3F838B04FF4804BC4F2884BC3F83CB010
:107F90004FF0000BC4F2BD4BC3F840B043F2333B8B
:107FA000C3F6337BC3F848B04BF2177BC3F6D11B43
:107FB000C3F854B04FF0000BC4F2202BC3F858B0F4
:107FC000C3F85CB04FF0000BC4F2963BC3F864B04A
:107FD0004FF0000BC4F2343BC3F868B04FF4C04B11
:107FE000C4F2E05BC3F874B04FF440404CF6CD44AB
:107FF00000254FF0000B00224FF07E51C4F2794073
:10800000C4F2A015C3F64C544FF07A59C4F27A3B2F
:10801000D9601D66C3F87890D8675A609A605A6430
:10802000DC641C65DA661A67C3F88000C3F888B0A0
:108030004FF0000BC4F2963BC3F88CB049F69A1B84
:10804000C3F6196BC3F890B04FF0000A4FF0000B65
:10805000C4F2A02AC4F2482BC3F894B0C3F89CA081
:10806000C3F8A0A0C3F8A4A04FF0000B4FF0000A83
:10807000C4F2343BC4F2702AC3F8A8B0C3F8ACA071
:1080800041F26F2B4FF0000AC3F6032BC4F2DA4A19
:10809000C3F89890C3F8B0B0C3F8B4A0C3F8B890D0
:1080A0004FF0000B4FF000094CF2AC5AC4F2962985
:1080B000C4F27A3BC3F2A77AC3F8C090C3F8C8B041
:1080C000C3F8D0A04FF000094DF20A7B4FF0000A30
:1080D000C3F6A079C3F6235BC4F6610AC3F8DC904B
:1080E000C3F8E0B0C3F8E890C3F8ECA04FF0000983
:1080F0004FF4204B4FF4404AC4F24839C4F28C4B41
:10810000C4F2734AC3F8F090C3F8F8B0C3F8FCA007
:108110004FF000084FF440494FF0000B4FF0000AB9
:10812000C4F21638C4F2F349C4F2FA3BC4F2E17A5D
:10813000C3F88400C3F80091C3F804B1C3F8BC804D
:10814000C3F8C480C3F8CC40C3F8D420C3F8D82007
:10815000C3F8E420C3F8F420C3F80821C3F80C21C5
:10816000C3F81021C3F81421C3F81821C3F81C2147
:10817000C3F82021C3F82421C3F82821C3F82C21F7
:10818000C3F83021C3F83421C3F83821C3F83C21A7
:10819000C3F84021C3F84421C3F84821C3F84C2157
:1081A000C3F85021C3F85421C3F85821C3F85C2107
:1081B000C3F86021C3F86421C3F86821C3F86C21B7
:1081C000C3F87021C3F87421C3F87821C3F87C2167
:1081D000C3F88021C3F88421C3F88821C3F88C2117
:1081E000C3F89021C3F8F4A14FF0000AC4F2E00AEA
:1081F000C3F8F851C3F808A2C3F81052C3F81452D8
:108200004FF000094DF20A7A0025C3F6A33AC4F2F2
:10821000A0094FF07F5BC4F2F015C3F8FC91C3F8DE
:1082200000B2C3F80CA2C3F89421C3F89821C3F894
:108230009C21C3F8A021C3F8A421C3F8A821C3F846
:10824000AC21C3F8B021C3F8B421C3F8B821C3F8F6
:10825000BC21C3F8C021C3F8C421C3F8C821C3F8A6
:10826000CC21C3F8D021C3F8D421C3F8D821C3F856
:10827000DC21C3F8E021C3F8E421C3F8E821C3F806
:10828000EC21C3F8F021C3F80422C3F81852C3F854
:108290002402C3F82C020020C4F24830C3F8300294
:1082A0000020C4F22F40C3F83C02C3F84002002073
:1082B000C4F22000C3F84C02C3F8540243F2333C2A
:1082C0004AF2E35748F65C7646F266694CF6CD4BC7
:1082D0000020CBF6D37CC3F69B47C3F64266C4F2BC
:1082E0003609C3F64C6BCCF282204FF07C55C3F8B4
:1082F0003492C3F844B2C3F85CC2C3F860C2C3F896
:1083000064C2C3F81C52C3F82022C3F82822C3F861
:108310003882C3F84822C3F85022C3F85822C3F861
:108320006822C3F86C22C3F87022C3F87422C3F821
:108330007822C3F87C22C3F88022C3F88422C3F8D1
:108340008822C3F88C72C3F89072C3F89472C3F891
:108350009822C3F89C2243F6715CC3F8A02247F62A
:10836000FA69C3F8A422C3F8A822C3F8AC22C3F860
:10837000B022C3F8B422C3F8B822C3F8BC22C3F8B1
:10838000C022C3F8C422C3F8C822C3F8CC22C3F861
:10839000D022C3F8D422C3F8D822C3F8DC22C3F811
:1083A000E022C3F8E422C3F8E822C3F8EC22C3F8C1
:1083B000F022C3F8F422C3F8F822C3F8FC22C3F871
:1083C0000023C3F80463C3F80863C3F80C63C3F85D
:1083D0001023C3F81423C3F81823C3F81C23C3F8CD
:1083E0002023C3F82423C3F82823C3F8A0034FF4A1
:1083F0002040CBF6AA7CC3F6EA59C4F20C50C3F86D
:108400004CC3C3F850C3C3F854C3C3F87C93C3F838
:108410008093C3F88493C3F82C23C3F83023C3F8A4
:108420003423C3F83823C3F83C23C3F84023C3F8EC
:108430004423C3F84823C3F85823C3F85C23C3F884
:108440006023C3F86423C3F86823C3F86C23C3F81C
:108450007023C3F87423C3F87823C3F88823C3F8C0
:108460008C23C3F89023C3F89423C3F89823C3F84C
:108470009C23C3F8A423C3F8A823C3F8AC234FF468
:108480000049C3F8B023C3F8B4030020C4F23B4949
:10849000C4F24830C3F8C093C3F8C4034FF4004B90
:1084A0004FF4204C4FF4804040F6A169C4F23B4B9E
:1084B000C4F20C5CC4F2B440C3F66A49C3F8B8B362
:1084C000C3F8BCC3C3F8CC03C3F8D4934FF4604BD8
:1084D00040F6413C002041F25D69C4F2C44BC3F652
:1084E000344CC4F26000C4F26D19C3F8C8B3C3F8C9
:1084F000D0C3C3F8E003C3F8EC9343F2333C03F575
:10850000806945F6C04043F2667BC4F2530CC4F266
:108510001310C4F2E92BC3F8D8A3C3F8E4C3C3F81B
:10852000E803C3F8F4B3C9F80020C9F8042049F6F9
:10853000364ADFF81C93C3F8DC234DF2AE6C42F6EA
:10854000CD104EF2C12BCCF26B2ACCF2D62CC4F259
:108550001720C3F6106BC3F8F0A3C3F8F8C3C3F831
:10856000FC03C9F804B04FF4006C46F6CD404AF65F
:10857000C5734FF6DB4BC4F2BD5CC4F28E50C3F63C
:108580007523C3F63F5BC9F808C0C9F80C00C9F8E9
:108590001030C9F814B046F6903C45F610004DF284
:1085A000D13341F61F1BC3F63F2CC4F28220C3F225
:1085B0009343C3F25E5BC9F818C0C9F81C00C9F840
:1085C0002030C9F824B04BF2600A40F6652C4FF613
:1085D0004F604FF406434CF6303BC3F69B5AC3F64C
:1085E0007E0CC3F6D500C3F28A33C3F2EB3BC9F865
:1085F00000A0C9F828C0C9F82C004EF6745CC9F870
:1086000030304EF27800C9F834B04CF6A9634DF61C
:10861000525BC3F2B81CC3F29640C3F29373C3F625
:10862000460BC9F838C0C9F83C00C9F84030C9F851
:1086300044B048F6C35C4AF2A40047F2EE6341F648
:10864000EF4BC3F6A00CC3F62100C3F63D53C3F6AF
:108650004A4BC9F848C0C9F84C00C9F85030C9F8AD
:1086600054B040F64A4C4CF2FC404DF6556343F290
:10867000FE5BC4F2720CC3F68140C3F62E63C3F6F0
:10868000C80BC9F858C0C9F85C00C9F86030C9F80F
:1086900064B043F63A3C09F1680B4BF2957049F22D
:1086A0006663C3F6994CC3F6C360C4F20053CBF8BB
:1086B00000C0CBF80400C9F870304FF4194C09F130
:1086C000780341F2A930C3F65040CCF2CA7CCBF813
:1086D0000CC01863586340F2DE5C0020C3F6CA4C3D
:1086E000CCF22010A9F1080AC9F88410C9F8881042
:1086F000C9F88C10C9F8B0C0C9F8B400C9F878201E
:10870000C9F87C20C9F88020C9F89420C9F89820BD
:10871000C9F89C20C9F8A020C9F8A420002309F1B9
:10872000B8094EF68530CCF2C813C4F26910CBF804
:108730002820C9F80030C9F80C00CBF86010CBF83D
:10874000641000234CF6CD4100204FF0814CCCF258
:108750002013C4F29411C4F27A40C9F818C0C9F8C1
:108760002030C9F82410C9F8280009F1280109F1BE
:1087700020004FF4404C4FF40053C4F2F34CC4F2C9
:10878000CB53C9F80420CAF8C820CBF86C40C9F80C
:108790002CC0C9F83820C9F84020C9F84420CAF8CC
:1087A0000821C9F84C20CBF8A020CBF8A420C9F8A8
:1087B0005820CBF8AC20C9F86820C9F87020C9F857
:1087C0007420CAF83821C9F87C20CBF8D020CBF827
:1087D000D4208B60CA604A618A63CA634A64C9F85C
:1087E0008820CBF8DC20C9F89820C9F8A020C9F867
:1087F000A420CAF86821C9F8AC20CBF80021CBF836
:108800000421C9F8B820CBF80C21C9F8C820C9F850
:10881000D020C9F8D420CAF89821C9F8DC20CBF8B8
:108820003021CBF834218A66CA664A67C1F898209D
:10883000C1F89C20C1F8A4200AF5CC7A09F1D0092E
:108840000BF5987BC0F8C820BDE8F00F704700BF5B
:10885000BC06001008B503F04FFD014640F2B420FD
:10886000C1F2000040F2AC52BDE8084015F02EB84D
:1088700008B503F041FD40F2B421C1F2000140F21D
:10888000AC5203F07DFCC0B208BD00BF2DE9F04F33
:108890008BB0002800F0A28003F02AF90028039092
:1088A0000290C0F2A08001214FF400700FF038FF59
:1088B0000121019080200FF033FF40F2000440F2CC
:1088C000B42582460027C2F20004C1F200050298D6
:1088D00001994FF0FF324FF4007303F07BF9002849
:1088E000834661DD002604E00AF8073001375E4563
:1088F000EDD0019A935D01360A2B01D07F2FF3D181
:108900004FF2B8514FF00008C0F601010AF8078095
:10891000504605AA09AB14F097FF022817D04FF272
:10892000D851C0F60101504605AA09AB14F08CFFDE
:1089300002280CD04FF2D051C0F60101504605AAD2
:1089400009AB14F081FF022801D04746CFE700278A
:108950003959102205A814F08BFF034607F10408CB
:10896000102205A8EF190BB90999396058F80410BD
:1089700014F07EFF18B905EB08070998386008F174
:10898000040905A859F80410102214F071FF08F129
:108990000807A94410B9099AC9F8002040F2AC5C54
:1089A0006745D5D10027A2E7039803F037F9BAF15C
:1089B000000F04D05046802101220FF0D3FE019B0E
:1089C0002BB118464FF4007101220FF0CBFE5FFA75
:1089D0008BFB4FFA8BF00BB0BDE8F08F4FF2845059
:1089E000C0F6010058E74FF29050C0F60100F9F7C9
:1089F000AFFF4FF0FF0BECE710B52DED028BFFF74B
:108A000029FF0020FFF742FF002842DB0EF0D0FDD7
:108A100003F072FC90ED008AB0EE480A13F07EFA83
:108A2000C8B9DFED257AB4EEE78AF1EE10FA14D476
:108A300040F2B423C1F20003D3ED007AB4EEE78A2A
:108A4000F1EE10FA2FDAB4EEE78AF1EE10FA1AD44A
:108A5000BDEC028B10BD9FED198A40F2B424C1F227
:108A60000004D4ED007A9FED147AF4EEC77AF1EEAB
:108A700010FAE3D5FFF73EFAD4ED007AB4EEE78AB8
:108A8000F1EE10FAE4D5BDEC028BBDE81040FFF723
:108A9000EFBE40F2B420002140F2AC52C1F200001F
:108AA00014F032FFB4E7FFF7D5FE40F2B420C1F274
:108AB0000000D0ED007AC6E70000CE4200000000C2
:108AC0002DE9F04FA5B0002871D003F011F800286F
:108AD0000390804670DB40F20003C2F200034FF2C5
:108AE00008663A4D1C1FC0F601064FF0FF3935E00D
:108AF0005868576812F034FE3A4682468B4604A8FE
:108B00003146CDE900AB14F089FE074604A9404682
:108B10004A463B4603F070F841B28F4237DC55F8C5
:108B20000C0F54F80C7F12F01BFE3A4682468B461F
:108B300004A83146CDE900AB14F070FE07463B4671
:108B4000404604A94A4603F057F85FFA80FA4FFA04
:108B50008AF39F421BDC1E4A944220D068686768F3
:108B600012F0FEFD3A4682468B4604A83146CDE916
:108B700000AB14F053FE07464A463B46404604A964
:108B800003F03AF840B2221D2B1D8742B0DD4FF2B0
:108B90001860C0F60100F9F7DBFE4FF0FF0A0398FA
:108BA00003F03CF84FFA8AF025B0BDE8F08F4FF2A1
:108BB0008450C0F6010088E74FF2E050C0F6010093
:108BC000F9F7C6FE4FF0FF0AECE700BFB002001055
:108BD000A80500202DE9F84340F68C4040F66004DB
:108BE00041F628752DED068BC0F60200C1F2000497
:108BF000C2F20005F9F7ACFE04F1240705F5826620
:108C0000ADE140F2B429C1F20009D9ED020ABDEE8E
:108C1000E00A41F6380810EE103AC1F20008181DBB
:108C2000D9ED187A38F9101006EE901AB8EEE67AF7
:108C3000B4EEE77AF1EE10FA08DC41F2D81CC1F28A
:108C4000000C9CF83805002800F0558201200EF039
:108C50008DFC41F2D813C1F2000393F83825002AA5
:108C600040F0F28140F2B42EC1F2000E9EED024AB5
:108C7000FDEEC43A41F6380813EE901AC1F200082E
:108C80000B1DDEED182A38F9130003EE100AB8EEBA
:108C9000C32ADEED127A72EE621A21EEA70ADFED28
:108CA000F38A27EEA86ABDEEC08AFDEEC65A18EE1A
:108CB000100A012115EE902A41F220190FF0FEFD55
:108CC000C1F200099FEDEA8AD9ED274A05EE100AA4
:108CD000F4EE484AF1EE10FAB8EEC5AA00F0688149
:108CE00040F2B423C1F20003D3ED05AAFDEEEA9AE7
:108CF00041F6380919EE900AC1F20009021DD3EDC0
:108D0000167A39F9121009EE101AB8EEC98AB4EEC3
:108D1000E78AF1EE10FA40F3368178EE677AD3ED08
:108D2000156A27EEA68A41F2D818C1F20008D8EDDC
:108D3000031A05F5806CDCED010A38EE210AFFF715
:108D4000AFF814F09FFB9FEDCB1AB4EEC10AF1EE21
:108D500010FA00F1D581D8ED030A40F2B42894ED61
:108D6000080AC1F20008FFF79BF8D8ED1A3A9FED08
:108D7000C24AF1EE634AC4EE840A83EE841A0FF00D
:108D8000A5FD94ED083A30EE030AFFF765F841F2CD
:108D9000D811C1F2000184ED080A91F83825032AA0
:108DA00000F0A18198ED040AD8ED037AFDEEC06AC7
:108DB000BDEEE77A16EE903A17EE100A41F6380942
:108DC000191DC1F20009031D39F911E039F9130029
:108DD0000AEE90EA09EE900AB8EEEA6A98ED139A64
:108DE000F8EEE98A98ED148A66EE095A28EE885A58
:108DF000012AC4ED025A84ED035A40F2788141F20F
:108E0000D818C1F20008D8F82800D8F82C10206132
:108E10006161384694ED020A0FF02EFE04F13C0029
:108E200084ED020A94ED030A0FF026FE04F15400CB
:108E300084ED030A94ED040A0FF01EFE04F16C00A9
:108E400084ED040A94ED050A0FF016FED4ED043A01
:108E500096ED014A96ED003A20EE042A23EE841A9C
:108E600013EE832A00EE031A40F2B42CC1F2000C78
:108E7000D4ED022AD4ED031ADCED116A9FED7C8A51
:108E800072EE227A71EE810AF4EE486AF1EE10FA7F
:108E900084ED050AC4ED067AC4ED070A00F0EE8001
:108EA000F7EE004AF4EE646AF1EE10FA00F03B814E
:108EB000B0EE489A05F5806EDEED010A94ED080AE1
:108EC000D4F89880D4F88C90FEF7EAFF4046F0EE94
:108ED000400A9FED670A08F02DFE40F22010C1F213
:108EE000000040F2B428D0F82831484600EE903A0D
:108EF00008F020FEC1F2000898ED191AF0EE409A31
:108F0000F1EE410AB0EE480A0FF0E0FC98ED191AB4
:108F1000F0EE40AAF1EE410AB0EE490A0FF0D6FC9D
:108F200098ED191AB0EE408AF1EE410AB0EE690AE6
:108F30000FF0CCFCF0EE480AF0EE401AB0EE6A1AE0
:108F4000B0EE4A0A04F0C2FE40F2201CC1F2000C4E
:108F50006068DCF88021411CC4F89C20616041F20B
:108F60000812C1F200020021107802F05FFF41F602
:108F70009420C1F2000090F8BC319B073FF541AE50
:108F800004F0E6FDE0E7B1EE677AB4EEC78AF1EEF1
:108F900010FA06D441F2D813C1F20003D3ED030A4C
:108FA000DBE638EE270AD3ED150A20EE208ABAE672
:108FB00005F5806E41F2D818DEF804C0D4F88800B8
:108FC000C4F820C0C1F20008B0EE480AC8F80CC0CE
:108FD000F0EE480A08F094FED4F88400B0EE480A97
:108FE000F0EE480A08F08CFED4F88C00B0EE480A87
:108FF000F0EE480A08F084FED4F89400B0EE480A77
:10900000F0EE480A08F07CFED4F89000B0EE480A72
:10901000F0EE480A08F074FED4F89800B0EE480A62
:10902000F0EE480A08F06CFE98F83825022A7FF422
:1090300057AE41F26000C1F2000090ED0E0B90EDD2
:10904000101B07F0ADFA4BE6D5F83C24986C92ED76
:10905000021A93ED0C0AF1EE410A08F06BFD40F2A2
:10906000B421C1F20001D1ED127A18E60000AF443C
:1090700000000000000034420000C84305F5816E86
:1090800040F22019DEED000AB0EE670AD4F8940031
:10909000C1F2000908F04EFDD9F82431D4F8880057
:1090A00000EE903AB0EE409AB0EE480A08F042FD69
:1090B00005F58061D1ED030AD4F8900030EE099AED
:1090C00094ED070A08F036FDD9F82021D4F8840081
:1090D000F0EE408A00EE902AB0EE480A08F02AFD31
:1090E00030EE288AE6E60022A260E26087E60023EE
:1090F000236163618DE60EF039FA04F029FD23E760
:10910000D4ED082A38EE220AFEF7A6FE98ED032ACF
:1091100084ED080A38EE020AFEF79EFEF0EE400AE1
:1091200088ED030A19E640F2201805F58161C1F2C5
:109130000008D1ED000AB0EE670AD4F89400D4F824
:10914000889008F0F7FCD8F82421484600EE902AD1
:1091500008F0F0FC05F5806CDCED030AD4F8900013
:10916000D4F88490B0EE409A94ED070A08F0E2FC3F
:10917000D8F8200100EE900A484608F0DBFCB0EE7B
:10918000408A97E62DE9F04F2DED048B40F6A44080
:109190008BB040F66004C1F200049FED8F8ADFEDD2
:1091A0008F8AC0F602009FED8E9A0994F9F7D0FBE2
:1091B0000021A0220998DFF82CB214F0A5FB04F1DD
:1091C0002400B0EE480AF0EE490AB0EE681A0FF03B
:1091D00043FC04F13C00B0EE480AF0EE490AB0EE60
:1091E000681A0FF039FC04F15400B0EE480AF4EEAE
:1091F000000AB0EE681A0FF02FFC4FF0000AB0EE34
:10920000480AF4EE000AB0EE681A04F16C000BF1A3
:1092100004070BF108060BF10C05CDF820A00FF0A8
:109220001BFCDDF820C00BF110040BF114080BF14E
:1092300018090BF11C0A394632462B4658468DE870
:109240001007CDF810C0CDF814C0CDF818C0CDF877
:109250001CC008F051FC3946099F8446C7F888C0F5
:109260008DE81007DDF8209032462B465846CDF8A1
:109270001090CDF81490CDF81890CDF81C9008F00F
:109280003BFCDDF824E0DDF820C004460BF12000B3
:10929000CEF8844000F11004009400F1140401940D
:1092A00004340BF124010BF128020BF12C0302947E
:1092B00004340394CDF810C0CDF814C0CDF818C014
:1092C000CDF81CC008F018FC04F10801099CDDF879
:1092D00020C00BF1400786460BF148050BF14C0608
:1092E000C4F88CE00BF1500807F11C042A46334601
:1092F0000BF154090BF1580A3846CDF810C0CDF8DF
:1093000014C0CDF818C0CDF81CC08DE80007039438
:1093100008F0F2FB3346099E8646C6F894E08DE8D5
:109320000007DDF8208003942A460BF144013846FB
:10933000CDF81080CDF81480CDF81880CDF81C80C1
:1093400008F0DAFBDDF82480DDF820E00646C8F8F6
:1093500090600BF1780C0BF168020BF164010BF1DA
:109360006C030BF170050BF174040BF160000BF151
:109370007C07CDF808C0CDF810E0CDF814E0CDF8AA
:1093800018E0CDF81CE000950194039708F0B4FBB9
:1093900040F6B4410346C0F60201C8F89830962062
:1093A0000FF012FA40F64064DDF820C0C2F200046B
:1093B000054648F6D530C0F6000005F51573614640
:1093C00049F2056225600EF0C7FB88F800000BB07B
:1093D000BDEC048BBDE8F08F0AD7233B00000000F2
:1093E000CDCCCC3D2003001040F64460C2F200001A
:1093F00008F0A0BC10B540F64464C2F20004204658
:1094000008F0A6FC237833B940F64661C2F20001A9
:109410000878012800D010BD40F64564C2F200046F
:1094200023785A1CD1B221700EF030FB2078431EF5
:10943000DAB2227010BD00BF08B540F64563C2F233
:1094400000031A78012A04D01A78511EC8B2187085
:1094500008BD42F23840C2F200000378012B11D05F
:1094600040F6466CC2F2000C9CF80010012906D0B0
:1094700040F64563C2F2000300221A7008BD0EF0E8
:1094800005FBF5E70CF07CF9EAE700BF4EF21401AA
:109490004EF2100C10B5CEF20001CEF2000C49F2E3
:1094A0003F034EF61C5ECEF2000E0724C0F202030C
:1094B0000B60CCF80040DEF80020174C4EF6205C24
:1094C000CEF2000C42F07F40CEF80000DCF8001035
:1094D0006FEA01436FEA1340CCF800000EF04EF93A
:1094E00000F05EF803F026FC40F64563C2F200038C
:1094F0004DF27D501A78511CCAB21A70002144F204
:1095000040022346C0F600000EF026FB2046BDE8D0
:10951000104008F02DBC00BFC827002042F2704266
:1095200042F2744042F2CC71C2F20000C2F2000278
:10953000C2F2000108B501231060086043710EF00B
:10954000EDF9BDE80840FFF777BF00BF70B50E46E4
:1095500082B00546082101200FF014F905608680CD
:1095600004466E83684610F0BBFF022000238DF88E
:10957000050001222846694600968DF806308DF8D0
:1095800004208DF8073010F0EFFE204602B070BDC9
:109590000368828859690A4214BF5A831A83704744
:1095A00010B4214B13F80B2C43F8103C0424002179
:1095B00064F3030203F80C1C03F80B2C0121103395
:1095C00013F80BCC03F80C1C481CC0B264F3030C5A
:1095D00003F1100243F8103C03F80BCC411C5B79FB
:1095E00042F8102CC9B264F30303132902F80B3CB0
:1095F00002F80C0C02F11003E2D140F64C63C2F207
:10960000000340F6486293F8350183F83411C2F242
:10961000000264F30300002183F83501C3F8301120
:10962000136010BC704700BF5C0E00202DE9F843AA
:1096300040F64563C2F2000340F648651C78C2F26A
:109640000005661C2C68F6B20746884691461E70D7
:1096500084B122682A60FFF7EFFE6179C4F80090B8
:1096600067F3030168F3071100206171E060204691
:10967000BDE8F883FFF7E0FEF9E700BF30B440F63D
:10968000456CC2F2000C04799CF80030C2680C7280
:109690005D1CEDB28CF80050437903F0F003102B01
:1096A00027D0202B0BD040F6466CC2F2000C0223D0
:1096B00001204B718CF8000030BCFFF7BDBE002AC2
:1096C0002AD00C7992F804C0A4451BD8106958B16F
:1096D0000379A34204D921E01A79A24216D8184688
:1096E0000369002BF8D1024611614A6100220A6128
:1096F000D9E70AB910E01A461369002BFBD11161B2
:109700004A61D0E7C1600A615161CCE7024611614C
:109710004A610B615961C6E7C160C4E70346F6E7D9
:1097200038B5C4680546002C22D02369C3600BB14C
:1097300000225A61E3690021FF2001332161207278
:1097400002D020460EF002FB6A7902F00F03022BD2
:109750000FD0032B1FD042F2704CC2F2000CDCF889
:1097600000309C4214D02046BDE838400EF098B836
:1097700038BDEA88296842F2704CC2F2000C531ED0
:10978000E160EB80DCF8003000209C422860EAD1E8
:109790000120607138BD2B68DA881D68988955F8FA
:1097A0002250B3F80AC0E560013291B201388C450D
:1097B000D9809881CFD10021D980CCE7027A016984
:1097C00040F64C63C2F2000303EB0213426949B155
:1097D00072B11161016900234A6103614361FF2293
:1097E0000272704742B11161FF22416102727047FB
:1097F0004A61D9600261F2E7DA60F0E72DE9F843E7
:10980000C56A8D4204460E4650D003797BB916B91D
:109810003046BDE8F883607804F130013246012318
:109820000BF0FEF800283BD1E662BDE8F88304F1B6
:109830003007407839462A4601230BF059F90028B1
:1098400031D1E369216A20715A189542DFD294F828
:109850000380B8F1010FDAD918F0010F4FF00109B8
:1098600001D10CE0E369ED1860784B4639462A4691
:109870000BF03EF908F1FF335FFA83F8E369ED1866
:10988000607839462A464B460BF032F908F1FF3032
:109890005FFA80F8B8F1010FE4D1002EB8D0BAE732
:1098A0000120BDE8F8830120BDE8F8830020BDE871
:1098B000F88300BF08B508B103780BB9092008BDCB
:1098C000C2888A4201D0092008BD40780BF094F884
:1098D00010F0010018BF032008BD00BF38B50446D2
:1098E0000A46407804F1300101230BF099F808B1E1
:1098F000032038BD94F82F2294F82EC24AF655233F
:109900004CEA02210AB2CFF6FF739A4201D002203C
:1099100038BD94F8682094F8695094F8661094F86B
:1099200067C0130443EA056242EA010343EA0C2ECE
:1099300044F246132EF07F41C0F254039942E7D01F
:1099400094F8842094F8855094F8820094F883E089
:10995000110441EA056242EA000C4CEA0E2121F0B2
:109960007F40C01A18BF012038BD00BF2DE9F0416B
:1099700003681C78303C092C154615D940F69070C8
:10998000C2F2000004680C6014B32178B1B16078B1
:109990000BF032F8C10711D4002D22D010F00400D2
:1099A00018BF0A20BDE8F0815A783A2AE6D102337E
:1099B0000360002CE2D00B20BDE8F0810020207075
:1099C00060700BF003F8C20705D50320BDE8F081F5
:1099D0000C20BDE8F0813DB1430705D50A20BDE864
:1099E000F0812846BDE8F08100212046FFF776FF90
:1099F000012807D00026032800F0C080D0B10D2038
:109A0000BDE8F08194F8F221002AF8D094F8F8210A
:109A100094F8F91194F8F6E194F8F761100440EA2B
:109A2000016343EA0E0C4CEA062620463146FFF756
:109A300055FFE0E794F83C3094F83BE04EEA032C05
:109A4000BCF5007FDBD194F8470094F8461051EA4A
:109A500000210ED194F8562094F8570094F854E061
:109A600094F855C0110441EA006343EA0E0242EA49
:109A70000C2194F84000E161431E5FFA83FCBCF1C5
:109A8000010FE070BBD894F83D20A270002AB6D038
:109A9000531E1342B3D194F8425094F841E04EEA79
:109AA000052313F00F0F2381A9D194F8447094F883
:109AB000435055EA07250FD194F8527094F853801B
:109AC00094F8505094F851E04FEA074747EA086786
:109AD00047EA050C4CEA0E2594F83F7094F83EE0F6
:109AE0005EEA07278BD000FB01FC07EB13106044F4
:109AF000854284D32D1AB5FBF2F2002A3FF47FAFE2
:109B000040F6F575AA4240F2B18005F57045AA42CB
:109B100000F2A280022502328019F719A261A06228
:109B20002762002B3FF46BAF6744022D676200F0A1
:109B30009180032505FB02F002F0010202EB5002C6
:109B4000012502F5FE72D31CB1EB532FFFF457AF82
:109B500000234FF0FF31032D2161E36011D04E4A05
:109B600025701088431C1FFA83FC0020A2F800C057
:109B7000A4F806C0E0622071BDE8F0810120BDE8D4
:109B8000F08194F8612094F860E063714EEA02235A
:109B9000F2186078626104F1300101230AF040FF9D
:109BA0000028DCD194F82F2294F82E324AF6552C56
:109BB00043EA022108B2CFF6FF7C6045CFD194F88A
:109BC000323094F8330094F830E094F831C01A043D
:109BD00042EA006141EA0E0345F2522E43EA0C20AC
:109BE000C4F2611E7045BAD194F8162294F8170297
:109BF00094F8143294F815E2110441EA006242EA42
:109C0000030C47F272204CEA0E21C6F24110814249
:109C1000A5D194F81E7294F81A6294F81B1294F865
:109C20001F8294F8183294F81C2294F81D0294F8BC
:109C300019E23F04360446EA016647EA086747EA44
:109C4000020146EA030C41EA00204CEA0E23E060E0
:109C5000236184E7520074E702328019F719A26188
:109C6000A062276223B10D20BDE8F081012552E7F3
:109C700094F85E3094F85F7094F85C0094F85DC0DE
:109C80001D0445EA076343EA000545EA0C236362C5
:109C90009200032555E700BF8C0F00200129F8B57D
:109CA0000C46054630D98369994209D20378022BC4
:109CB00048D0032B2AD0012B04D04FF0FF30F8BD41
:109CC0000120F8BD016A04EB540601EB5621FFF7B1
:109CD00095FD0028F1D1F305286ADF0D0136EA1958
:109CE00000EB5621284692F83070FFF787FD0028D8
:109CF000E3D1F605F60DAD19E30795F8301047EA04
:109D0000012031D50009F8BD0120F8BD036A03EB3D
:109D1000D111FFF773FD0028CFD1640605EBD455B0
:109D200095F8320095F8332095F830C095F831E079
:109D3000030443EA026141EA0C0040EA0E2222F0E9
:109D40007040F8BD006A00EB11212846FFF756FD70
:109D50000028B2D1240605EBD45595F8311095F8BA
:109D600030C04CEA0120F8BD0205100DF8BD00BF5F
:109D700081680023012910B50446C38003D0006820
:109D80008369994201D3022010BD81B90278032A68
:109D90000AD001890023E3600029F4D0426A2261DD
:109DA00030306061002010BD416A0029F1D0827816
:109DB00032B10CE00128E6D920688369994212D2B9
:109DC000FFF76CFF421C0146F4D1012010BD8A1E32
:109DD000023B9A42E1603DBF8178836A01FB023217
:109DE00000222261DCE7022010BD00BF70B501290E
:109DF00082B00C46054602D98369994202D30220FB
:109E000002B070BD0378022B28D0032B05D0012BA4
:109E10003AD0022001222A71F2E7036A019203EB91
:109E2000D111FFF7EBFC019A0028F3D1640605EB92
:109E3000D45494F833100B0603F070463243C2F347
:109E40000726110C130E84F83020012284F83160AB
:109E500084F8321084F833302A71D1E7006A019215
:109E600000EB11212846FFF7C9FC019A0028D1D147
:109E7000240605EBD454C2F3072184F830200122D4
:109E800084F831102A71BBE7016A019204EB540691
:109E900001EB5621FFF7B2FC019A0028BAD1F00578
:109EA000C30D14F0010425D0E9185FFA82FC91F883
:109EB00030E00EF00F0040EA0C11C8B2296A05EB41
:109EC000030C013601238CF830002B7101EB562175
:109ED00028460192FFF792FC019A00289AD1F605D4
:109EE000F60D4CB1C2F30712AE1986F830200122EC
:109EF0002A7185E7D0B2E1E705EB060CC2F3032235
:109F00009CF8303023F00F0E4EEA0202ECE700BF5F
:109F10002DE9F0410E460546002926D1C768836920
:109F2000DFB19F4228BF01273C4601349C424FF0DD
:109F3000020802D3012F15D9444628462146FFF7CF
:109F4000ADFED8B1431C0BD0012809D0BC4209D0CA
:109F5000AB6901349C42EDD2EFE70127E4E72046EC
:109F6000BDE8F0810020BDE8F081FFF797FE0128F1
:109F700018D9AB699842F3D33746D5E7284621462E
:109F80006FF07042FFF732FF2746A8B96EB92B6910
:109F9000EF60591CE3D0581E012328616B712046E5
:109FA000BDE8F0810120BDE8F08128463146224617
:109FB000FFF71CFF0028EAD0012814BF01204FF052
:109FC000FF30BDE8F08100BF2DE9F8430446C088AA
:109FD000451CADB20E4615B90420BDE8F8832369CF
:109FE000002BF9D028070AD02068303005F00F0286
:109FF00000EB42106061E5800020BDE8F883E16875
:10A00000206801332361C9B183785A1E12EA1513FF
:10A01000EBD1FFF743FE0128074613D9411C5ED060
:10A02000206881698F424DD3002ED5D0E168FFF7BB
:10A030006FFF074648B90720BDE8F8830189A942A8
:10A04000CAD9D2E70220BDE8F8830128FAD0421C21
:10A0500045D020680021FFF7D1FB00283FD12668BA
:10A06000024606F1300306F50C70194601F8012B83
:10A070005A704B1C8342F8D123689E69B91EB01EEA
:10A08000814204D293F802809A6A08FB01220026DA
:10A09000DA624FF00108B1460CE080F804802068D5
:10A0A0004946FFF7ABFB0136E0B92368D96A4A1C81
:10A0B000DA62F6B2206890F802C0B445EDD8C36AFF
:10A0C0009E1BC6628369E760991E023F8F423DBFB7
:10A0D0008278816A02FB07110021216185E7012056
:10A0E000BDE8F8834046BDE8F88300BF2DE9F84F8E
:10A0F0000B782F2B0D46044600F00C815C2B00F0F2
:10A1000009810026A6602B781F2B40F20A8140F6B9
:10A11000D44640F60C5BA369C0F6020BC0F60206FB
:10A1200020224FF000081A705A709A70DA701A7173
:10A130005A719A71DA711A725A729A7247464FF0CE
:10A140000809C246A446E95D0137202923D92F29F1
:10A1500048D05C2946D02E2927D0C84525D20806EC
:10A160003AD422290C461DD0304601E0944219D041
:10A1700010F8012F002AF9D1A1F14100C2B2192A29
:10A1800020D84AF0020A03F80810E95D01372029B7
:10A1900008F10108DBD86446ED1951460422B8F1F4
:10A1A000000F26D10620BDE8F88FB9F1080FF9D1CC
:10A1B0002E29F7D14FEA8A00C8465FFA80FA4FF09D
:10A1C0000B09C0E7A1F16100C2B2192ADBD820391E
:10A1D0004AF0010AC9B2D6E780394AF0030A1BF8EF
:10A1E0000110BEE76446ED1951460022B8F1000F98
:10A1F000D8D01F78E52F00F09D80B9F1080F00F04E
:10A200009E800AF00307012F0AF00C0A08BF42F0F3
:10A210001002BAF1040F08BF42F00802DA722046B9
:10A22000FFF7A6FD0746002F65D120682169FFF7DB
:10A23000E5FA00285FD162691178002961D092F8AF
:10A240000BC01CF0080F50D1A36993F8008088451B
:10A250004BD192F8018093F801E0F04545D192F896
:10A2600002809978884540D192F8038093F803E002
:10A27000F0453AD192F804801979884535D192F8A1
:10A28000058093F805E0F0452FD192F80680997982
:10A2900088452AD192F8078093F807E0F04524D149
:10A2A00092F80880197A88451FD192F8098093F8AE
:10A2B00009E0F04519D193F80A80917A884514D1C4
:10A2C00093F80BE05FEA4E7137D41CF0100F2ED0DC
:10A2D000517D177D92F81B90927E47EA012842EA51
:10A2E000092040EA0842A2601AE720463946FFF7F3
:10A2F0006BFE002899D0A3690428DB7A03D0BDE85F
:10A30000F88FA369DB7A13F0040F0CBF052004203B
:10A31000BDE8F88F01350026A6602B781F2B3FF68D
:10A32000F6AE2046FFF724FD6661BDE8F88F0520F4
:10A33000BDE8F88F052018705FE7BDE8F88F890049
:10A340005FFA81FA5DE700BF08B10B20704740F665
:10A350009073C2F200031B6803B1187009B10020AA
:10A36000087040F69072C2F200020020116070473F
:10A370002DE9F04F8DB00CAB02F01F0643F82C1DF9
:10A380000021016006F01E02054602A91846FFF7EB
:10A39000EDFA09AA03460892B8B1079C16F01C0F03
:10A3A000324607D06BB1042B00F0BF8018460DB0C9
:10A3B000BDE8F08F002BF9D1E37AD9063DD504230F
:10A3C000F4E773070DD50823F0E702A80199FFF71A
:10A3D0008DFE079C03460028E0D1002C08BF062311
:10A3E000DCE7E17A11F0110F2BD1170733D4029F6C
:10A3F000F86AAE71E8612C62667D217D94F81BC01D
:10A40000A37EB7F806E043EA0C2041EA062240EAC0
:10A4100002462E61A17FE67F237F607F2F600A04C2
:10A4200042EA066141EA030C4CEA00220023EA609A
:10A43000AB60AB61A5F804E0B8E7B20703D5DB0772
:10A4400001D50723B2E706F00803029F002BCFD007
:10A4500046F02006CCE70AF0B7FA94F8159094F885
:10A46000148094F81BC0A17EA073030CC0F30722D4
:10A47000029FE273000E48EA092841EA0C214FF0DE
:10A48000000A6074012051EA0849237484F80BA083
:10A4900084F81CA084F81DA084F81EA084F81FA0D6
:10A4A00084F81AA084F81BA084F814A084F815A0DE
:10A4B0003871CDD0F86AB9F1010F009053D0BB6963
:10A4C000994550D2CB4600E0C34659463846FFF77F
:10A4D000E5FB8046594638465246B8F1000F15D084
:10A4E000B8F1010F3FD0B8F1FF3F70D0FFF77EFC0D
:10A4F000034600287FF45AAF3B69581C03D0591C0F
:10A50000012239617A71B8698045DDD302980099DA
:10A5100009F1FF32C260FFF771F9034600287FF4AA
:10A5200045AF029F46F0200662E702AF3846FFF7CC
:10A530001FFC034600287FF439AF012406990298D6
:10A54000FFF75CF9034621463846002B7FF42EAF17
:10A55000079A1378E52B08D03BB1FFF735FD03468A
:10A560000028EBD022E7022320E702980699FFF7A4
:10A5700045F9034600287FF419AF079C04F1200138
:10A5800023461F4607F8010B58707B1C8B42F8D1FD
:10A5900008990F7827704A7862708B78A370C87812
:10A5A000E0700F7927714A7962718B79A371C8794C
:10A5B000E0710F7A27724A7A62728B7AA372029CD8
:10A5C000012046F008062071079C32460DE7012362
:10A5D000ECE600BF2DE9F04F04461F46A388006853
:10A5E00088460021396083B019469146FFF762F929
:10A5F000064628B9A3791A0606D4DB0706D407262F
:10A60000304603B0BDE8F08F0226F9E7A368E5689D
:10A61000ED1AA94538BF4D46002DF1D004F12402B2
:10A6200001928246D805C10D00292CD1226892F8EA
:10A6300002B00BF1FF3101EA53265FFA86FBBBF152
:10A64000000F5BD0606996690238B31E984263D3ED
:10A65000A07960F07F02A2710226D1E7A1794906B4
:10A6600000F19980A269B24209D02068019940782E
:10A67000324601230AF0D4F9002840F08180A36813
:10A68000A661D905C90DC1F50079A94528BFA9461C
:10A69000B9F1000F26D02031611809F1FF3C91F883
:10A6A00004E0434662464E1D0CF0010C03F801EB3A
:10A6B000BAB1BCF1000F06D091F805E08E1D013A49
:10A6C00003F801EB0DD03046194610F801CB01F824
:10A6D00001CB96F801E0461C83F801E04B1C023ADE
:10A6E000F1D1A3683E684B4406EB0902B5EB0905BE
:10A6F000A360C8443A6095D1564681E7002B45D106
:10A7000020690128A4D9461C3AD022686061966964
:10A710000238B31E98429BD29378916A03FB0016CD
:10A72000002E95D05FEA55295E4497D00BEB090CBB
:10A730009C4588BFCBEB030950785FFA89F341460B
:10A7400032460AF06DF9A379D8B9580614D5A36931
:10A750009B1B994510D908EB432304F1230103F512
:10A76000007691F801E01A4602F801EB88785870FB
:10A77000531C0231B342F4D14FEA4929A368B1E72F
:10A78000A37963F07F06A671012639E76169104657
:10A79000FFF784FAB5E750780199A26901230AF01E
:10A7A000A7F9A3790028ECD123F04003A37159E75E
:10A7B0002DE9F04F04461F46A38800688B46002110
:10A7C000396083B019461546FFF774F8064628B974
:10A7D000A379190606D49A0706D40726304603B093
:10A7E000BDE8F08F0226F9E7E268A368D54207D3F7
:10A7F0009A42A27938BFE36042F02003A371EDE7EB
:10A80000002DF5D004F12400009004F5097801969C
:10A81000DA05D10D002932D122689078411E01EA73
:10A820005326F6B26EB9002B40F0C2802069002892
:10A8300000F0C980012810D0431C00F0B3802268CA
:10A84000606194F806C05FEA4C6100F19E80616926
:10A8500093690239981E81424DD3A67966F07F0232
:10A86000A2710226BAE7A069A368484503D0E6684A
:10A87000B342C0F0B180D905C4F81890C90DC1F534
:10A88000007AAA4528BFAA46BAF1000F22D05B463B
:10A89000203161180AF1FF3C13F8016B62460E711A
:10A8A0000CF001004E1DA2B128B113F8010B8E1D52
:10A8B000013A48710DD01846314610F801CB01F825
:10A8C00001CB93F801E0431C86F801E04E1C023AEC
:10A8D000F1D1A368A67946F04002A27138685344CA
:10A8E00000EB0A01B5EB0A05A360D34439608FD1B0
:10A8F000019EE2687CE79378906A01FB03010029DE
:10A90000ABD05FEA552A06EB0109ACD006EB0A0E84
:10A910009E4588BFC6EB030A50785FFA8AF3594612
:10A920004A460AF0E5F800283CD1A369C9EB0309BF
:10A93000CA4526D94FEA492C009B1BF80C00DA4384
:10A9400003F8010B08EB0201434501F001020BEB98
:10A950000C0112D032B111F8010F009E01334345B2
:10A9600070700AD091F801E01E4606F801EB8A7873
:10A970005A70731C02314345F4D1A17921F0400390
:10A98000A3714FEA4A2AA368A8E750780099A26900
:10A9900001230AF0ADF8A37928B923F04003226817
:10A9A000A37154E7A37963F07F02A271012615E732
:10A9B00061691046FFF7ACFA00287FF43BAF019EB7
:10A9C000A368E26814E710463146FFF7A1FA206158
:10A9D00000287FF42FAFF2E7507800994A46012310
:10A9E0000AF01EF80028DDD1A36844E72DE9F04FF6
:10A9F000044683B00068A188FEF75CFFC0B9A37964
:10AA00009A0615D558060DD52146A26951F8243B62
:10AA1000587801230AF06CF800284BD1A17921F075
:10AA20004000A0712068E169FEF7E8FE064616B115
:10AA300003B0BDE8F08F256AE87A40F02001E972A2
:10AA4000E2682A77A389180A6877E189A977E27B07
:10AA5000EA772369AB76208A010AE976628A2A7549
:10AA6000638A180A687509F0AFFFC0F30721020C6A
:10AA7000030EE9752A766B76A875A079256820F013
:10AA800020030122A3712A71256831462846FEF76A
:10AA9000B5FE0446002CCBD195F800C0BCF1030FE5
:10AAA0000AD0002168780A460AF08AF8003018BFF8
:10AAB0000120BDE70120BBE76B79002BF1D005F148
:10AAC0003001EC6205F50C700B461E4606F8014B92
:10AAD0005C70731C8342F8D1EB68D5F8108085F860
:10AAE0001C324FEA134BCDF800B04FEA136B6122D2
:10AAF000CDF804B0C3F3072C4FF0550B009B85F83D
:10AB0000322085F81722019A85F818824FF0520EEC
:10AB100041267227C8F3072A4FEA184985F82EB252
:10AB20004FEA18684FF0AA0B85F81E3285F81F22ED
:10AB3000687885F82FB285F830E085F831E085F83F
:10AB4000336085F8147285F8157285F8166285F8F9
:10AB500019A285F81A9285F81B8285F81DC26A69C8
:10AB6000012309F0C5FF6C719BE700BF10B50446D7
:10AB7000FFF73CFF00B9206010BD00BF2DE9F04198
:10AB800004460F460068A188FEF794FE054600289B
:10AB900051D1A379190651D4E268BA4203D213F015
:10ABA000020F08BF17460023A268A360002F42D0FF
:10ABB000206881784FEA4128002A43D0013A7B1E61
:10ABC000B3FBF8FCB2FBF8FEF4453BD3C8F1000040
:10ABD00002406169A260BF1A00293ED1A3680E46F7
:10ABE000DA05D00D00286BD0A269B24268D094F883
:10ABF00006C05FEA4C610BD5214651F8243B5878DA
:10AC0000012309F075FFA37910BB23F04001A17166
:10AC10002146324651F8240B0123407809F000FF09
:10AC2000A8B9A368E268A661934204D9A179E36058
:10AC300041F02002A2712846BDE8F0810225284695
:10AC4000BDE8F0812169002930D06161C4E7A379B2
:10AC500063F07F05A5710125EDE7474532D92068EE
:10AC600013E0FFF755F90146002842D0481CEED00A
:10AC7000012915D920688369994211D2A2686161BE
:10AC800008EB0203B845A3601DD294F806C05FEA42
:10AC90008C73C8EB0707E4D4FFF700F80146E5E73B
:10ACA000A17961F07F05A5710225C4E7FFF730F9AE
:10ACB00001280146F4D0421CC9D0206161618BE7B4
:10ACC000E268B1E7A368FE05DB19F60DA360002E6C
:10ACD00086D022689069023902388142E0D292F827
:10ACE00002E0926A0EFB01210029D9D001EB572620
:10ACF00076E7A3684746E6E730B587B006AB04467B
:10AD000043F8141D002218462146FEF72FFE08B115
:10AD100007B030BD03A8A06101992046FFF7E6F90E
:10AD2000B0B9636973B1DA7AD00615D593F81BE030
:10AD3000987E5D7D1A7D40EA0E2C42EA05234CEA9E
:10AD40000341A1602368D9882046A180FFF710F84D
:10AD5000042808BF0520DBE70520D9E72DE9F04FDF
:10AD60000D468BB0164618B10B200BB0BDE8F08F26
:10AD700040F69073C2F200031C6834B1207009F0F1
:10AD800025FEC20703D50320EFE70C20EDE710F006
:10AD9000040001D00A20E8E7012109AA09F010FF08
:10ADA000002840F0F581099B7F2B40F2F181002DB6
:10ADB00014BF07463F27721EDB1B3242099340F047
:10ADC0000782002E00F00482760A00F0FE81802EB9
:10ADD00034BFB3464FF0800BB3FBFBF240F6F57186
:10ADE0008A4240F2E08101F570494A4540F22883E9
:10ADF000920002F50070C61D4FF00008760A4FF071
:10AE00000309CDF80C804FF0200A0AEB070ECDF8AD
:10AE100008E0DDF80CC0DDF808800CEB060EF0440D
:10AE200008EB0B018B4201D20E209EE7002003218C
:10AE300008AA09F0C5FE20B9089B13B1B3F5004F6D
:10AE400001D901230893089B581E594200EB0802C0
:10AE500002EA0100C8EB0002B9F1030F0892099B56
:10AE600000F0E581B618CAEB030EDDF80CC0C6EBA6
:10AE70000E01CCEB0100B0FBFBF2B9F1020F059221
:10AE800000F08881002D40F0CD8104F1300CDB19F9
:10AE900004F50C706246114601F8015B55704A1CBE
:10AEA0008242F8D140F2FF38C0F2FB080122802034
:10AEB000434584F8EE0184F8EF2184F8F02184F80A
:10AEC000F15100F2F38143F6C16EB3FBFEF3990832
:10AED00041F03F0584F8F53184F8F451FE20B9F1D2
:10AEE000030F84F8F30100F0DD81099BB3F5803F87
:10AEF0002CBF0625042584F8F251099B1A0E4FF049
:10AF0000000E190CC3F307254FF03F0884F8FA31FF
:10AF100084F8FD215523AA2284F8FC1184F82E32EE
:10AF200084F82F22704684F8F68184F8F7E184F8DB
:10AF3000F8E184F8F9E184F8FB5161467246012397
:10AF400009F0D6FD002840F02381F820049004F198
:10AF5000300804F50C75434600211A4602F8011B1F
:10AF60005970531CAB42F8D1EB2284F83B10FE2100
:10AF700084F8302084F8311090224D215320099B11
:10AF800084F8322084F8331044224F2184F83400AE
:10AF900084F8352084F836103522302184F83700C3
:10AFA0002E20B9F1030F14BF4FF0020E4FF0000E28
:10AFB000CAF3072C84F8382084F8390002220120D3
:10AFC00084F83A100021B3F5803F84F83C2084F8DF
:10AFD0003DB084F83EA084F83FC084F8400084F877
:10AFE000411084F842E080F01081C3F3072084F818
:10AFF000433084F84400DDF810E084F84C704FF0E2
:10B00000000A3F20FF2384F845E084F8480084F8D4
:10B0100049A084F84A3084F84BA084F84DA084F805
:10B020004EA084F84FA009F0CFFCB9F1030F0890AF
:10B0300000F04281C74A84F85700010C12F801ABB6
:10B0400084F85910030EC0F3072EC6F3072C802096
:10B05000292184F85A3084F847C084F8466084F87F
:10B0600058E084F8540084F8561004F16E0C84F80B
:10B070005BA004F15C031146184611F801EB52780D
:10B0800000F801EB5A70431C4A1C6345F3D155216B
:10B09000AA2384F82E1284F82F32002041463A4623
:10B0A000012309F025FD002872D1B9F1030F00F04A
:10B0B000A1814346002103F8011BC5EB0802D043E0
:10B0C0009D4200F001020BD01AB103F8011B9D4212
:10B0D00006D0184600F8011B5970431C9D42F8D158
:10B0E000B9F1030F00F08C814FF47F40B9F1010FEB
:10B0F000C0F2FF00DDF810C018BF6FF0FF0040EA9B
:10B100000C03FF22190E089384F8303084F83120A4
:10B1100084F8322084F8331000204146029A01233B
:10B1200009F0E6FC002833D14346C5EB080203F8DA
:10B13000010BD1439D4201F001020BD01AB103F87B
:10B14000010B9D4206D0194601F8010B58704B1CAB
:10B150009D42F8D10123DDF808A008939E420AEB36
:10B1600003057ED94FF0000A9C4604E0089B581C5A
:10B170008642089075D92A46634650464146CDF826
:10B1800004C009F0B5FC0135DDF804C00028EDD09D
:10B190000120EAE5DDF814C040F6F57294453FF66B
:10B1A00071AE0E20E1E502EB4200411C4A08D61CBC
:10B1B0004FF0010906F5FE72D61C4FF0200C760AFE
:10B1C000CDF80CC04FF0010A1FE64FF0010B03E66B
:10B1D00044F6D350C1F26200A0FB0301CE09B6F5DC
:10B1E000806F10D240F68C51C0F60201002231F877
:10B1F000028F01324645FAD340F6BC46C0F602063D
:10B2000036F81260E0E50022F6E7C3F3072A190CCE
:10B210001A0E84F8503084F851A084F8521084F843
:10B220005320E8E64FF0F00CCDF810C08FE69244C2
:10B23000CAEB0301DDF80CC0C6EB010ECCEB0E002F
:10B24000B0FBFBF10591DDF814C04FF6F57EF44537
:10B250007FF6EAADDDF808E00EEB0208CDF80880D5
:10B2600010E6DDF80CC00026B9F1030F18BFE34665
:10B270004FF0010A2A4630464146534609F038FC51
:10B280000135002884D1BBF1010BF3D1B9F1030FD3
:10B2900064D000200146024609F092FC003018BF3D
:10B2A000012062E50C2184F8F21126E6FF2284F8E1
:10B2B000F42184F8F52111E6274B84F87300020C81
:10B2C00013F8011B0792320EC0F3072C06914FEAC8
:10B2D000106E310CC6F3072084F85720062284F83C
:10B2E00074C084F85500DDF81CC084F856100220A4
:10B2F000012184F86220069A84F85C0084F86010CA
:10B300008020292184F875C084F8772084F854605F
:10B3100084F876E084F85DA084F85EA084F85FA0ED
:10B3200084F861A084F863A084F8700084F8721037
:10B3300004F18A0C04F178021946104611F801EB69
:10B340005B7800F801EB5370421C4B1C6245F3D153
:10B350009DE600BFF80C0208E40C0208DDF814902A
:10B3600009F1FF35C5F307230293290C2A0E84F84F
:10B370001852029D039104924FF0520E84F830E06F
:10B3800084F831E084F81952DDF80CE0049D84F86B
:10B390001AE24FF0550AFF204FF0410C4FF06109BF
:10B3A000722684F82EA24FF0AA0A7A1C4146012385
:10B3B00084F81C0284F81D0284F81E0284F81F021F
:10B3C00084F82FA284F8329084F833C084F8146291
:10B3D00084F8156284F816C284F8179284F81B5218
:10B3E000584609F085FBFA1D58464146012309F0ED
:10B3F0007FFB4EE7BA1D4146012309F079FB58E671
:10B40000DDF810E0FF236EF0FF020F21089284F8B0
:10B41000302084F8313084F8323084F8333084F8C6
:10B42000343084F8353084F8363084F8373084F896
:10B43000383084F8393084F83A3084F83B106BE6C1
:10B44000911C4E004FF00209B4E600BF10B590F811
:10B45000603282B00446ABB1D4F84C12002904DB50
:10B4600004F12400FFF78AFBB8B9D4F84812D4F8E5
:10B47000502204F1240001ABFFF79AF968B9019852
:10B4800002B010BD00F12400611C0A22FEF770FF1B
:10B4900048B9012084F86002DEE7002184F86012D8
:10B4A0004FF0FF30ECE74FF0FF30E9E710B590F8D0
:10B4B000603282B00446ABB1D4F84C12002904DBF0
:10B4C00004F12400FFF75AFBB8B9D4F84812D4F8B5
:10B4D000502204F1240001ABFFF77CF868B9019811
:10B4E00002B010BD00F12400611C0122FEF740FFF4
:10B4F00048B9012084F86002DEE7002184F8601278
:10B500004FF0FF30ECE74FF0FF30E9E710B590F86F
:10B51000603204462BB100F12400FFF767FA18B936
:10B5200010BD4FF0FF30FBE7002084F860024FF0C1
:10B53000FF3010BD30B583B090F860320022044671
:10B540000192DBB940F69470C2F2000000F560652C
:10B55000043540F6A451D0F8442EC0F60201631C15
:10B56000284612F05BF904F1240029460A22FEF76E
:10B57000FFFE00283DD1012184F86012D4F8582242
:10B58000D4F85C32D01A12F04FF8B0F5007F2EDB01
:10B59000D4F85852D4F85C028542CBBFD4F8585244
:10B5A000D4F85C02D4F85C02D4F850522A1AB2F5EE
:10B5B000007F01D9510A4A02D4F85C32D4F848120B
:10B5C00004F12400C91801ABFFF7F2F8D4F85C527B
:10B5D000019BD4F8502205EB030CBCFBF2F502FBF7
:10B5E00015C2C4F85C2220B9184603B030BD019BD7
:10B5F000FAE74FF0FF30F8E710B5044690F8600224
:10B6000000B910BD04F12400FFF7B0FA4FF00003B9
:10B61000002884F8603218BF4FF0FF3010BD00BF23
:10B6200010B590F86132032B044618D0012B1BD0C3
:10B63000022B1ED0042B21D0052B07D0207800210F
:10B6400084F86112BDE8104000F0ECBCFFF7D4FFB5
:10B65000C4F8540294F86132032BEFD110BDFFF708
:10B6600069FFC4F85402F5E7FFF720FFC4F854025D
:10B67000F0E7FFF7EBFEC4F85402EBE7FFF746FFF5
:10B68000C4F85402E6E700BF38B5084C40F6B055A0
:10B69000C0F602050B4602462946204612F0BEF8C7
:10B6A0002046BDE83840F7F753B900BF981D002089
:10B6B000F0B540F69474C2F2000404F53C6040F624
:10B6C000C0510430C0F6020183B0FFF715FB032818
:10B6D000014600F08B80012800F0888080B140F6A0
:10B6E000C450C0F60200FFF7CFFF0020014602461B
:10B6F000FFF734FB0146002840F08480C4F8440E74
:10B7000040F69474C2F2000440F6086104F53E6706
:10B71000C0F6020138460122FEF72AFE054600283F
:10B7200046D040F69473C2F20003D3F8444E611C35
:10B73000B1F57A7FC3F8441E36D240F69474C2F253
:10B74000000440F6086104F53E65C0F60201284693
:10B750000A22FEF70DFE014600284AD104F560607A
:10B76000061D41F21C51D4F8442EC0F602013046A9
:10B7700012F054F8304612F041F93146024601AB5E
:10B780002846FFF715F806462846FFF7EFF9002E82
:10B790002CD140F63060C0F60200D4F8441EFFF70A
:10B7A00073FF304603B0F0BD0025C3F8445EC4E724
:10B7B00004F560660436402201AB38463146FEF798
:10B7C00009FF019B012B0DD941F21C5104F5646264
:10B7D0000432C0F60201304612F036F80028D8BF15
:10B7E000C4F8445E0C48FFF7C1F99AE74FF0FF3008
:10B7F000D8E740F61460C0F60200FFF745FF4FF0AF
:10B80000FF30CFE740F6EC50C0F60200FFF73CFFF8
:10B810004FF0FF30C6E700BF741B002040F64460C5
:10B820002DE9F843C0F6020040F69474C2F2000419
:10B83000F7F78EF804F5186704F53C6904F5986588
:10B840000126143709F104090C3500200BF086FE9F
:10B8500000214FF40972384612F056F8484600218C
:10B860001C2212F051F8002E41D131464FF40972DA
:10B8700004F1280012F048F84FF0FF38207984F8DE
:10B880006462C4F8588200F0CDFB31464FF409726F
:10B8900004F5237012F038F894F8680284F8C8644C
:10B8A000C4F8BC8400F0BEFB31464FF4097204F5C5
:10B8B0009E6012F029F894F8CC0484F82C67C4F840
:10B8C000208700F0AFFB04F5EA6031464FF40972BF
:10B8D000043012F019F894F8300784F89069C4F82D
:10B8E000848900F09FFB4FF47A700CF059FA3946C6
:10B8F0000020FEF729FD0146002840F0C280052106
:10B90000607800F093FAD4F8481E4B1CC4F8483E07
:10B91000FFF7CEFE0028C0F2B28001200BF01EFE21
:10B9200017E094F8C964002E3AD194F82D67002EE0
:10B930005AD194F89169002E78D1607800F018FB04
:10B940006078052100F072FAD4F8480E461CC4F85D
:10B95000486E94F86522002AE3D0261D3046FFF792
:10B960005FFE94F865020328DBD1D4F85812002951
:10B970007FDBD4F8483E44F6D351581CC1F2620133
:10B98000A1FB001291094FF47A7C0CFB1103002BF0
:10B99000C7D13046FFF7BAFD94F8C964002EC4D071
:10B9A00004F51A763046FFF73BFE94F8C9040328E5
:10B9B000BBD1D4F8BC1400295BDBD4F8482E44F684
:10B9C000D35C531CC1F2620CACFB031081094FF431
:10B9D0007A7E0EFB1132002AA7D13046FFF796FD82
:10B9E00094F82D67002EA4D02846FFF719FE94F88E
:10B9F0002D37032B9DD1D4F82017002939DBD4F83B
:10BA0000480E44F6D3510130C1F26201A1FB00138C
:10BA10009A094FF47A7606FB1201002989D128464B
:10BA2000FFF774FD94F89169002E86D004F5E66660
:10BA30003046FFF7F5FD94F89129032A7FF47DAF96
:10BA4000D4F88419002914DBD4F8483E44F6D351C5
:10BA5000581CC1F26201A1FB001291094FF47A7ED9
:10BA60000EFB1103002B7FF468AF3046FFF74EFD4D
:10BA700063E740F67C60C0F60200FFF705FE002693
:10BA8000E3E640F65860C0F60200FFF7FDFDBDE8B2
:10BA9000F8430CF007B900BF70B540F69474C2F2D9
:10BAA000000440F64C620021204611F02DFF0021D9
:10BAB000084600F035F940F69C610346C0F60201E5
:10BAC000A02063700CF080FE41F6E0550646C2F2FD
:10BAD00000054BF61D00C0F6000006F51F7300219F
:10BAE0004AF23E022E600CF037F8207070BD00BFA5
:10BAF00070B540F69474C2F20004054694F866628C
:10BB00003EB3601D294611F051FF00283CD094F847
:10BB1000CA34EBB104F51A700130294611F046FF22
:10BB2000B0B194F82E1759B304F598600D3029463A
:10BB300011F03CFF20B394F892291AB304F5E663A0
:10BB4000581C294611F032FFE0B1FF2040B270BD11
:10BB5000012640F69470C2F200004FF4197404FB01
:10BB600006040122294684F86622601D11F0FCFEBD
:10BB70000020014600F0D4F82071F0B240B270BD50
:10BB80000226E6E70326E4E70646E2E710B50446A8
:10BB900090F86202D8B140F6947CC2F2000CC4F86E
:10BBA00048129DF808109CF8010084F86112C4F84E
:10BBB0004C22C4F8503200F035FA207800F0D8F961
:10BBC0002078002100F032F9D4F8540210BD4FF073
:10BBD000FF3010BD30B540F69474C2F200044FF44B
:10BBE000197505FB004083B0012404300094FFF771
:10BBF000CDFF03B030BD00BF30B540F69474C2F243
:10BC000000044FF4197505FB004083B00224043092
:10BC10000094FFF7BBFF03B030BD00BF38B540F65E
:10BC20009473C2F200034FF4197505FB00352C1D07
:10BC300094F86222DAB194F8600228B9002184F8FD
:10BC40006212D4F8540238BD5878052384F8613262
:10BC500000F0E8F9287900F08BF90021287900F04C
:10BC6000E5F8002184F86212D4F8540238BD4FF090
:10BC7000FF3038BD40F69471C2F200014FF41972E2
:10BC800002FB0013D3F85C02704700BF40F6947CBF
:10BC9000C2F2000C4FF4197202FB00C3C3F85C122D
:10BCA000704700BF10B440F6947CC2F2000C4FF411
:10BCB000197404FB00C393F86602043348B10320EF
:10BCC00083F86102C3F84812C3F85022012010BC67
:10BCD00070474FF0FF30FAE742F2704CC2F2000CAE
:10BCE000DCF800309861C3608160027441F6E4536F
:10BCF000C2F200031B693BB90360436041F6E451A3
:10BD0000C2F20001C86004E0186043604FF0000216
:10BD1000026041F6E453C2F200031861704700BFAD
:10BD2000F8B540F64564C2F20004267806F1010534
:10BD3000EAB2227041F6E453C2F200039D6815F0A6
:10BD4000010F10D04FF001031F46DCB21E4603FA6C
:10BD500003F22A4236D10BE0DCB21E4607FA03F2A8
:10BD60002A4220D104E04FF001024FF00006344691
:10BD700041F6E45CC2F2000C42EA0503CCF808305C
:10BD800001FA06FEDCF800104EEA0102CCF80020B1
:10BD900000FA06F1DCF8043041EA0300CCF80400B4
:10BDA000FDF74AFB0CE003F10103DCB21E4607FA83
:10BDB00003F22A4209D1DBE7FDF73EFB4FF0FF0417
:10BDC0002046F8BD03F10103C6E703F10103202B70
:10BDD000C2D1F1E708B541F6E453C2F200031B6893
:10BDE0004FF0010202FA00F018421BD040F6456EF7
:10BDF000C2F2000E9EF800C00CF10102D1B28EF822
:10BE0000001041F6E45CC2F2000CDCF8042000EA09
:10BE1000020123EA0100CCF80000FDF70DFB4FF012
:10BE2000000008BD4FF00C0008BD00BF70B586B023
:10BE30000C4640F64461C2F200010B78002B40F042
:10BE40008C8040F6456CC2F2000C9CF80020002A61
:10BE500040F0868040F64563C2F2000393F800C0CC
:10BE60000CF10102D1B2197041F6E45EC2F2000E8B
:10BE7000DEF800304FF0010505FA00F51D420DD047
:10BE800041F6E450C2F200004268154023EA050181
:10BE90000160FDF7D1FA4FF0000066E042F2704613
:10BEA000C2F2000636685CBB01A829464FF00202C8
:10BEB000FFF712FF4FF00203737140F64662C2F2C1
:10BEC00000024FF001011170FDF7B6FAB46140F6BF
:10BED000456CC2F2000C9CF8000000F10103DAB2DC
:10BEE0008CF8002041F6E453C2F2000359680D407B
:10BEF000186820EA05051D60FDF79EFA204634E02B
:10BF000001A829464FF00202FFF7E6FE304621461F
:10BF10000BF0D0FEFDF790FAB06920B34FF00004AB
:10BF2000B46140F6456CC2F2000C9CF800E00EF1E2
:10BF30000103D8B28CF8000041F6E45EC2F2000EB4
:10BF4000DEF804201540DEF8001021EA0505CEF8E1
:10BF50000050FDF771FA204607E04FF0030004E0BF
:10BF60004FF0150001E04FF0050006B070BD00BFB6
:10BF700041F6E453C2F200034FF0010101FA00F16F
:10BF80001A6822EA010018604FF00000704700BFF5
:10BF90000368A3B9436843B941F6E453C2F200030E
:10BFA0004FF00002DA601A6117E041F6E45CC2F279
:10BFB000000CCCF810304FF0000119600DE0426821
:10BFC00042B941F6E451C2F20001CB604FF00002E9
:10BFD0005A6002E05A6042681360C3684FF0000084
:10BFE0009861704738B50546FFF7D2FFEC68E36902
:10BFF000B3F1FF3F02D020460BF0A8FE4FF0FF3216
:10C00000A26142F27041C2F200010868844203D189
:10C010004FF00103637102E020460BF041FC2868F9
:10C0200038BD00BF38B541F6E453C2F200031B68C7
:10C030004FF0010505FA00F51D4230D141F6E452FA
:10C04000C2F2000245EA0301116040F64560C2F207
:10C05000000090F800C00CF10103D9B20170D06863
:10C06000D8B11446027C5AB98368226803EA0201F7
:10C070008B420FD1FFF7B6FF61680D420DD10AE088
:10C08000226883681A4205D0FFF7ACFF61680D4251
:10C0900003D100E000680028E4D1FDF7CDF94FF0AE
:10C0A000000038BD08B5014640F64560C2F2000008
:10C0B000037853B14FF003004FF0000209F02AFB60
:10C0C00000280CBF1220002008BD0846FFF7AAFF79
:10C0D00008BD00BF00F1784243F6FF739A420FD9C2
:10C0E000A2F580429A4201D8082070474FF4004CD4
:10C0F000CFF2FF7C00EB0C01994203D8102070476F
:10C10000002070474FF48041CFF2FF7142189A42ED
:10C1100001D81820704700F1774303F57F0CBCF578
:10C12000803F01D2202070474FF6FF7203F57E0159
:10C13000C0F20102914201D82820704703F57C0C1F
:10C14000944501D83020704703F57A01914201D817
:10C150003820704703F5780C944501D8402070478B
:10C1600003F57603934201D84820704700F17742E7
:10C1700002F57400B0F5003F2CBF582050207047E6
:10C180002DE9F0470024C0F60E04002814BF06462F
:10C190002646904689460EF03BF8F3200EF054F800
:10C1A0003046FFF797FF044606EB0800FFF792FFC3
:10C1B000031B02251B07074618D5BC42294620460B
:10C1C00024D80EF095F80246082A294620467FD04A
:10C1D0000EF08EF808287BD0204602210EF088F859
:10C1E00000240EF027F82046BDE8F08784420DD8E1
:10C1F000204629460EF07CF8082805D0204629461E
:10C200000EF076F80828E7D10834D6E7B8F1000F29
:10C210005CD04C46304654F8041B0EF049F808F147
:10C22000FF37082807F0010711D054F8041C3046E6
:10C230000EF03EF808280AD054F8041C30460024BA
:10C240000EF036F80DF0F6FF2046BDE8F087002529
:10C2500001350436454539D08FB154F8041B3046BA
:10C260000EF026F8082806D054F8041C30460EF0CC
:10C270001FF80828E0D101350436454526D054F88A
:10C28000041B30460EF014F8014608293046A1463A
:10C2900005D054F8041C0EF00BF80828CCD1043655
:10C2A000216830460EF004F803460135082B30466D
:10C2B000374609F1040405D054F8041C0DF0F8FFCA
:10C2C0000828B9D101353E1D4545D8D1012488E75C
:10C2D0000834294620460EF00BF88446BCF1080FBE
:10C2E00029462046A24604D00EF002F808287FF422
:10C2F00073AF0AF1080460E70020C0F60E00704733
:10C3000047F61023C1F6FF7353F82000704700BFB3
:10C310004EF63073CEF200035A6822F000415960A5
:10C32000586820F080425A60704700BF2DE9F00F36
:10C3300041F23803C1F2000390B0197E4A0700F1C0
:10C34000DC80DA7AB3F81480DF78B3F806A0DD7900
:10C35000B3F8109093F804C01E7A1C7BD3F804B095
:10C3600058880492DA7B0CF03F0C0592DA7C4FEA95
:10C370004C1C4CEAD70CCBF38A1BC0F30A00CAF35F
:10C380004A07DDF810A00F92ADF808B0ADF8000034
:10C39000E400D3F808B0588944EA5A1406F07F063E
:10C3A000D3F80CA0360146EA1516CBF3CA15C0F334
:10C3B0008A0BCAF30A20B3F80EA04FEAC959CAF390
:10C3C000CA0AADF818A04FEAD959DDF814A04FEA0F
:10C3D000890949EA9A19D3F810A0CAF34A2AADF894
:10C3E00020A0B3F812A04FEA8852CAF30A1AADF897
:10C3F00028A04FEA9258DDF83CA04FEA480848EAE6
:10C40000DA18D3F814A0CAF38A2AADF830A0BDF820
:10C4100008A0CAF5D46ACDF808A0BDF800A0AAF516
:10C42000806ACDF800A041F63802ACF5806AC1F20E
:10C430000002CDF810A0DDF808A0BDF818C0A2F8E1
:10C4400008A0DDF800A0A7F58067A2F80AA0DDF833
:10C4500010A00597A2F80CA0C6F58066DDF814A020
:10C460000E96A2F80EA0C5F58065DDF838A00F95F0
:10C47000BDF82070BDF82860BDF83050A2F810A0BB
:10C48000DDF83CA0C4F58064C0F58060CBF5806B1E
:10C49000CCF5806CC9F58069C7F58067C6F5806604
:10C4A000C8F58068C5F580651083A2F812A0A2F8CF
:10C4B00014B0D482A2F81AC0A2F81C90D7831684B4
:10C4C000A2F822809584DC8A11F0010F4FF6E04338
:10C4D0000CBF18464FF44870C4F34A1411F0020F11
:10C4E00018BF4FF44873C4F58061D184108553851B
:10C4F000012010B0BDE8F00F70474FF0FF30F8E7B3
:10C5000041F23803C1F200031A78012A09D003D39B
:10C51000022A12D0002070470F284FF0000013D0DD
:10C5200070475A7899180132D2B2172A88705A7017
:10C53000F0D1022018700020704700221A7008B154
:10C5400010467047FFF7F2BE01221A70587070470C
:10C5500070B541F2380000254FF4984448F2A066C7
:10C5600086B0C4F2000429461922C0F20106C1F2C5
:10C57000000011F0C9F9202331462A4620460095D3
:10C5800008F090FE41F6380CC1F2000C024602A8F9
:10C59000CCF804200EF0BCFF4FF400514FF4806043
:10C5A000ADF80E10ADF810000423204602A9029643
:10C5B000ADF80C50ADF81450ADF812300EF028FF65
:10C5C000204601210EF0B0FF06B070BD41F25400CC
:10C5D00000210C2270B5C1F2000011F095F940F273
:10C5E000B423C1F2000393EDF17ADFED507AB4EE9B
:10C5F000677AF1EE10FA5ED09FED4D1AC1EE070A90
:10C60000DFED4C6A20EEA60AD3EDEB6ABCEEC07AF1
:10C61000F4EE676A17EE105AF1EE10FAADB268D177
:10C62000FF2640F2B423C1F20003D3EDEC7AF5EE1D
:10C63000407AF1EE10FA3FD1FF2432061BD440F2CB
:10C64000B420C1F20000D0EDF25ABCEEE55A294602
:10C6500015EE102AF0B24FF0FF3305F0FDFC41F269
:10C660005402C1F2000240F6FC61C0F602015060C3
:10C670000846F6F76DF923061DD440F2B42EC1F238
:10C68000000E9EEDF37ABCEEC76AE0B216EE102AF9
:10C6900029464FF0FF3305F0DFFC41F25403C1F2AD
:10C6A000000340F61C7CC0F6020C98606046BDE8B2
:10C6B0007040F6F74DB970BDB2EE0C3AF4EEC37AA5
:10C6C000F1EE10FAB8D8F7EE004A37EEE44AFDEE84
:10C6D000C43A13EE904AE4B2204605F0B5FC0028B7
:10C6E000ABD040F6D060C0F60200F6F731F9FF2477
:10C6F000A3E7F2EE0C7AF4EEE76AF1EE10FA8FD8C7
:10C70000F7EE002A36EEE22AFDEEC21A11EE906A2A
:10C71000F6B2304605F098FC002882D040F6A460BE
:10C72000C0F60200F6F714F9FF267AE700000000D1
:10C730000000484300409C4510B541F25403C1F24B
:10C7400000032DED028B5A68002A5CD040F2B4221F
:10C75000C1F2000292ED091AFDEEC10A41F6380C51
:10C7600010EE900AC1F2000C011DD2EDF46A3CF902
:10C77000110000EE100AB8EEC07A41F2D81187EE2F
:10C78000267AC1F20001DFED5A7A91ED006A06EED9
:10C79000277AD3ED007AF4EE477AF1EE10FA07D05B
:10C7A00037EEC72AD2EDF61A42EE617AC3ED007A6F
:10C7B0005049DFED4F5A91ED005A40F2B42E45EE4C
:10C7C000657AC1F2000EDEEDF24A46EEA74ADEEDD2
:10C7D000F03A9EEDEF3ABDEEE44AFDEEE36AFDEE7F
:10C7E000C32A14EE100A12EE902A16EE901A0CF0DC
:10C7F00065F84FF4406CC4F2000C42F21073DCF8A0
:10C8000024209A4269D841F25400C1F200008168A4
:10C8100000293CD040F2B424C1F2000494EDF76A40
:10C82000B5EE406AF1EE10FA334B33D193ED034A83
:10C83000DFED2F4AD4EDF53A64EE646AD4EDF37A75
:10C8400046EEA37AD4EDEE6AD4EDED5ABDEEE77A6A
:10C85000BDEEE66ABDEEE55A17EE100A15EE102A97
:10C8600016EE101A0CF02AF84FF4406CC4F2000CCB
:10C8700042F21073DCF824209A4280B207D941F2C8
:10C88000540EC1F2000EDEF8082011680860BDECFD
:10C89000028B10BD93ED038ABDEEC83A13EE100A69
:10C8A00010F0C2FE94EDF72ADFED142AC2EE820AE0
:10C8B00001EE900AB8EEE11A9FED0D0AC1EE207A62
:10C8C00094EDF57A28EE678AD4EDF37A28EE008AA3
:10C8D000D4EDEE6A48EE077AB6E741F2540CC1F2A5
:10C8E000000C80B2DCF804301A6810608BE700BFDF
:10C8F00000007A4430230020282300200000C84292
:10C9000038B540F2201441F26003C1F20004C1F2D4
:10C910000003D4F88041D3F8A05049F28062611B33
:10C92000C0F298029142054637D993F82440621C20
:10C930005FFA82FC4FFA8CF1881C83F824C053F80C
:10C9400020205AB341F26004C1F2000440F63C706A
:10C95000C0F60200F5F7FCFF94F92420911C28464C
:10C9600054F8211008F006FE0BF030FC40F2B42C15
:10C97000C1F2000C9CED3B0AFCEEC07A284617EE93
:10C98000901A08F0F7FD0BF0D9FB40F22010C1F22D
:10C990000000D0F88031C4F8A03038BD83F82420DE
:10C9A000D0E700BF70B5204D20486C68F5F7D0FF88
:10C9B0000BF0FAFB0A200BF0F3F92046FFF7A0FF7B
:10C9C000AB6A1A689B8851690B420CBF002601268E
:10C9D00006B91383204608F093FD02462046A2B113
:10C9E00008F09CFDC0B20BF057FD012814D00228BE
:10C9F00016D00328EED12046FFF782FF204608F02C
:10CA00007FFD02462046002AEAD1002ED2D1A96A33
:10CA100008688E884683CDE7A878FFF703FBD9E73F
:10CA20006878FFF7FFFAD5E760100010580F02088A
:10CA3000F0B540F6707041F2600489B0C1F20004B4
:10CA4000C0F6020040F2B427F5F782FFC1F20007FA
:10CA5000A8220021204610F057FF97ED3B1A4FF413
:10CA600016524FF48056FCEEC10AC4F20206E26090
:10CA70004FF461334FF4E132002501213046236148
:10CA800062614FF496434FF41642C4ED020AA3616B
:10CA9000E261256284F82450FCF758FD97ED3B0ACB
:10CAA000B0F804C0D0F800E0A062FCEEC07A4FF409
:10CAB00000774FF49040AEF81AC017EE901A2A464D
:10CAC0003B46C4F20000009708F0ECFB29460746FD
:10CAD00028466760FFF724F9294603462846637015
:10CAE000FFF71EF940F67C710246C0F6020168208D
:10CAF000A2700BF069FE41F6F857C2F200078646B5
:10CB00004CF6A5100EF5CE73C7F800E046F62302EA
:10CB10002946C0F600000BF01FF8034603A8237057
:10CB200002270DF0DDFC304603A903978DF8105065
:10CB30008DF813500DF018FC012104200EF064F85C
:10CB40000126082205A88DF8192005978DF81850A0
:10CB50008DF81A600DF012FB072107A88DF81C1044
:10CB60008DF81D508DF81E508DF81F6000F040FDAF
:10CB70004FF410534FF47842C4F67413C7F64222B0
:10CB8000A3662365E364C4F8A42009B0F0BD00BF28
:10CB900010B44FF4406141F26003C4F20001C1F2ED
:10CBA0000003496AD3F8944048F20F1C0C1BCFF6DF
:10CBB000F17C48F29E6004EB0C02C0F2010082425C
:10CBC00007D8D3F8A420A2EBC424A2EB6410C3F8C6
:10CBD000A40041F26003C1F20003D3F89000C3F84F
:10CBE0009410C3F88C00022010BC0DF00BBB00BFEA
:10CBF0002DE9F04F2DED028B840089B00E340546EF
:10CC000000AF24F00700ADEB000DC7F80CD040F2E8
:10CC10002014ADEB000DC7F808D04FF00008ADEBC5
:10CC2000000DC1F200049FED2B8A3D60C7F804D0CF
:10CC30004646A146D4F88021D4F880319342FBD0F7
:10CC4000D9F83811D9F83C01D9F840219346FA684F
:10CC50004FEA880302EB030C8A467A68B968CCF87D
:10CC600000A008F10108C918D318AE4298FBF5F2EC
:10CC70000860C3F800B005FB128818DA0136B54227
:10CC8000D8DAD7ED060A97ED051A97ED077A31EE57
:10CC9000200A70EE077AF4EEC87AF1EE10FAC9DCD9
:10CCA00007F12407BD46BDEC028BBDE8F08FF868A4
:10CCB000396807F11402FAF7BBFF3968B86807F161
:10CCC0001802FAF7B5FF7868396807F11C02FAF71D
:10CCD000AFFFD3E7CDCC4C3D10B541F20814C1F203
:10CCE00000040C220021204610F00EFE002101203D
:10CCF000FFF716F80021034601202370FFF710F814
:10CD00006070BDE81040F4F72BBD00BF41F208137E
:10CD1000C1F20003996818784A1C9A60FFF782B93B
:10CD200041F20813C1F20003596858784A1C5A604E
:10CD3000FFF778B941F6FC5341F6CC60C2F200032C
:10CD400041F6C462C2F2000010B40021C2F2000237
:10CD500003F1C80482E81800036019605960996003
:10CD600010BC70470A6802604B6843600820704737
:10CD70000B680360042070470B8803800220704713
:10CD80000B7803700120704770B541F21416C1F2A0
:10CD9000000696F90B00FEF76DFF32684123141868
:10CDA00013540546712148206170A070B27A40F298
:10CDB000AC51E270201DC2F20001C62210F086FDC7
:10CDC0003468EB1CE418012322781946D6B2581CAB
:10CDD00014F801C002EB0C03225CD9B28B1801EBF2
:10CDE000060EDAB2431C52FA8EFCC72B5FFA8CF6A1
:10CDF0001946ECD141F21410C1F2000084F8C720AA
:10CE0000B0F808C090F90B0084F8C860C8226544E7
:10CE100002FB0CF195FBF1FE01FB1E51BDE87040D9
:10CE2000FEF734BFF8B541F21416C1F2000696F9C8
:10CE30000B00FEF71FFF34684122251822540746D5
:10CE400071214D206970A870B37A83B10335002435
:10CE5000706800EBC40E50F83410DEF80430284639
:10CE6000984796F80AC00134A4450544F0DC41F225
:10CE70001415C1F200052E892968B51E032D394409
:10CE80003CDDCA780423AB4205F00100D4B21EDABF
:10CE900048B111F803C002EB0C00C2B2052314190B
:10CEA000AB42E4B213DA11F803C0013302EB0C0019
:10CEB00011F803E05FFA80FC0CEB0E020CEB0400AF
:10CEC000D2B2013352FA80F4AB42E4B2EBDB013E62
:10CED00041F2141E4A55C1F2000E8C55BEF80820CE
:10CEE0009EF90B00C821D71901FB02F397FBF3F160
:10CEF00003FB1171BDE8F840FEF7C8BE002404260C
:10CF000003252246E4E700BF2DE9F04F41F2141457
:10CF1000C1F20004632305221846A3728BB00821D6
:10CF200022810BF02FFCA37A6060002B00F0CA80F6
:10CF300041F62875C2F200054CF67157D5F83C84CD
:10CF40002589CDF8048008F1340308F138024CF645
:10CF500065560293039208F13C0308F10C02C0F6F7
:10CF60000007C0F600064CF6815C4CF6795B049332
:10CF7000059208F1100308F11402B646C0F6000C41
:10CF8000002140F2AC5408F1300A0693079208F1F0
:10CF9000040308F1080208F14009C0F6000BB84686
:10CFA000089366460992F4460B46C2F200045F46B7
:10CFB000C64614F813209B46622A66D8DFE812F0B2
:10CFC0002C0132012F014701440141013E0183013F
:10CFD00080017D017A017701740171016E016B019D
:10CFE0006801650162015F015C015901560126017A
:10CFF000230120011D011A011701140111010E0165
:10D000000B01080105010201FF00FC00F900F60018
:10D01000F300F000ED00EA00E700E400E100DE00CC
:10D02000DB00D800D500D200CF00CC00C900C6007C
:10D03000C300630063008B028802850282027F02C4
:10D040007C02D101CE01CB01C801C501C201BF01E3
:10D05000BC01B901B601B301B001AD01AA01A7013C
:10D06000A401A1019E019B019801950192018F01EC
:10D070008C0189018601530150014D014A013B0198
:10D0800038013501290140F8019004EB4B0898F86C
:10D0900001B0BBF1070F09D8DFE80BF032202020E8
:10D0A00043430404421801355660ADB241F21412F4
:10D0B000C1F20002013392F80AB008319B453FF7F4
:10D0C00078AF158141F21414C1F20004C8202189FF
:10D0D0000BF026FB20600BB0BDE8F08F00EB010BDE
:10D0E00041F21412C1F20002CBF804E092F80AB047
:10D0F0000133043508319B45ADB23FF75AAFE0E745
:10D1000042180133C2F804C041F21412C1F2000205
:10D11000083592F80AB008319B45ADB23FF749AFE8
:10D12000CFE700EB010841F21412C1F20002C8F887
:10D13000047092F80AB00133023508319B45ADB254
:10D140003FF737AFBDE7079A42509EE7069A425035
:10D150009BE7059A425098E7049A425095E7039A54
:10D16000425092E7029A42508FE740F801A08CE7C4
:10D170007D4A425089E77D4A425086E77C4A4250C8
:10D1800083E77C4A425080E77B4A42507DE77B4AF6
:10D1900042507AE77A4A425077E77A4A425074E737
:10D1A000794A425071E7794A42506EE7784A4250D4
:10D1B0006BE7784A425068E7774A425065E7774A1A
:10D1C000425062E7764A42505FE7764A42505CE757
:10D1D000754A425059E7754A425056E7744A4250E0
:10D1E00053E7744A425050E7734A42504DE7734A3E
:10D1F00042504AE7724A425047E7724A425044E777
:10D20000714A425041E7714A42503EE7704A4250EB
:10D210003BE7704A425038E76F4A425035E76F4A61
:10D22000425032E76E4A42502FE76E4A42502CE796
:10D230006D4A425029E76D4A425026E76C4A4250F7
:10D2400023E76C4A425020E76B4A42501DE76B4A85
:10D2500042501AE76A4A425017E76A4A425014E7B6
:10D26000694A425011E7694A42500EE7684A425003
:10D270000BE7684A425008E7674A425005E7674AA9
:10D28000425002E7664A4250FFE6664A4250FCE6D8
:10D29000654A4250F9E6654A4250F6E6644A425011
:10D2A000F3E6644A4250F0E6634A4250EDE6634AD0
:10D2B0004250EAE6624A4250E7E6624A4250E4E6F9
:10D2C000614A4250E1E6614A4250DEE6604A42501D
:10D2D000DBE6604A4250D8E65F4A4250D5E65F4AF4
:10D2E0004250D2E65E4A4250CFE65E4A4250CCE619
:10D2F0005D4A4250C9E65D4A4250C6E65C4A425029
:10D30000C3E65C4A4250C0E65B4A4250BDE65B4A17
:10D310004250BAE65A4A4250B7E65A4A4250B4E638
:10D32000594A4250B1E6594A4250AEE6584A425034
:10D33000ABE6584A4250A8E6574A4250A5E6574A3B
:10D340004250A2E6564A42509FE6564A42509CE658
:10D35000554A425099E6554A425096E6544A425040
:10D3600093E6544A425090E6B00200102C0200109E
:10D37000200200101C0200102802001038020010C9
:10D3800034020010C8100010BC100010B8100010BB
:10D39000B4100010FC100010B0100010AC10001001
:10D3A000A8100010A010001098100010F810001025
:10D3B00090100010E4100010E0100010DC100010BD
:10D3C000D8100010D4100010D01000106C02001003
:10D3D0006802001062180010A0020010DC010010AA
:10D3E000D8010010601800105E1800105C180010C2
:10D3F000EC010010E8010010E4010010E001001051
:10D400005A18001058180010561800105418001020
:10D4100064020010600200105C020010580200104C
:10D4200054020010500200104C02001010020010B4
:10D430000C0200100802001004020010000200108C
:10D44000FC010010F8010010F4010010F0010010C0
:10D4500052180010501800104E1800104C180010F0
:10D460004A18001048180010461800104418001000
:10D47000421800104018001074180010B811001065
:10D48000B4110010B0110010BC1100107611001082
:10D490007411001072110010701100106E11001044
:10D4A0006C1100106A110010681100106611001054
:10D4B0006411001062110010084A4250E5E5084A64
:10D4C0004250E2E5074A4250DFE5099A4250DCE566
:10D4D000089A4250D9E5019A4250D6E560110010F1
:10D4E0005E1100105C11001010B541F21414C1F26D
:10D4F000000400210C22204610F006FAFFF704FD7C
:10D5000040F6A070C0F60200FEF7F2FA2389216807
:10D51000E072C82202FB03F2FEF7C4FBBDE8104034
:10D52000FFF732BC38B5FEF7F3FE05F0ABFA4FF467
:10D53000A06000F053F8FBF7A9FF40F6A471C0F615
:10D5400002014FF486700BF03FF940F67404054673
:10D5500000F58463C2F2000442F28D6040F60C4292
:10D56000C0F201020C330021C0F6000025600AF071
:10D57000F3FAFBF7D3FF002038BD00BF70B54EF6BD
:10D58000FC54CEF200044FF4805322680F4D104E2D
:10D59000CEF2000342F080712160186841F2040469
:10D5A00040F0010282B01A60CEF200040BF058F88D
:10D5B0002B68581C28602268002101922160019884
:10D5C00033689842F2D201993160EFE7D01E002013
:10D5D0007406002008B500F0BBFAFEE74FF46D4377
:10D5E00040F0BE61CEF2000341F42020D8607047C5
:10D5F000C37830B47BB900784FF4614C410900F036
:10D600001F02CEF2000C2031012313FA02F04CF875
:10D61000210030BC70474FF46D45CEF200054178D3
:10D62000EC6885780278E343C3F30223C3F1040C6A
:10D630005FFA8CF411FA04F40F2151FA03F303EAB0
:10D640000501E4B24FF4614CCEF2000C41EA040350
:10D6500019010CEB0203C9B283F800130278012010
:10D66000510902F01F0310FA03F24CF82120D0E711
:10D6700010B541F22014C1F2000494F8A430002B3C
:10D6800075D141F22014C1F2000494F8A5000028DD
:10D6900040F0908041F22014C1F2000494F8A600FA
:10D6A000002840F0AA8041F22014C1F2000494F84E
:10D6B000A700002840F0C58041F22014C1F2000408
:10D6C00094F8A800002840F0E08041F22014C1F254
:10D6D000000494F8A900002840F0FB8041F22014D7
:10D6E000C1F2000494F8AA00002840F0168141F22B
:10D6F0002014C1F2000494F8AB00002840F03181FE
:10D7000041F22014C1F2000494F8AC00002840F06B
:10D710004C8141F22014C1F2000494F8AD000028BD
:10D7200040F0678141F22014C1F2000494F8AE0089
:10D73000002840F0828141F22014C1F2000494F8E4
:10D74000AF00002840F09D8141F22014C1F2000496
:10D7500094F8B000002840F0B88141F22014C1F2E2
:10D76000000494F8B100002840F0D38110BD40F2CD
:10D77000B42CC1F2000CDCED3E0A9CED400ABDEE7B
:10D78000E07AFDEEC07AB4F93C0017EE101A17EEFD
:10D79000902A0BF093F8636882B21968A28741F26D
:10D7A000201410B2C1F20004086094F8A50000280B
:10D7B0003FF470AF40F2B42EC1F2000EDEED3E2A0F
:10D7C000DEED401ABDEEE22ABDEEE11AB4F93E00EC
:10D7D00012EE101A11EE102A0BF070F8A36882B244
:10D7E0001968E28714B20C6041F22014C1F20004FF
:10D7F00094F8A60000283FF456AF40F2B42CC1F2D2
:10D80000000CDCED3E4ADCED403ABDEEE44ABDEEF4
:10D81000E33AB4F9400014EE101A13EE102A0BF09C
:10D820004DF8E36882B21968A4F8402014B20C6085
:10D8300041F22014C1F2000494F8A70000283FF43C
:10D840003BAF40F2B42EC1F2000EDEED3E6ADEEDDB
:10D85000405ABDEEE66ABDEEE55AB4F9420016EE56
:10D86000101A15EE102A0BF029F8236982B21968F4
:10D87000A4F8422014B20C6041F22014C1F200045A
:10D8800094F8A80000283FF420AF40F2B42CC1F275
:10D89000000CDCED3E0A9CED400ABDEEE07AFDEEA8
:10D8A000C07AB4F9440017EE101A17EE902A0BF064
:10D8B00005F8636982B21968A4F8442014B20C60B8
:10D8C00041F22014C1F2000494F8A90000283FF4AA
:10D8D00005AF40F2B42EC1F2000EDEED3E2ADEEDC1
:10D8E000401ABDEEE22ABDEEE11AB4F9460012EE8E
:10D8F000101A11EE102A0AF0E1FFA36982B219682A
:10D90000A4F8462014B20C6041F22014C1F20004C5
:10D9100094F8AA0000283FF4EAAE40F2B42CC1F219
:10D92000000CDCED3E4ADCED403ABDEEE44ABDEED3
:10D93000E33AB4F9480014EE101A13EE102A0AF074
:10D94000BDFFE36982B21968A4F8482014B20C60E4
:10D9500041F22014C1F2000494F8AB0000283FF417
:10D96000CFAE40F2B42EC1F2000EDEED3E6ADEED27
:10D97000405ABDEEE66ABDEEE55AB4F94A0016EE2D
:10D98000101A15EE102A0AF099FF236A82B219685C
:10D99000A4F84A2014B20C6041F22014C1F2000431
:10D9A00094F8AC0000283FF4B4AE40F2B42CC1F2BD
:10D9B000000CDCED3E0A9CED400ABDEEE07AFDEE87
:10D9C000C07AB4F94C0017EE101A17EE902A0AF03C
:10D9D00075FF636A82B21968A4F84C2014B20C6017
:10D9E00041F22014C1F2000494F8AD0000283FF485
:10D9F00099AE40F2B42EC1F2000EDEED3E2ADEED0D
:10DA0000401ABDEEE22ABDEEE11AB4F94E0012EE64
:10DA1000101A11EE102A0AF051FFA36A82B2196897
:10DA2000A4F84E2014B20C6041F22014C1F200049C
:10DA300094F8AE0000283FF47EAE40F2B42CC1F260
:10DA4000000CDCED3E4ADCED403ABDEEE44ABDEEB2
:10DA5000E33AB4F9500014EE101A13EE102A0AF04B
:10DA60002DFFE36A82B21968A4F8502014B20C604A
:10DA700041F22014C1F2000494F8AF0000283FF4F2
:10DA800063AE40F2B42EC1F2000EDEED3E6ADEED72
:10DA9000405ABDEEE66ABDEEE55AB4F9520016EE04
:10DAA000101A15EE102A0AF009FF236B82B21968CA
:10DAB000A4F8522014B20C6041F22014C1F2000408
:10DAC00094F8B00000283FF448AE40F2B42CC1F204
:10DAD000000CDCED3E0A9CED400ABDEEE07AFDEE66
:10DAE000C07AB4F9540017EE101A17EE902A0AF013
:10DAF000E5FE636B82B21968A4F8542014B20C607E
:10DB000041F22014C1F2000494F8B10000283FF45F
:10DB10002DAE40F2B42EC1F2000EDEED3E2ADEED57
:10DB2000401ABDEEE22ABDEEE11A12EE101A11EE15
:10DB3000102AB4F956000AF0C1FEA36B1FFA80FC4C
:10DB40001A68A4F856C00FFA8CF1116010BD00BF1E
:10DB500040F2B423C1F2000310B493ED3F0A41F246
:10DB60002011C1F20001FDEEC07A91F8A44017EE39
:10DB7000900A034602B21CB14C68888721680A608B
:10DB800041F22011C1F2000191F8A50018B1886896
:10DB9000CB8701680A6041F22011C1F2000191F8BF
:10DBA000A60020B1C868A1F8403001680A6041F2BF
:10DBB0002011C1F2000191F8A70020B10869A1F875
:10DBC000423001680A6041F22011C1F2000191F86F
:10DBD000A80020B14869A1F8443001680A6041F208
:10DBE0002011C1F2000191F8A90020B18869A1F8C3
:10DBF000463001680A6041F22011C1F2000191F83B
:10DC0000AA0020B1C869A1F8483001680A6041F251
:10DC10002011C1F2000191F8AB0020B1086AA1F80F
:10DC20004A3001680A6041F22011C1F2000191F806
:10DC3000AC0020B1486AA1F84C3001680A6041F29A
:10DC40002011C1F2000191F8AD0020B1886AA1F85D
:10DC50004E3001680A6041F22011C1F2000191F8D2
:10DC6000AE0020B1C86AA1F8503001680A6041F2E4
:10DC70002011C1F2000191F8AF0020B1086BA1F8AA
:10DC8000523001680A6041F22011C1F2000191F89E
:10DC9000B00020B1486BA1F8543001680A6041F22D
:10DCA0002011C1F2000191F8B10020B1886BA1F8F8
:10DCB000563003681A6041F2201CC1F2000C0022A9
:10DCC000CCF89C20CCF8A02010BC704738B541F2AD
:10DCD0002015C1F200052DED068BD5ED283A9FEDFC
:10DCE000EEAA40F2B424C1F20004B0EE608AF0EE75
:10DCF000418AF0EE4A0A94ED401A30EE630AB0EE23
:10DD0000619A0AF0E3FD94ED413AD4ED422AF0EE37
:10DD1000409A33EE400AD4ED430A94ED441A20EEC3
:10DD2000220A0AF0D3FD40F22013C1F2000393ED62
:10DD3000442ADFEDDA1A93ED431A62EE217A95F860
:10DD4000A4202B6877EEC10AB7EE007A80EEA76AAE
:10DD500008EE008A36EE076A48EE808A09EE009ADD
:10DD6000D4ED3E6A94ED407AD5ED287A82B3D3EDB6
:10DD7000005A9FEDCB1A69EEA53A93ED013A03EEF6
:10DD800081AA68EE032A93ED020A02EE81AA28EE28
:10DD9000802AD3ED031A02EE01AA69EE210AF0EE01
:10DDA000664A00EE81AA4AEE064ABDEEE44A14EE47
:10DDB000100A01B205EE101AF8EEC55AA887F4EE63
:10DDC000475AF1EE10FA04BFDFEDB65A77EEA57AA6
:10DDD00041F22012C1F2000292F8A540A4B3D3EDA3
:10DDE000044A9FEDAF0A29EEA44ADFEDAB1A93ED8A
:10DDF000055A44EE001A68EE055AD3ED063A45EE90
:10DE0000801A28EEA33AD3ED072A43EE001A29EE32
:10DE1000222AB0EE661A42EE001A01EE861AFDEED4
:10DE2000C14A14EE90CA0FFA8CFE04EE10EAB8EE66
:10DE3000C45AA2F83EC0B4EE475AF1EE10FA04BF3D
:10DE40009FED985A77EE857A41F22012C1F20002D6
:10DE500092F8A60098B3D3ED081ADFED913A29EEB7
:10DE6000A11ADFED8D2AD3ED090A41EE232A68EECF
:10DE7000204A93ED0A4A44EEA32A28EE845AD3EDB1
:10DE80000B5A45EE232A29EE253AB0EE660A43EEF8
:10DE9000232A02EE860AFDEEC01A11EE901A0CB289
:10DEA00001EE104AF8EEC10AA2F84010F4EE470A5B
:10DEB000F1EE10FA04BFDFED7B0A77EEA07A41F2B3
:10DEC0002012C1F2000292F8A700A0B3D3ED0C2AF1
:10DED0009FED735A29EEA20ADFED6F5A93ED0D2ADA
:10DEE00040EE055A68EE021A93ED0E1A41EE855A7D
:10DEF00068EE810AD3ED0F4A40EE855A29EE244A96
:10DF0000F0EE663A44EE055A45EE863AFDEEE32A17
:10DF100012EE90CA0FFA8CF100EE101AB8EEC02A79
:10DF2000A2F842C0B4EE472AF1EE10FA04BF9FED0A
:10DF30005D2A77EE827A41F22012C1F2000292F855
:10DF4000A840A4B3D3ED105A9FED551A69EEA53A37
:10DF5000DFED510A93ED113A43EE810A68EE032A90
:10DF600093ED120A42EE810A28EE802AD3ED131AAD
:10DF700042EE010A69EE214AB0EE665A44EE810A89
:10DF800000EE865AFDEEC55A15EE90EA0FFA8EF0B5
:10DF900003EE900AB8EEE33AA2F844E0B4EE473A52
:10DFA000F1EE10FA04BF9FED3F3A77EE837A41F22B
:10DFB0002012C1F2000292F8A910A1B3D3ED140A05
:10DFC0009FED370A29EEA04ADFED331A93ED155A7B
:10DFD00044EE001A68EE055AD3ED163A45EE801A63
:10DFE00028EEA33AD3ED172A43EE001A29EE222A8F
:10DFF000B0EE661A42EE001A01EE861AFDEEC10A74
:10E0000010EE904A0FFA84FC05EE10CAB8EEC54A2D
:10E01000A2F84640B4EE474AF1EE10FA04BF9FED75
:10E02000214A77EE847A41F22012C1F2000292F87E
:10E03000AA0000283FD0D3ED181ADFED193A29EED7
:10E04000A11ADFED152AD3ED194A41EE232A68EE15
:10E05000240A93ED1A4A40EEA32A28EE845AD3EDFF
:10E060001B5A45EE232A29EE253AB0EE660A43EE06
:10E07000232A02EE860AFDEEC01A11EE90EA0FFA8C
:10E080008EF101EE101AF8EEC14AA2F848E0F4EE63
:10E09000474AF1EE10FA09E000000000CDCC6C40D8
:10E0A0000AD7233C9A99993E0000000004BF5FED17
:10E0B000034A77EEA47A41F22012C1F2000292F8EC
:10E0C000AB40A4B3D3ED1C2A1FED0B5A29EEA20AD4
:10E0D0005FED0B5A93ED1D2A40EE055A68EE021AC9
:10E0E00093ED1E1A41EE855A68EE814AD3ED1F0A60
:10E0F00044EE855A29EE204AF0EE663A44EE055A7F
:10E1000045EE863AFDEEE32A12EE90CA0FFA8CF045
:10E1100000EE100AB8EEC02AA2F84AC0B4EE472AB0
:10E12000F1EE10FA04BF1FED212A77EE827A41F258
:10E130002012C1F2000292F8AC10A1B3D3ED205A24
:10E140001FED291A69EEA53A5FED290A93ED213AF0
:10E1500043EE810A68EE032A93ED220A42EE810A19
:10E1600028EE802AD3ED231A42EE010A69EE214AF5
:10E17000B0EE665A44EE810A00EE865AFDEEC55AAC
:10E1800015EE904A0FFA84FE03EE90EAB8EEE33AF9
:10E19000A2F84C40B4EE473AF1EE10FA04BF1FED7E
:10E1A0003F3A77EE837A41F22012C1F2000292F8F0
:10E1B000AD00A0B3D3ED240A1FED470A29EEA04A13
:10E1C0005FED471A93ED255A44EE001A68EE055AA2
:10E1D000D3ED263A45EE801A28EEA33AD3ED272A4E
:10E1E00043EE001A29EE222AB0EE661A42EE001A19
:10E1F00001EE861AFDEEC10A10EE90CA0FFA8CF1FC
:10E2000005EE101AB8EEC54AA2F84EC0B4EE474A61
:10E21000F1EE10FA04BF1FED5D4A77EE847A41F209
:10E220002012C1F2000292F8AE40A4B3D3ED281A36
:10E230005FED653A29EEA11A5FED652AD3ED294A13
:10E2400041EE232A68EE240A93ED2A4A40EEA32ADF
:10E2500028EE845AD3ED2B5A45EE232A29EE253A8F
:10E26000B0EE660A43EE232A02EE860AFDEEC01ADD
:10E2700011EE90EA0FFA8EF001EE100AF8EEC14AA4
:10E28000A2F850E0F4EE474AF1EE10FA04BF5FED59
:10E290007B4A77EEA47A41F22012C1F2000292F892
:10E2A000AF10A1B3D3ED2C2A1FED835A29EEA20A99
:10E2B0005FED835A93ED2D2A40EE055A68EE021A5F
:10E2C00093ED2E1A41EE855A68EE814AD3ED2F0A5E
:10E2D00044EE855A29EE204AF0EE663A44EE055A9D
:10E2E00045EE863AFDEEE32A12EE904A0FFA84FCE0
:10E2F00000EE10CAB8EEC02AA2F85240B4EE472A87
:10E30000F1EE10FA04BF1FED992A77EE827A41F2FE
:10E310002012C1F2000292F8B000A0B3D3ED305A3F
:10E320001FEDA11A69EEA53A5FEDA10A93ED313A0E
:10E3300043EE810A68EE032A93ED320A42EE810A27
:10E3400028EE802AD3ED331A42EE010A69EE214A03
:10E35000B0EE665A44EE810A00EE865AFDEEC55ACA
:10E3600015EE90EA0FFA8EF103EE901AB8EEE33A4A
:10E37000A2F854E0B4EE473AF1EE10FA04BF1FEDF4
:10E38000B73A77EE837A41F22012C1F2000292F896
:10E39000B1408CB3D3ED343A1FEDBF5A29EEA33A06
:10E3A0005FEDBF0AD3ED352A43EE050A28EE220AB7
:10E3B00093ED362A40EE050A68EE821A93ED371A7D
:10E3C00041EE850A69EE014A44EE850A40EE866A0E
:10E3D000BDEEE64A14EE103A18B206EE100AF8EE58
:10E3E000C66AA2F85630F4EE476AF1EE10FA04BF9E
:10E3F0001FEDD47A77EE877A41F22014C1F200043F
:10E40000C4ED287AFFF734F940F2B422C1F20002D9
:10E41000D4ED285A92ED407A5FEDDE6AF6EE007A8E
:10E4200035EEE60A5FEDE00A27EE271A0AF04EFA0B
:10E4300084ED248A84ED280AC4ED258A84ED269A89
:10E44000C4ED279ABDEC068B38BD00BF10B540F671
:10E45000AC702DED048BC0F60200F4F779FA41F2AE
:10E4600020100021B422C1F200000FF04DFA40F25A
:10E47000B423C1F20003D3ED3D7A9FEDE67AF4EECA
:10E48000C77AF1EE10FA07DD9FEDE00AF4EEC07AEC
:10E49000F1EE10FA00F1738440F2B423C1F20003EC
:10E4A0009FEDDB8AD3ED457A41F22012C1F20002E2
:10E4B000F4EE487A03F58A71F1EE10FA116007D193
:10E4C00093ED462AB4EE482AF1EE10FA00F02C84BF
:10E4D00040F2B424C1F20004D4ED3E1ABCEEE11ABD
:10E4E000002011EE102A40F6C411034603F0B4FDDB
:10E4F00041F2201CDFEDC60AC1F2000CD4ED468AC1
:10E5000094ED479A94ED488ACCF8040078EEA08AFE
:10E51000012039EE209A38EE208A8CF8A40041F2CE
:10E52000201EC1F2000EDFEDBA7ADEF80040D4ED15
:10E53000043AF4EE673AF1EE10FA07D194ED056A69
:10E54000B4EE676AF1EE10FA00F0DD8340F2B42217
:10E55000C1F20002D2ED3E5ABCEEE55A40F6C411BB
:10E56000002315EE102A012003F076FD41F220135E
:10E57000C1F20003012183F8A510D4ED056AD4EDA2
:10E58000064A94ED074A78EEA68A39EE249A38EEC8
:10E59000048A986041F22010C1F20000DFED9C7AFD
:10E5A0000468D4ED080AF4EE670AF1EE10FA07D118
:10E5B00094ED093AB4EE673AF1EE10FA00F0928366
:10E5C00040F2B42EC1F2000EDEED3E2ABCEEE22A8D
:10E5D000002312EE102A022040F6C41103F03CFD85
:10E5E00041F2201CC1F2000C01238CF8A630D4EDBE
:10E5F000091A94ED0A1AD4ED0B7A78EEA18A39EE55
:10E60000019A38EE278ACCF80C0041F22014C1F2AE
:10E610000004DFED7F7A2468D4ED0C4AF4EE674AFB
:10E62000F1EE10FA07D194ED0D0AB4EE670AF1EE9F
:10E6300010FA00F0468340F2B420C1F2000090EDE1
:10E640003E7ABCEEC76A40F6C41116EE102A0320CB
:10E65000002303F001FD41F22011C1F2000101226B
:10E6600081F8A720D4ED0D6AD4ED0E5A94ED0F5A1F
:10E6700078EEA68A39EE259A38EE058A086141F2CD
:10E68000201CC1F2000CDFED627ADCF80040D4ED12
:10E69000101AF4EE671AF1EE10FA07D194ED114A50
:10E6A000B4EE674AF1EE10FA00F0FA8240F2B42EAE
:10E6B000C1F2000EDEED3E3ABCEEE33A40F6C41184
:10E6C000002313EE102A042003F0C6FC41F22013AD
:10E6D000C1F20003012183F8A810D4ED112A94EDB2
:10E6E000122AD4ED137A78EEA28A39EE029A38EE25
:10E6F000278A586141F22014C1F20004DFED447A08
:10E700002468D4ED145AF4EE675AF1EE10FA07D1EA
:10E7100094ED151AB4EE671AF1EE10FA00F0AF821C
:10E7200040F2B420C1F20000D0ED3E0ABCEEE00A97
:10E73000052010EE102A40F6C411002303F08CFCD3
:10E7400041F2201CC1F2000C01228CF8A920D4ED6A
:10E75000156A94ED167A94ED176A78EEA68A39EE6A
:10E76000079A38EE068ACCF8180041F22013C1F25D
:10E770000003DFED277A1C68D4ED182AF4EE672A2F
:10E78000F1EE10FA07D194ED195AB4EE675AF1EE92
:10E7900010FA00F0638240F2B42EC1F2000EDEEDFA
:10E7A0003E4ABCEEE44A40F6C41114EE102A06209C
:10E7B000002303F051FC41F22011C1F200010122BB
:10E7C00081F8AA20D4ED193A94ED1A3AD4ED1B7AC7
:10E7D00078EEA38A39EE039A38EE278AC86141F2AF
:10E7E0002014C1F20004DFED0A7A246894ED1C7A4B
:10E7F000B4EE677AF1EE10FA0ED194ED1D2AB4EE64
:10E80000672AF1EE10FA00F0188205E0EC51804022
:10E81000000000000AD7233C40F2B420C1F20000FF
:10E82000D0ED3E1ABCEEE11A002311EE102A0720AB
:10E8300040F6C41103F010FC41F2201CC1F2000CA0
:10E8400001238CF8AB30D4ED1D6AD4ED1E0A94ED93
:10E850001F0A78EEA68A39EE209A38EE008ACCF8A4
:10E86000200041F22011C1F200015FED177A0C681F
:10E87000D4ED203AF4EE673AF1EE10FA07D194EDB8
:10E88000216AB4EE676AF1EE10FA00F0C58140F239
:10E89000B42EC1F2000EDEED3E5ABCEEE55A082061
:10E8A00015EE102A40F6C411002303F0D5FB41F207
:10E8B000201CC1F2000C01228CF8AC20D4ED214ABE
:10E8C00094ED224AD4ED237A78EEA48A39EE049AA4
:10E8D00038EE278ACCF8240041F22014C1F200045B
:10E8E0005FED357A2468D4ED240AF4EE670AF1EE80
:10E8F00010FA07D194ED253AB4EE673AF1EE10FA2A
:10E9000000F0798140F2B420C1F20000D0ED3E2A3F
:10E91000BCEEE22A40F6C411002312EE102A0920B0
:10E9200003F09AFB41F22013C1F20003012183F8A6
:10E93000AD10D4ED256AD4ED261A94ED271A78EEA1
:10E94000A68A39EE219A38EE018A986241F2201C9B
:10E95000C1F2000C5FED527ADCF80040D4ED284A99
:10E96000F4EE674AF1EE10FA07D194ED290AB4EEFD
:10E97000670AF1EE10FA00F02D8140F2B42EC1F2D8
:10E98000000E9EED3E7ABCEEC76A002316EE102AFA
:10E990000A2040F6C41103F05FFB41F22013C1F2DC
:10E9A0000003012283F8AE20D4ED295A94ED2A5AAF
:10E9B000D4ED2B7A78EEA58A39EE059A38EE278ABF
:10E9C000D86241F22014C1F200045FED6F7A24682E
:10E9D000D4ED2C1AF4EE671AF1EE10FA07D194ED8B
:10E9E0002D4AB4EE674AF1EE10FA00F0E28040F2F0
:10E9F000B420C1F20000D0ED3E3ABCEEE33A40F65E
:10EA0000C411002313EE102A0B2003F025FB41F262
:10EA10002011C1F20001012381F8AF30D4ED2D6A3D
:10EA2000D4ED2E2A94ED2F2A78EEA68A39EE229A7A
:10EA300038EE028A086341F2201CC1F2000C5FED3F
:10EA40008C7ADCF80040D4ED305AF4EE675AF1EEDF
:10EA500010FA07D194ED311AB4EE671AF1EE10FAFC
:10EA600000F0968040F2B42EC1F2000EDEED3E0AB8
:10EA7000BCEEE00A40F6C41110EE102A0C20002370
:10EA800003F0EAFA41F2201194ED317A94ED326A02
:10EA9000D4ED337AC1F20001012278EE878A39EE93
:10EAA000069A38EE278A486381F8B02041F2201494
:10EAB000C1F200045FEDAA7A2468D4ED342AF4EEA2
:10EAC000672AF1EE10FA06D1D4ED356AF4EE676AE2
:10EAD000F1EE10FA4DD040F2B42CC1F2000CDCED96
:10EAE0003E7AFCEEE75A002315EE902A0D2040F600
:10EAF000C41103F0B1FA41F22013C1F2000394ED06
:10EB0000355AD4ED364A94ED374A986378EE858AC3
:10EB1000012039EE249A38EE048A83F8B100B0EE71
:10EB2000680A0EF0AFFC1FEDC56AB4EEC60AF1EE3E
:10EB300010FA00F31D81B0EE490A0EF0A3FC1FEDA0
:10EB4000CB7AB4EEC70AF1EE10FA00F30A81B0EE08
:10EB5000480A0EF097FC5FEDD10AB4EEE00AF1EE40
:10EB600010FA00F3F780BDEC048BBDE81040FEF70F
:10EB7000EFBF94ED363AB4EE673AF1EE10FAAAD14F
:10EB8000D4ED373AF4EE673AF1EE10FAC7D0A2E7C7
:10EB9000D4ED321AF4EE671AF1EE10FA7FF462AF98
:10EBA00094ED332AB4EE672AF1EE10FA7FF45AAFEF
:10EBB0007CE7D4ED2E4AF4EE674AF1EE10FA7FF4CA
:10EBC00016AF94ED2F5AB4EE675AF1EE10FA7FF4B7
:10EBD0000EAF30E7D4ED2A0AF4EE670AF1EE10FA30
:10EBE0007FF4CBAE94ED2B1AB4EE671AF1EE10FA67
:10EBF0007FF4C3AEE5E6D4ED263AF4EE673AF1EEE3
:10EC000010FA7FF47FAE94ED274AB4EE674AF1EE36
:10EC100010FA7FF477AE99E694ED227AB4EE677A33
:10EC2000F1EE10FA7FF433AE94ED230AB4EE670AE6
:10EC3000F1EE10FA7FF42BAE4EE6D4ED1E2AF4EE80
:10EC4000672AF1EE10FA7FF4E7AD94ED1F3AB4EEC7
:10EC5000673AF1EE10FA7FF4DFAD02E6D4ED1A5A0E
:10EC6000F4EE675AF1EE10FA7FF495AD94ED1B6A5D
:10EC7000B4EE676AF1EE10FA7FF48DADAFE5D4ED36
:10EC8000161AF4EE671AF1EE10FA7FF449AD94ED1E
:10EC9000172AB4EE672AF1EE10FA7FF441AD64E56D
:10ECA000D4ED124AF4EE674AF1EE10FA7FF4FEACAE
:10ECB00094ED135AB4EE675AF1EE10FA7FF4F6AC05
:10ECC00018E5D4ED0E0AF4EE670AF1EE10FA7FF4BF
:10ECD000B2AC94ED0F1AB4EE671AF1EE10FA7FF4AD
:10ECE000AAACCCE4D4ED0A3AF4EE673AF1EE10FAAD
:10ECF0007FF466AC94ED0B4AB4EE674AF1EE10FA7D
:10ED00007FF45EAC81E494ED067AB4EE677AF1EEBE
:10ED100010FA7FF41BAC94ED070AB4EE670AF1EE2B
:10ED200010FA7FF413AC35E4D3ED472AF4EE482A09
:10ED3000F1EE10FA7FF4CCAB93ED483AB4EE483ADA
:10ED4000F1EE10FA7FF4C4ABB0EE489AF0EE488AC8
:10ED5000FFF7E5BB41F25000C0F60200F3F7F8FD03
:10ED600001E741F22800C0F60200F3F7F1FDEEE6FC
:10ED700040F6FC70C0F60200F3F7EAFDDBE640F671
:10ED8000BC70C0F60200BDEC048BBDE81040F3F788
:10ED9000DFBD00BF10B540F64563C2F2000341F687
:10EDA00024721C78C2F20002601C1478C1B2092CD3
:10EDB000197004D9FF24FAF73FFB204610BD631CED
:10EDC0001370FAF739FB41F6D462C2F2000202EB8B
:10EDD000C40CFF2100208CF80100CCF804008CF852
:10EDE000031002F834108CF80210204610BD00BF4A
:10EDF000F8B540F64461C2F200010B780BB1032074
:10EE0000F8BD40F64563C2F200031A780AB1152036
:10EE1000F8BD42F27044C2F2000441F6D4622468A4
:10EE20001978E071C2F2000202EBC0054E1C69784D
:10EE3000F6B21E7061B9217902F83010A279AA7079
:10EE4000A3790120EB706870FAF7F6FA0020F8BD9C
:10EE50000129F9D1AE78227942F2744E06EB860C84
:10EE6000C2F2000E0EEBCC063079904212D9A17995
:10EE700073793271E97033B3337AFF2B0AD040F6DD
:10EE80004C67C2F2000707EB0317787900F0F00235
:10EE9000202A1FD00223637140F6466C6A68C2F2D2
:10EEA000000C002101208CF80000216261620AB987
:10EEB00007E01A46136A002BFBD1146262622362D8
:10EEC000C2E76C60C0E7304608F028FD304608F025
:10EED000E7FCDFE73046FAF771FC38463146FAF7CF
:10EEE000CDFBD7E770B540F64461C2F200010B7864
:10EEF0000BB1032070BD41F6D464C2F2000404EBF0
:10EF0000C00440F6456CC2F2000CA0789CF80010DA
:10EF1000666842F2744200EB8003C2F200024D1CAC
:10EF200002EBC302EDB2FF218CF80050D171002E2C
:10EF300028D0E578854217D01579FF22A270217874
:10EF400008F00AFD6368196A61601E792670987975
:10EF50000026A07018461D711E625E6208F0A0FCBB
:10EF6000FAF76AFA304670BD3579366A002EE4D079
:10EF700033799D42F9D9B279E270366A1D46002E86
:10EF8000F6D1DAE76670A170FAF756FA304670BD2E
:10EF900038B5026AC47941F6D463C2F2000303EBC8
:10EFA000C404436A002A22D053621BB1416A002381
:10EFB0000A6243620362FF23C371E278807982426E
:10EFC00000D038BDA57863682178E57043B11A791F
:10EFD000914202D998791146E0701B6A002BF6D154
:10EFE000FF222846A27008F0B7FCA57038BD13B107
:10EFF0001A624262DFE76360DDE700BF41F2D813C7
:10F00000C1F20003D3ED010A70EE807AC3ED017AFC
:10F01000704700BF10B52DED028BB0EE408A0CF0AA
:10F0200063FF40B941F2D813C1F2000383ED038AB4
:10F03000BDEC028B10BD41F2D814C1F2000494ED76
:10F04000040A38EE000AF8F707FF84ED030AEFE739
:10F050002DE9F00141F2600241F62875C2F2000587
:10F06000C1F2000241F2D813C1F2000392ED0E6B1F
:10F0700040F2B42703210026C1F20007D5F83C0472
:10F0800083F82D1583F82C6505F58064D7ED817A1A
:10F0900003F5A06CD0F84080D7F8FC6165688CED72
:10F0A000006B92ED106B03F5A26103F5A464F5EE1D
:10F0B000407A03F5A167F1EE10FAC1F8008087ED00
:10F0C000006BCE60656007D090ED107A77EE877A9E
:10F0D00003F5A863C3ED007ABDE8F001704700BFF7
:10F0E00010B541F2D814C1F2000404F5A06104F592
:10F0F000A16091ED000B90ED001B01F051FA94F826
:10F100002C3504F5A262D2ED007A002B39D094EDB3
:10F11000017A77EE877AC4ED017A41F2D814C1F210
:10F12000000404F5A46E04F5A263DEF800C0DA68FA
:10F13000C4F81CC09EED010AA261FFF76BFF94EDBD
:10F14000060AB5EE400AF1EE10FA06D140F2B421FB
:10F15000C1F20001D1F8FC01A06141F2D813C1F263
:10F160000003D3ED070AF5EE400AF1EE10FA07D1DD
:10F1700040F2B422C1F20002D2F854C2C3F81CC05B
:10F1800010BDC4ED017AC8E72DE9F84F41F2D8135C
:10F190002DED028BC1F2000300EB400103EB0111E6
:10F1A000044691F87D20551EEDB2042D63D891F8E8
:10F1B0007C00002856D1964ED1ED181A96ED001A13
:10F1C00071EEC10AC3ED010A41F2D815C1F2000582
:10F1D00004EB440305EB031696ED1B8AD6ED1C8A5F
:10F1E000012A85ED068AC5ED078A48D0032A72D028
:10F1F000042A00F09380022A00F0D380052A00F050
:10F20000C280B5EE408AF1EE10FA0BD140F2B42282
:10F21000C1F2000241F2D813D2F8FCC1C1F20003DE
:10F22000C3F818C0F5EE408AF1EE10FA0AD140F2A8
:10F23000B42CC1F2000C41F2D810DCF85412C1F227
:10F240000000C16141F2D813C1F200030022204640
:10F25000C3F8302583F83A45BDEC028BBDE8F84F82
:10F26000F3F72ABC93ED010A91ED187A77EE007A54
:10F27000C3ED017AA8E7BDEC028BBDE8F88F95F8E5
:10F280002C1505F5A262D2ED007A002978D0D5EDD3
:10F29000012A37EEA22A85ED012A41F2D815C1F2E2
:10F2A000000505F5A06105F5A16E91ED000B9EED41
:10F2B000001B01F075F905F5A46C05F5A263DCF8F7
:10F2C000040093ED038ADCED008AA86085ED068AD0
:10F2D000C5ED078A95E7D6E914AB4FF000084FF06B
:10F2E00000095046594642464B460CF0C9FD48B904
:10F2F000D6E9166742464B46304639460CF0C0FD0B
:10F30000002879D041F2D810C1F2000004EB440388
:10F3100000EB031CDCF87420826072E7D6E914ABC2
:10F320004FF000084FF000095046594642464B4600
:10F330000CF0A6FD80B9D6E9166742464B4630462A
:10F3400039460CF09DFD38B94BEC10AB47EC116B16
:10F3500001F026F9D5ED078A41F2D81EC1F2000E60
:10F3600004EB440340F2B4220EEB0310C1F200029E
:10F37000416F92ED7F8ACEF808108EED068A40E745
:10F38000C5ED017A89E7F5EE408AF1EE10FA7FF4D7
:10F3900038AF4FF2C350C3F6A860E86108EE900A98
:10F3A0002FE741F2600EC1F2000E9EED0E0B9EEDB6
:10F3B000101B01F0F5F896ED1C3A1649B5EE403AEF
:10F3C000DFED153A4B68F1EE10FA08BFB0EE633A84
:10F3D000AB6085ED073AFFF73BFE686805F5A26272
:10F3E00005F5A46C4FF000411060CCF8041095EDC9
:10F3F000068AD5ED078A04E74BEC10AB47EC116B9E
:10F4000001F0CEF895ED068AD5ED078A7AE700BFC0
:10F410006823002028230020C3F5A83E2DE9F843E7
:10F4200040F220122DED028B41F26003C1F2000385
:10F43000C1F200029E6AD2F88041D3F89850306839
:10F44000B68841F2D81244F23F21671BC1F2000294
:10F45000C0F20F018F4292F83A55468309D893EDD6
:10F46000137AF0EE087AB4EEE77AF1EE10FA00F1D2
:10F470005A8141F2D813C1F2000393F838050128EC
:10F4800040F2CE8393F83975002F40F0508140F25E
:10F49000B426C1F20006D6ED072ABDEEE22A12EE2E
:10F4A000102A41F6380E101DC1F2000E3EF9102050
:10F4B00012F1F90380F26B8141F6287641F2D81CF3
:10F4C000C2F20006C1F2000C0025D6F83C348CF8DC
:10F4D00038558CF83A55186CCCF8040041F2D81322
:10F4E000C1F2000303F5A867D7ED007AF5EE407A84
:10F4F000F1EE10FA1DD041F62872C2F20002D2F8E5
:10F500003C1491ED107AF4EEC77AF1EE10FA40F166
:10F51000E98293F83C05002840F0CF824FF4406E1A
:10F52000C4F2000E012783F83C75DEF8246083F8EE
:10F530003E6540F2B423C1F2000393ED083AFDEEBC
:10F54000C32A41F6380C12EE907AC1F2000C3E1D2F
:10F550003CF91630FA2B00F3E382FA33C0F25D83F4
:10F5600041F62870C2F20000DFEDB97AD0F83C1401
:10F57000D1ED030AF4EE670AF1EE10FA91ED040AF8
:10F5800040F0ED81B4EE670AF1EE10FA40F0E78149
:10F5900041F2D816C1F2000641F2D81E96F838356D
:10F5A000C1F2000E042BCEED047ACEED057A00F008
:10F5B0000382032B00F0B782042B00F0508241F647
:10F5C0002877C2F2000741F2D816C1F20006D7F838
:10F5D0003C34306C9FED9E8AD3ED030AB0EE480AAE
:10F5E00002F0A8FAD7F83C74706C86ED080AD7EDE3
:10F5F000040AB0EE480A02F09DFAF0EE407AC6ED39
:10F60000097A96ED080AD6ED066A27EEA71A00EEEB
:10F61000001AB1EEC17AF4EEC76AF1EE10FA0FD516
:10F6200080EE070A41F2D81EC1F2000EC7EE877ABB
:10F6300026EE800A26EEA77A8EED080A8EED097A6C
:10F6400041F62877C2F2000741F2D816C1F200064F
:10F65000D7F83C24B06BD2ED000A02F06BFAF1EE61
:10F66000401AC6ED0A1AD7F83C14F06B96ED090A59
:10F67000D1ED010A02F05EFA96F8383586ED0B0AF4
:10F68000002B00F0B88140F2B421C1F2000191EDED
:10F69000023AFDEEC32A41F6380E12EE902AC1F26C
:10F6A000000E171D91ED177A3EF917C0ACF52F70BB
:10F6B00002EE100AF8EEC27AB4EEE77AF1EE10FA32
:10F6C00040F1D08096F83D65002E40F0CB80F5EEFD
:10F6D000C07A40F2B422F1EE10FAC1F2000200F357
:10F6E000B882D2ED800A37EE875ADFED5A4A25EE0E
:10F6F000206A41F2D81C26EE240AC1F2000C8CEDDF
:10F700000D0A042B00F0CC8341F6287EC2F2000ED5
:10F7100041F2D817DEF83C24C1F20007116C97EDD6
:10F72000071A7960D0E00123068382F8393540F268
:10F73000B422C1F20002D2ED071ABDEEE11A41F681
:10F74000380E11EE102AC1F2000E131D3EF913609F
:10F75000FA2E7FF7A6AE41F2D816C1F2000696F84F
:10F76000380502287FF4BAAE182D3FF6B7AE05EB88
:10F77000450706EB071C9CF87D1000293FF4AEAE50
:10F780002846FFF701FD042386F83835A6E641F246
:10F79000D816C1F2000696F83815002900F0448307
:10F7A00041F2D816C1F2000696F8390500283FF458
:10F7B00095AE96F83815022900F07E82032900F0F4
:10F7C0007B8241F26003C1F2000393ED0E0B93EDD7
:10F7D000101B00F0E5FE4FF0000806F5A0634FF0A7
:10F7E0000009D3E9000142464B460CF049FB0028D2
:10F7F00040F0A18306F5A166D6E9000142464B46DA
:10F800000CF03EFB002840F0968341F2D816C1F27E
:10F81000000696F83825012A40F22A8440F2B420E6
:10F82000C1F2000041F2D81EC1F2000ED0F8FCC1B6
:10F83000D0F85472CEF818C0022641F29000C0F6FB
:10F840000200CEF81C708EF83865F3F781F845E6B3
:10F8500000000000E73EBB3A0AD7233C0000B44258
:10F86000E02E6542F1EE473AF4EEE73AF1EE10FA97
:10F870003FF72DAF042B0CD141F2D813C1F2000396
:10F8800005EB450703EB071090F87D60052E00F0AF
:10F89000928341F62872C2F2000241F2D816C1F2F8
:10F8A0000006D2F83C14F06CD1ED100A96ED010A76
:10F8B00002F040F940F2B423C1F2000386ED0D0AD4
:10F8C00096ED071AD3ED800AF4EEC10AF1EE10FAB4
:10F8D000CCBFF1EE410AF1EE600A41F2D81608F011
:10F8E000F5FFC1F2000696ED0C1A1FED257A70EEB9
:10F8F000417A96F8382507EE871A042A86ED0D0A14
:10F9000086ED0C1A78D105EB450006EB001EDEED06
:10F910001E7AF5EE407AF1EE10FA6DD041F6287CB1
:10F92000C2F2000C96ED050ADCF83C7497ED104A23
:10F9300074EE673A23EEA33A00EE003AF1EEC32AE2
:10F9400080EE220A0CF0DAFF96F838255FED3D1ABA
:10F950001FED3D2A50EE021AC6ED001A52E0F1EEFC
:10F96000600AB1EE400A0DF063F85FED434A20EE05
:10F97000240AF8F771FA41F62876C2F2000641F23D
:10F98000D81CC1F2000C8CED040AD6F83C2492ED90
:10F99000046A92ED034A66EE063A44EE043AF1EE4A
:10F9A000E35A41F2D816C1F20006CCED055A96F89A
:10F9B0003835042B7FF4FDADD6F83035002B40F000
:10F9C0005B8105EB450706EB07132F4693F87D3067
:10F9D000032B00F06C82012B00F06982042B00F0F5
:10F9E0001483022B00F0AA8241F2D81EC1F2000E4D
:10F9F0009EF83835DDE51A4641F2D813C1F200030E
:10FA000000261E60042A00F0DA8141F2600500261B
:10FA10000027C1F20005D5E90E0132463B460CF045
:10FA20002FFA90B9D5E9100132463B460CF028FA7E
:10FA300058B941F2D813C1F2000393F839150029DF
:10FA400040F0B981022083F83B0541F2D81CC1F295
:10FA5000000CCCF83445BDEC028BBDE8F88341F2D4
:10FA6000D816C1F2000605EB450C06EB0C1797F80B
:10FA70007D0004287FF4A3ADD6ED050A306C97ED28
:10FA8000190A02F057F8E04A97ED1B5AD2ED014AE5
:10FA9000B1EE406AF1EE450AD2ED005A24EEA00A1A
:10FAA00066EE247A15EE860A40EEA57A86ED080AFF
:10FAB000C6ED097AD6ED066AA7E54FF44062C4F2B6
:10FAC000000293F83E15506AC1EB000C02EE10CA1A
:10FAD000DFEDCE1AB8EE421AB4EEE11AF1EE10FAEA
:10FAE00000F30F8241F2D813C1F20003B3F83C15C2
:10FAF00000293FF41EADF4EEC77AF1EE10FAFFF6DE
:10FB000018AD93F83D05002840F0628241F2D81EFE
:10FB1000C1F2000E00228EF83C258EF83D2508E546
:10FB2000FFF796FA1CE540F2B427C1F2000797ED03
:10FB3000044AFDEEC46A41F6380E16EE901AC1F280
:10FB4000000E0B1D97ED161A3EF91300AE4F03EE93
:10FB5000900A41F2D812F8EEE32AC1F2000240F214
:10FB6000B42CF4EEC12AD2ED066A9FEDA93AC1F297
:10FB7000000CF1EE10FA9CED032AC8BF72EEC15AD8
:10FB800026EE830AF1EE417AF4EEE72AFDEEC21A80
:10FB9000CCBF65EEC05ADFEDA35AF1EE10FA48BFB4
:10FBA00072EE812A11EE906A41F6380348BF62EE88
:10FBB000C05AC1F20003311D97ED015A33F911E02B
:10FBC00000EE90EAB8EEE07AD7ED004AB4EEC71A3C
:10FBD000F1EE10FA48BF77EE410AF4EEC77A4CBF57
:10FBE00060EE800ADFED8F0AF1EE10FAC8BF31EE49
:10FBF000071A65EE857AC8BF61EE000A41F2D81295
:10FC000025EE200A14EEA50A40EEA47AC1F2000205
:10FC100082ED080AC2ED097AF7E4FFF761FA9FE482
:10FC200040F2B42CC1F2000CDCED070ABDEEE00A94
:10FC300041F6380E10EE102AC1F2000E101D002100
:10FC40003EF9102083F8391512F1F903FFF634ACB0
:10FC50009DE5D2ED950A77EEC75ADFED6E6A25EE87
:10FC6000A04A41F2D81024EE260AC1F2000080ED2D
:10FC70000D0AD2ED800A44E59C427FF6F0AE05EB1A
:10FC8000450706EB071E9EF87D20052A3FF4E7AEE8
:10FC90000135EDB2182D00F2458105EB450106EB6B
:10FCA000011C9CF87D30002B00F03C812846FFF7BA
:10FCB0006BFA96F838357CE440F2B423C1F20003C5
:10FCC00093ED045AFDEEC54A41F6380214EE900A4F
:10FCD000C1F20002071DD3ED167A32F9176006EE65
:10FCE000106AB8EEC67AB4EEE77AF1EE10FA59DC93
:10FCF000F1EE676AB4EEE67AF1EE10FA52D4D3ED83
:10FD0000030ABDEEE00A10EE107A3E1D32F91630FD
:10FD100007EE103AB8EEC77AF4EEC77AF1EE10FAB1
:10FD200040D4F4EEC76AF1EE10FA3BDC03297FF40D
:10FD3000D5AB41F6287EC2F2000E9FED377ADEF891
:10FD40003C34D3ED007AF4EEC77AF1EE10FA40F1CC
:10FD50004681DFED326AF4EEE67AF1EE10FA40F316
:10FD60003E81D3ED017AF4EEC77AF1EE10FA40F15C
:10FD70003681F4EEE67AF1EE10FA40F3308141F28A
:10FD8000600EC1F2000E9EED0E0B9EED101B00F0FA
:10FD900007FC41F2D812C1F20002022182F83815A4
:10FDA000FFF79CBB41F2D812C1F20002032182F896
:10FDB0003815FFF793BB032283F83B2545E641F254
:10FDC000D817C1F2000797ED020AFFF723F905EBF8
:10FDD000450207EB021191F87D50052D7FF415AE19
:10FDE00040F2201EC1F2000EDFED0D5ADEF8400198
:10FDF00006EE900AF4EEE56AF1EE10FA7FF505AE34
:10FE000007F092F801E600BF382300208096984A58
:10FE10006F12033BE73EBB3ACDCCCC3DCDCCCCBD45
:10FE20000F5C6BC10000000041F62877C2F20007AA
:10FE300041F2201CD7F83C34B06CD3F840E093ED8D
:10FE4000024AC1F2000CB1EE440ADCED270AC6F802
:10FE500004E001F055FFD7F83C14F06C5FED0F0A99
:10FE600091ED100A01F04CFFD7F83C2440F2B42386
:10FE7000C1F20003D2ED023AD3F854C2B1EE633AB4
:10FE8000012741F27800C0F6020086ED0D3A86EDBA
:10FE90000C3AC6F81CC086F83875F2F759FD7FE4B5
:10FEA00041F2D813C1F2000393ED071A0CE541F2B9
:10FEB000D812C1F2000207EB470102EB011892EDE4
:10FEC000055A98ED197AB4EEC75AF1EE10FA7FF59B
:10FED00085AD41F6287CC2F2000C92ED010ADCF8F7
:10FEE0003C04D0ED106A30EE660A0DF0CBFAD8ED86
:10FEF000190AB4EEE00AF1EE10FA49D498F87D3010
:10FF00006CE5566A93F83D2583F83E65002A00F0BB
:10FF1000A88041F2D813C1F20003012783F83D7590
:10FF2000FFF707BB41F2D810C1F20000022680F8AB
:10FF30003865FFF744BBFFF78BF866E441F2D8164B
:10FF4000C1F2000607EB470006EB001808F1600855
:10FF500096ED053AD8ED013AB4EEE33AF1EE10FA37
:10FF60007FF5A7AE41F6287CC2F2000C96ED014A5F
:10FF7000DCF83C2492ED106A34EE460A0DF082FA69
:10FF8000D8ED015AB4EEE50AF1EE10FA7FF591AE24
:10FF900041F2D816C1F2000607EB470006EB00114C
:10FFA00028468B6E1F19C6F83075F2F7D9FC96F803
:10FFB0003835FFF7FEBA93ED071A40F2B42CB1EED4
:10FFC000410AC1F2000C83ED0D0ADCED800A7BE4EE
:10FFD00041F2CC00C0F60200F2F7BAFC96E540F21E
:10FFE000B427C1F20007D7ED087AFDEEE76A41F6C3
:10FFF000380C16EE906AC1F2000C331D3CF9130068
:020000040801F1
:1000000010F1FA03BFF66AAAB9E641F2D816C1F2B6
:10001000000607EB470106EB011896ED058AD8EDBF
:10002000192A38EE620A0DF02DFA41F62873C2F251
:100030000003D6ED011AD3F83C2492ED102AB0EE5D
:10004000408A31EEC20A0DF01DFA38EE001AF0EEC9
:10005000007AB4EEE71AF1EE10FA99D498F87D30F0
:10006000BFE441F2A800C0F60200F2F771FC50E7CD
:1000700041F628771FED958AC2F2000786ED0A8ABD
:10008000D7F83C24B06B86ED0B8AF0EE480A92ED6F
:10009000000A01F035FED7F83C34F06B93ED010A0D
:1000A000F0EE480A01F02CFED7F83C14306C91EDCC
:1000B000030AF0EE480A01F023FE706CD7F83C64A6
:1000C000F0EE480A96ED040A01F01AFEFFF7A6BB0F
:1000D0002DE9F04F41F2FC00654E41F2D81589B090
:1000E0000024C1F20005C0F60200F2F731FC371D12
:1000F00021464FF4A96228460DF006FC06F10809D6
:1001000006F10C0A06F1100B39462246234630460A
:100110008DE800060294CDF80CB004940594069482
:10012000079401F0E9FC39468646224623463046CC
:10013000C5F838E08DE800060294CDF80CB00494C0
:1001400005940694079401F0D7FC06F1200806F107
:100150001C07844606F118018DE8800122462346DB
:1001600006F114000837C5F83CC0039702940494C4
:1001700005940694079401F0BFFC083F814606F100
:1001800018018DE880012246234606F11400083745
:10019000C5F840900397029404940594069407943C
:1001A00001F0AAFC06F1380706F1300C06F1340E16
:1001B000804606F12C0106F12800224623468DE8F0
:1001C0000050C5F844800397029404940594069463
:1001D000079401F091FC06F1480906F1440C8646AB
:1001E00006F14001234606F13C00224641F62877FD
:1001F0004C36CDF800C0C2F20007C5F848E0CDF893
:10020000049002940396049405940694079401F0D4
:1002100073FC05F5A86107F580624FF0000892EDC8
:10022000010AC1F80080E86485F83C4585F83D4541
:1002300085F83845FEF7EEFED7F83C344CF6CD4C49
:100240000120C3F6CC5C1A6C85F87D00C5F864C04B
:10025000196C6A604FF07E500523A967C5F89C00B1
:10026000C5F8A880AC6685F8AD3009B0BDE8F08F60
:10027000BC04001041F2D813C1F20003002093F82F
:100280007D2082B10120303307E093F8AD200130AA
:10029000603332B10130192804D093F87D10002961
:1002A000F3D170477047704741F2D813C1F2000391
:1002B00093F83825042A10D0002203F5966083F8BD
:1002C0007D20303303F1300183F87D206033834299
:1002D00081F87D20F6D1012070470020704700BFD3
:1002E00041F2D813C1F2000300EB400003EB001011
:1002F0005030704700487047D816001090ED001A33
:10030000FDEEC10A92ED007A10EE90CA01EB8C006E
:1003100090ED090A77EE407AC3ED007A704700BF8E
:1003200091ED107A92ED000A77EE007AC3ED007A33
:10033000704700BFD1ED101A92ED001A71EE810ADC
:10034000C3ED000A91ED057A92ED010A77EE007A8D
:10035000C3ED017A704700BF91ED033AD2ED002A58
:1003600033EE222A83ED002AD1ED041A92ED011A10
:1003700071EE810AC3ED010A91ED057A92ED020A50
:1003800077EE007AC3ED027A704700BF91ED003A34
:10039000D2ED002A33EE222A83ED002AD1ED011A94
:1003A00092ED011A71EE810AC3ED010A91ED027A14
:1003B00092ED020A77EE007AC3ED027A704700BF31
:1003C0009FED081A08B5DFED080A80EE010A0CF06F
:1003D00033FEF7EE007A37EEC00A9FED047A20EE86
:1003E000070A08BD80E6C5475C8F423E2B2A2D4791
:1003F00041F62870C2F2000000F58862D0F83C3463
:10040000D3ED100A70EE607AC2ED007A704700BF3B
:100410002DE9D0432EA3D3E900232DED048B51EC1D
:10042000100B0BF03BFB41EC100B41EC190B0CF0EB
:10043000FFFE51EC100B02460B460BF02FFB26A3E0
:10044000D3E900230BF02AFB0B4600210246C3F63A
:10045000F07100200BF0DCF99FED1B1B41EC100B41
:1004600041EC180B0CF0ECFC1DA1D1E9000153ECA0
:10047000102B0BF0C9FBB0EE480AF0EE680A41F60B
:100480002874C2F20004C4E90C010CF0C5FF57EC5B
:10049000106BB0EE490AF0EE690A0CF02DFB59EC36
:1004A000108B32463B4610A1D1E900010BF0ACFBAA
:1004B00042464B460BF0F2FAC4E90E01BDEC048B48
:1004C000BDE8D083AFF30080000000000000F83FDB
:1004D000000000A046DF913F00000000916B7B3FD1
:1004E0002CF52966E4FEFA4080D6C1D6772DFB4074
:1004F00041F62873C2F2000370B403F1400103F126
:10050000E002F0EE407A03F5C073002691ED006A38
:1005100076EE275A0D46E5EC015A92ED005A75EE3B
:10052000204A1446E4EC014A93ED004A74EE013A85
:100530001846E0EC013A91ED013A73EE272A0236B3
:10054000C1ED012A92ED012A72EE201A291DC2ED99
:10055000011A93ED010A30EE017A221D83ED017A32
:10056000031D282ED2D141F62872C2F20002B0EE4D
:10057000410AD2F83C14D1ED031AD1ED046A91ED91
:10058000057A71EEA77A76EEA00A37EE011AC1ED70
:10059000037AC1ED040A81ED051A70BCFEF72EBD89
:1005A0002DE9D04F41F62874C2F200042DED028BE4
:1005B00057EC106BD4E90CAB82B0D4E90823304679
:1005C000394659EC118B0BF023F952465B460BF080
:1005D00065FA0BF0E1F894ED0E7BD4E90A2308EEFE
:1005E000100A494640468DED007B0BF011F9DDE91C
:1005F00000230BF053FA0BF0CFF8324608EE900AC6
:100600003B4630463946C4E90867C4E90A890BF01D
:10061000FFF802460B46504659460BF03FFA0BF0E6
:10062000BBF807EE900A42464B464046494637EE35
:10063000C88A0BF0EDF802460B46DDE900010BF02D
:100640002DFA0BF0A9F800EE900A9FED061A70EE55
:10065000E80AB0EE480A02B0BDEC028BBDE8D04F0C
:10066000FFF746BF00000000D1ED014A91ED003ACE
:1006700064EEA43A43EE033A91ED024A44EE043AA2
:10068000D1ED036A46EEA63AB1EEE30AC3EE002AC4
:10069000C0ED002A91ED012AC2EE001AC0ED011A48
:1006A00091ED021AC1EE000AC0ED020A91ED037A43
:1006B000C7EE007AC0ED037A704700BF92ED026A80
:1006C00092ED005A76EE067AD2ED035A91ED023A97
:1006D00067EE856AD1ED004A25EE054A75EEA52A3A
:1006E00026EE837A04EE247A91ED012A62EE853AB1
:1006F000D2ED016A03EEC27A66EEA63A66EEA70A6A
:1007000004EEA37A02EE207A66EEA21A25EEA52A5E
:1007100003EE217A04EEC27A26EE063A76EEA61AA7
:1007200004EEC37A21EE861A80ED007AD1ED014AFB
:10073000D1ED000A23EE247A01EE207A26EE220A79
:1007400091ED021A75EE052A00EE017A22EEA50A55
:1007500025EE215A00EE807A02EE647A04EE247AC5
:1007600001EE457A03EEE47A25EEA70A80ED017AE0
:1007700091ED015AD1ED004A65EEA15A60EE057A7D
:1007800045EEA47A91ED027A42EE077A26EE226ACD
:1007900066EEA26A44EEC67A43EE477A45EE267AC2
:1007A00043EEC77A44EE077AC0ED027A704700BF85
:1007B00000B592ED011AD2ED020A92ED030A85B05E
:1007C0001368F1EE416AB1EE607AF1EE407A6A4662
:1007D0000093CDED016A8DED027ACDED037AFFF73E
:1007E0006DFF05B000BD00BF38B51C4601F13003F8
:1007F000154620460E491A46FFF7DAFFD5ED002AC6
:1008000094ED003A33EE222AD4ED011A84ED002A49
:1008100095ED011A71EE810A94ED027AC4ED010A98
:1008200095ED020A77EE007AC4ED027A38BD00BF7A
:10083000381F002038B51C4601F13003154620460C
:100840000E491A46FFF7B4FFD5ED002A94ED003AA1
:1008500033EE222AD4ED011A84ED002A95ED011A17
:1008600071EE810A94ED027AC4ED010A95ED020A57
:1008700077EE007AC4ED027A38BD00BF2C1F00204D
:10088000D2ED010A91ED010AD2ED006A91ED007AF4
:1008900020EE805A06EE875AD1ED027AD2ED025A46
:1008A00005EEA75A80ED005AD2ED044A91ED014AB7
:1008B00092ED033AD1ED003A64EE841A43EE231A26
:1008C00092ED052AD1ED022A42EE221AC0ED011A5C
:1008D00092ED076A91ED011A92ED060AD1ED000A38
:1008E00066EE017A40EE207AD2ED086A91ED027A46
:1008F00046EE877AC0ED027A704700BFD2ED030A58
:1009000091ED010AD2ED006A91ED007A20EE805A55
:1009100006EE875AD1ED027AD2ED065A05EEA75AB5
:1009200080ED005AD2ED044A91ED014A92ED013A70
:10093000D1ED003A64EE841A43EE231A92ED072AB1
:10094000D1ED022A42EE221AC0ED011A92ED056A9B
:1009500091ED011A92ED020AD1ED000A66EE017ADC
:1009600040EE207AD2ED086A91ED027A46EE877A5F
:10097000C0ED027A704700BF91ED007AD1ED015AC7
:1009800091ED026AD1ED036A27EE077A65EEA55A6A
:1009900026EE066A66EEA66A002A7ED075EE860A04
:1009A000B7EE005A30EEA60A70EE077AC5EE277A47
:1009B000F1EE652A35EEC62A76EE651A32EEC61AD3
:1009C00072EE660A31EEE60A71EE266A30EE875A5A
:1009D00070EE075A36EE877A25EE276A65EEA74A4B
:1009E00027EE274A80ED006AC0ED044A80ED084AF0
:1009F000D1ED013A91ED023A91ED032AD1ED002AB1
:100A000063EE831A22EE221A71EE810A31EEC10AD8
:100A100030EEA05A70EE005A65EE276A25EEA76AFE
:100A2000C0ED036A80ED016A91ED017AD1ED034AD0
:100A3000D1ED023A91ED004A27EE243A63EE842A82
:100A400033EE622A73EE221A32EE021A71EEA10A16
:100A500021EE270A20EEA75A80ED060A80ED025A01
:100A6000D1ED025A91ED036A91ED017AD1ED006A60
:100A700065EE864A27EE264A74EE843A34EEC43A8E
:100A800073EEA32A33EE032A62EEA71A22EE271A88
:100A9000C0ED071A80ED051A7047F7EE007A87E778
:100AA00070B52DED088BD0ED039AD0ED008A90ED56
:100AB000018A90ED029A28EEA8AA69EEA9AA28EE6A
:100AC000A91A08EE091A7AEE6A1A29EE09BA68EE2E
:100AD00008BA71EECB0A31EE010A70EEAB0A0C4691
:100AE00015461E460BF0A4FF69EE287A58EE297AC7
:100AF00084ED000AB8EE000A27EE800A0BF0FEFE35
:100B000028EE288A09EE298A3AEE2AAA38EE088ABF
:100B10003AEE4BBA85ED000A3BEE6BBA88EE0B0A53
:100B20000BF0F0FE86ED000ABDEC088B70BD00BF37
:100B3000D2ED016A70B592ED005A26EEA66A05EE76
:100B4000056AD2ED025A2DED048B1446054605EEDA
:100B5000A56A0E46B0EE409AF1EEC68AB6EE008A5D
:100B600068EE888AB0EE680A0CF042FC20EE087A43
:100B7000D4ED007AC7EE280AD4ED014A94ED024A7A
:100B8000F1EE603A27EEA33A64EEA32A24EE232A7C
:100B900084ED003AC4ED012A84ED022A96ED018A23
:100BA000D6ED001A28EE088A01EEA18A96ED021A07
:100BB00001EE018A96ED030A00EE008AB0EE680AA3
:100BC0000CF07EF8F7EE006A48EE486A96ED011ADE
:100BD00026EE895AD4ED005A05EE090A96ED005A20
:100BE00061EE250A40EE050AD6ED025A94ED016A3F
:100BF00045EE860A94ED027A96ED036A46EE070A00
:100C000060EE013AC5ED000AD4ED007A47EEC53A30
:100C1000D4ED024A45EEE43A94ED014A46EE043A38
:100C2000C5ED013A94ED023AD4ED012A61EE031AC2
:100C300042EEC51A40EE251A94ED002A46EE421AFD
:100C4000C5ED021AD4ED016AD4ED020A61EE267AEE
:100C500050EEC57A94ED007A45EE877A40EE067A3A
:100C6000C5ED037ABDEC048B70BD00BF91ED002A89
:100C7000D0ED060A2DE9F04140EE020A2DED028B7F
:100C8000C2ED060AD1ED015A90ED074A00EE254A61
:100C90000E4682ED074AD1ED023AD0ED087A40EED9
:100CA000237A92B0C2ED087A91ED033AD0ED096A49
:100CB00040EE036A02F13008C2ED096AD6ED042A5B
:100CC00090ED0A1A00EE221A044682ED0A1AD6EDB9
:100CD000051AD0ED0B4A40EE214A1546C2ED0B4AEB
:100CE00093ED035A93ED047A93ED056A76EE850A47
:100CF00074EE867A31EE074A96ED062AD6ED075A4B
:100D0000D6ED083A74EE252A77EEA31A30EE823A31
:100D100022EE807A63EE006A21EE801A00F1300143
:100D20000FAA4046B0EE408A1F46CDED0F6A8DED0A
:100D3000107A8DED111AFFF7FBFE6846414601223D
:100D4000FFF71AFE97ED005AD5ED064A97ED012AF6
:100D5000D5ED070A97ED026A95ED084A75EE243A3B
:100D600072EE205A36EE043A0CA809A96A46CDED77
:100D7000093ACDED0A5A8DED0B3AFFF781FDD4ED1E
:100D8000007ADDED0C2A48EE227AD6ED0A1A37EE0B
:100D9000A14A9DED0D1A85ED004AD4ED016A48EE99
:100DA000016A96ED0B0A36EE801A9FED2C7A85EDDE
:100DB000011A9DED0E5A94ED022A75EE074AD6ED02
:100DC0000C0A08EE242A32EE202AF6EE000A85EDFF
:100DD000022AD4ED003A74EE235AD4ED032A25EE0C
:100DE000A06A96ED0D3A46EE082A72EE831AC5ED1A
:100DF000031AD4ED017A71EE276A94ED045A26EEB7
:100E0000A00A96ED0E7A00EE085A75EE074AC5ED77
:100E1000044A94ED024A72EE043A94ED053A63EE08
:100E2000A05A96ED0F6A05EEC83A73EE062AC5ED94
:100E3000052AD4ED021A32EE211A94ED100A61EE61
:100E4000207AD6ED096A07EEC80A30EE267A85EDDB
:100E5000107A12B0BDEC028BBDE8F0810AE81C41AB
:100E600070B541F62874C2F200042DED028BD4F85F
:100E70003C0430300146FFF7F7FBD4F83C0404F59E
:100E8000806504F581663030291D05F10C0332467A
:100E9000FFF706FE9FED168A95ED011A21EE080A6E
:100EA000F6F7DAFFD5ED036AF0EE400A96ED000A98
:100EB000DFED108A20EE087A26EE888A20EEA80A56
:100EC000C5ED010A86ED007A85ED038A0BF0F8FE88
:100ED000D5ED017A04F5826484ED000A27EEA80AB4
:100EE0000CF086FA84ED010ABDEC028B70BD00BFE8
:100EF000E02E654235FA8E3CF0B540F22013C1F287
:100F0000000341F62874D3F838C1D3F83C11D3F864
:100F10004071D3F82C61D3F83051D3F83421C2F2A8
:100F2000000487B08E462068CDF800C0694693ED76
:100F3000630A039604950592CDF804E0029704F045
:100F4000B9FFD4F83C24D4F80034D66804EB83010C
:100F50000E641569C1F8E0505069C1F88001D2F8FB
:100F600000C0C1F820C256680D4646F26760591CA1
:100F7000C6F26660C5F8C06280FB015CCE17C6EBA6
:100F80002C10956804EB830300EB8002A1EBC201F7
:100F9000C3F86053C4F8001407B0F0BD00B507EE05
:100FA000100A89B0F8EEC77A05AA08A941F6287C8C
:100FB00061ED017AC2F2000C01924CF2AC5340F2A6
:100FC000FD22C3F22773C0F60102059302920123AA
:100FD000DCF80000009306AA8DED060A05F058F92A
:100FE00009B000BD00B51B4989B0086804900590A0
:100FF000FFF7E6F941F62873C2F2000303F58862B1
:10100000D2ED007AF5EE407AF1EE10FA8DED060A97
:101010008DED070A18680ED140F2353204A9C0F6EA
:101020000102022301910292002106AA009305F019
:101030002FF909B000BD40F2213204A9C0F6010227
:10104000012301910292002106AA009305F020F9E4
:10105000EFE700BF1C07001041F6287CC2F2000C2D
:1010600010B5DCF83C2492ED074AD2ED063A30EE9A
:10107000842A70EE232A92ED086A22EE023A2DEDC0
:10108000028B02EEA23A71EE060A8AB000EEA03A96
:10109000F1EEC36AC2EEA61A40F2B424C1F2000413
:1010A00004F58C6104F58E6482EE267A80EEA61A31
:1010B0009FED1E0A30EE660A91ED038ACDED071A08
:1010C0008DED087A8DED091A0CF0DCF9D4ED007A7B
:1010D00041F69420C1F2000000EE278A90F8BC315E
:1010E0005B078DED048A05D4DFED114A28EE248AD2
:1010F0008DED048A41F6287EC2F2000E40F63501DD
:1011000004AAC0F60101DEF8000001920323029157
:1011100007AA00218DED058A8DED068A009305F062
:10112000B7F80AB0BDEC028B10BD00BF0AE81C4145
:101130006F12833A00B541F69420C1F20000204AB4
:1011400090F8BC31D2ED017A8BB05A07CDED047A1C
:1011500005D49FED1C7A67EE877ACDED047A60EEB8
:10116000A02A40EE002ACDED057ACDED067A41EEBB
:10117000012AB1EEE22AF7EE007AC7EE821A41F6B2
:10118000287CC2F2000C40F2E97104AAC0F6010109
:10119000032301920291DCF800000093002107AACA
:1011A00020EE210A60EEA10A21EE211A8DED070A38
:1011B000CDED080A8DED091A05F06AF80BB000BDF7
:1011C000240700106F12833AF0B5F1EE007A2DED8E
:1011D000088BB0EE40AAF0EE60AAB0EE41BAF0EE95
:1011E00061BAF4EEE72AF1EE10FA8BB0B0EE628A43
:1011F0000546F0EE428AB0EE439A40F1F98041F2A2
:101200006003C1F2000393ED1F0AB5EE400AF1EE50
:1012100010FA00F0ED8041F62874C2F20004D4E91F
:10122000086700223046394600230AF029FE0028CC
:1012300040F0158132463B4651EC1A0B0AF0E8FAB1
:10124000D4E90C230AF02AFC0AF0A6FAD4E90A230E
:10125000064651EC1B0B04960AF0DAFAD4E90E2389
:101260000AF01CFC0AF098FA4FF44062CDED068AB1
:10127000C4F2000240F220130590C1F20003D3ED46
:10128000636A05EE105A536A8749D4F800249FED2B
:10129000877AD1ED007AB8EE456A05EE903A26EEEF
:1012A000877A76EE277AF8EE656ABDEEC77A76EE33
:1012B000E77AB8EEC77A41F62874C7EE877AC2F2A9
:1012C0000004FDEEE77A17EE903AD31A48BF2833B0
:1012D000272B88BF002304EB8301D4F83C24D1EDF5
:1012E000106A03F13801603304EB830304EB8101DE
:1012F000D1ED005A93ED006AD2ED038AC2ED036A84
:101300000968D2ED049A1161196841F2600392ED07
:1013100005AAC1F200035161D3ED1F7A40F2B42255
:1013200067EEA77A93ED207AC1F2000202F5896197
:1013300079EEE59AF0EE675A78EEE68A3AEE46AA3A
:10134000D1ED006A47EE075AF1EEE55A02F58861E1
:1013500091ED036A68EE255AB0EE665A05EE865A9C
:1013600093ED217AF0EE455AB0EE675ACDED075A6B
:1013700007EE075AB1EEC57A28EE078A93ED1E7A7A
:1013800046EE086A47EE077ACDED086AF1EEE77A95
:1013900002F58A6292ED017A27EE899AD2ED007AFF
:1013A000032549EE077A2B46009507AD019540F2DB
:1013B00059352068002104AAC0F60105CDED097A4F
:1013C000029504F065FFD4F83C34D3ED036A93ED45
:1013D000047AD3ED057A76EEA88A77EE299A37EE6D
:1013E0008AAAC3ED038AC3ED049A83ED05AA2EE011
:1013F00041F6287EC2F2000E41F6942CDEF83C3411
:10140000C1F2000C196C9CF8BC0106910022410746
:10141000049205921FD44BF69573C3F2D63341F66E
:10142000287007930893C2F20000002340F259315C
:10143000C4F2C82307AAC0F601010068099301920B
:101440000323029104AA0021009304F021FF0BB0B2
:10145000BDEC088BF0BD0023C4F22013DFE7B0EE33
:101460004A0AF0EE6A0A84ED08AB84ED0ABBFEF787
:10147000CFFFB0EE4A0AF0EE6A0AB0EE4B1AF0EE79
:101480006B1AFFF78DF8D4F83C3493ED030AD3EDD3
:10149000040A93ED051AB1EE400AF1EE600A38EE47
:1014A000C11AFFF725F8D2E72C0700100024744971
:1014B00030B5F0EE007A2DED048BF4EEE71AF1EE84
:1014C00010FA8BB040F1D88041F26003C1F2000302
:1014D00093ED1F2AB5EE402AF1EE10FA00F0CC8011
:1014E0004FF4406C8DED040ACDED050A8DED061A22
:1014F000C4F2000C40F2201EC1F2000EDCF82430D1
:101500007849DEED636A08EE900A9FED771AD1ED17
:10151000030A26EE810AB8EE689A07EE103A79EED1
:10152000207AB8EE472ABDEEC05A32EE676AF8EE6E
:10153000C54A41F62872C6EE245AC2F20002D2F819
:101540000054BDEEE54A14EE104A2B1B48BF283369
:1015500041F62874C2F20004272B88BF002304EB55
:101560008300D4F83C54D0ED883A03F1B001D8336D
:1015700004EB810E04EB830295ED008ADEED002A78
:1015800092ED001AC5ED003ADEF800C0D5ED018AF3
:10159000C5F804C0106841F2600E95ED029AC1F2E0
:1015A000000EA8609EED1F3A40F2B42C23EE033AE1
:1015B000DEED200AC1F2000C0CF58B63F0EE436AFD
:1015C00038EE638A78EEE28AD3ED003A39EE419A3A
:1015D00040EEA06AB1EEE67A0CF58A6191ED036AFD
:1015E00021EE870AB0EE635A00EE065A9EED212ADC
:1015F000F0EE437A8DED075A42EE027AF1EEE74AB9
:1016000061EEA45A9EED1E4A46EE253A04EE043AD7
:10161000CDED083AF1EEC32A0CF58C6292ED011A79
:10162000D2ED000A61EEA21A032541EE810A20687C
:1016300000952B4607AD019540F28D35002104AA97
:10164000C0F60105CDED090A029504F021FED4F89B
:101650003C04D0ED006A90ED017A90ED020A36EE7E
:10166000888A77EE288A30EE099A80ED008AC0EDEC
:10167000018A80ED029A28E041F69422C1F200022C
:10168000002392F8BC01049340070593069320D4ED
:101690004BF6957CC3F2D63CCDF81CC0CDF820C0EB
:1016A000CDF824C041F6287EC2F2000E40F28D3201
:1016B00007A9C0F60102DEF800000191032302929F
:1016C000002104AA009304F0E3FD0BB0BDEC048BF1
:1016D00030BD0020C4F2A0004FF080410790089078
:1016E0000991DFE724070010002474492DE9F04F29
:1016F00041F62876C2F200062DED068BD6F83C8422
:10170000002740F22014C8F80070C8F80470C8F828
:101710000870C8F80C70C8F81070C1F20004D3B09B
:1017200094ED470AFEF74CFED6F83C544FF07E533A
:1017300088ED050AAF61EF612F626F62AF62EF6201
:101740002B636F63AF63EF6394ED470AFEF738FED8
:10175000142085ED100AFBF74BFA00273D46D4F81C
:101760008021D4F880019042FBD0D4F82CB1D4F879
:1017700030A1D4F83491D4F84401D4F84811D4F805
:101780004C21D4F83831D4F83C81D4F840E146F209
:10179000676C0AEE908A0AEE103AC6F2666C7B1C01
:1017A0008CFB03C84FEAE37CBF006AEEAA7ACCEB5D
:1017B000E80C0DF5A47803EE10EA4AEE0A7A08EB7D
:1017C000070E0DF1040847440CEB8C0CC7F800B071
:1017D0004EF8F4AC4EF8A49CA3EB8C0708EE900AEC
:1017E00009EE101A08EE102A43EE037AF1EEE79A9A
:1017F00069EE092A48EEA82A8AEE29AACAEEA9AA01
:1018000048EE082AC3EE299AB1EEE22AD6F83C1433
:10181000012230313DA8C8EE828A89EE029A88EE14
:10182000028AFFF7A9F846A845493DAAFFF766F8DE
:1018300006F1100149A83DAAFFF760F8DDED4A1A4C
:101840009DED4B1ADDED490A9DED460ADDED473A67
:101850009DED484A61EE094A20EE885A61EEA85A89
:1018600051EE884A64EE2A6A11EE285A20EE297A4F
:1018700050EE895A63EE8A7A53EEA96A14EE0A7A18
:1018800050EE2A7AB6EE006AD6F83C0454EEC66AE8
:1018900015EE467A55EEC67A303001464CAA9FEDD9
:1018A000290ACDED4C6A8DED4D7ACDED4E7AFFF7DC
:1018B0003FF9132D33DC0135642D7FF750AFDDED9B
:1018C000504A9DED4F5A9DED516A75EE245ADFED59
:1018D0001E6A35EE867AB4EEE67AF1EE10FA3FF73C
:1018E0003EAF41F62874C2F2000401A8D4F83C24AB
:1018F00014212432F6F718F9D4F83C2414212832A4
:1019000015A8F6F711F9D4F83C2429A82C32142193
:10191000F6F70AF953B0BDEC068BBDE8F08F01A8CD
:1019200014214FAAF6F784F9142150AA15A8F6F746
:101930007FF929A8142151AAF6F77AF9BBE700BF6D
:101940002C1F0020CDCCCC3D6F12833B2DE9F04FF6
:101950002DED068B41F62875C2F2000540F2B42445
:10196000A5B0C1F2000400214FF48A6228460BF0B2
:10197000CBFFDFED5F8AD4EDE82A9FED5E9A002071
:1019800022EEA80ACBF68070E86085ED019A85ED1D
:10199000029A0BF095F994EDE82AF0EE409A22EEC7
:1019A000280A0BF025FDD4EDE91AB0EE40AA21EE8D
:1019B000A80A0BF085F9D4EDE97A29EE808A27EEA2
:1019C000A80A0BF015FD00EE498A94EDE91A21EE04
:1019D000280A85ED048A0BF073F9D4EDE90AB0EE1C
:1019E000408A20EEA80A0BF003FD29EE800A08EEDB
:1019F000090A032140F66D4610220B46B1EE4AAAB1
:101A00001120C0F6010685ED050A009685ED06AAAF
:101A100004F054F80146296004F5816803F0C8FF1A
:101A200004F5806A04F5826C04F5846204F5836B26
:101A300004F58569DBF800E0DCF80C70D9F800608B
:101A4000DAF80CB0D8F80090DCF804A0DCF80080DC
:101A5000D2F804C01368D168CDF84CC004F5866292
:101A600004F5886C04F58764C5F83C04CDF824E0DF
:101A7000CDF828E0CDF82CE00C970D970E970F933A
:101A80001093119312931496159616961791189118
:101A9000CDF80C90CDF81090CDF814B0CDF818809A
:101AA000CDF81C80CDF820A019911168D668D2F825
:101AB00004E0DCF800202468DCF8047028681A913F
:101AC00000231B911C91239203A914AACDF874E062
:101AD00000931E961F9620972194229403F06AFF8C
:101AE000FFF704FE25B0BDEC068BBDE8F08F00BF0C
:101AF00035FA8E3C00000000F8B505460C46012082
:101B0000582116461F4606F03DFE0699079B089A87
:101B1000C161036209990A9B42628162C3620B9AA6
:101B20000C990D9B0561C460466187610263416346
:101B30008363F8BD0169C2684369F0EE407A91EDB4
:101B4000006A92ED007A002B00F0CD80D3ED005AB0
:101B50008369002B00F0CD80D3ED006AC36A5BB1CE
:101B6000B3F9003001EE103AB8EEC10A9FED625AA7
:101B700060EE064A04EE856A036B5BB1B3F90020A0
:101B800003EE102AF8EEC32A9FED5B2A62EE871A55
:101B900001EE827A436B5BB1B3F9001005EE101AC7
:101BA000F8EEC54A9FED544A65EEA43A43EE845AD6
:101BB000836B5BB1B3F900C002EE10CAF8EEC21A33
:101BC0009FED4D1A26EEA10A40EE016A37EEE05A6B
:101BD000C36926EE056A80ED126AD3ED004AB4EEC1
:101BE000E46AF1EE10FA6EDCF1EE644AB4EEE46AF7
:101BF000F1EE10FA67D490ED026A75EE062A026AD9
